 FarCmds

 Timestamp is 657a56ca (Thu Dec 14 01:13:46 2023)

 Preferred load address is 0000000180000000

 Start         Length     Name                   Class
 0001:00000000 00000ac8H .text                   CODE
 0001:00000ac8 00011c1cH .text$mn                CODE
 0001:000126e4 000005b8H .text$x                 CODE
 0002:00000000 00000360H .idata$5                DATA
 0002:00000360 00000008H .00cfg                  DATA
 0002:00000368 00000008H .CRT$XCA                DATA
 0002:00000370 00000008H .CRT$XCZ                DATA
 0002:00000378 00000008H .CRT$XIA                DATA
 0002:00000380 00000010H .CRT$XIC                DATA
 0002:00000390 00000008H .CRT$XIZ                DATA
 0002:00000398 00000008H .CRT$XPA                DATA
 0002:000003a0 00000010H .CRT$XPX                DATA
 0002:000003b0 00000008H .CRT$XPXA               DATA
 0002:000003b8 00000008H .CRT$XPZ                DATA
 0002:000003c0 00000008H .CRT$XTA                DATA
 0002:000003c8 00000008H .CRT$XTZ                DATA
 0002:000003d0 00000000H .gehcont$y              DATA
 0002:000003d0 00000000H .gfids$y                DATA
 0002:000003d0 000060b0H .rdata                  DATA
 0002:00006480 00000000H .rdata$CastGuardVftablesA DATA
 0002:00006480 00000000H .rdata$CastGuardVftablesC DATA
 0002:00006480 00000444H .rdata$r                DATA
 0002:000068c4 000002fcH .rdata$zzzdbg           DATA
 0002:00006bc0 00000008H .rtc$IAA                DATA
 0002:00006bc8 00000008H .rtc$IZZ                DATA
 0002:00006bd0 00000008H .rtc$TAA                DATA
 0002:00006bd8 00000008H .rtc$TZZ                DATA
 0002:00006be0 00000ce0H .xdata                  DATA
 0002:000078c0 00000150H .xdata$x                DATA
 0002:00007a10 000000a8H .edata                  DATA
 0002:00007ab8 00000064H .idata$2                DATA
 0002:00007b1c 00000014H .idata$3                DATA
 0002:00007b30 00000360H .idata$4                DATA
 0002:00007e90 000007aaH .idata$6                DATA
 0003:00000000 00000ae8H .data                   DATA
 0003:00000ae8 000000a8H .data$r                 DATA
 0003:00000b90 000000e0H .data$rs                DATA
 0003:00000c70 00005108H .bss                    DATA
 0004:00000000 00000a80H .pdata                  DATA
 0005:00000000 00000060H .rsrc$01                DATA
 0005:00000060 00000348H .rsrc$02                DATA

  Address         Publics by Value              Rva+Base               Lib:Object

 0000:00000000       __guard_fids_count         0000000000000000     <absolute>
 0000:00000000       __guard_longjmp_table      0000000000000000     <absolute>
 0000:00000000       __arm64x_extra_rfe_table   0000000000000000     <absolute>
 0000:00000000       ___safe_se_handler_table   0000000000000000     <absolute>
 0000:00000000       __x64_code_ranges_to_entry_points_count 0000000000000000     <absolute>
 0000:00000000       __hybrid_code_map          0000000000000000     <absolute>
 0000:00000000       __volatile_metadata        0000000000000000     <absolute>
 0000:00000000       __arm64x_extra_rfe_table_size 0000000000000000     <absolute>
 0000:00000000       ___safe_se_handler_count   0000000000000000     <absolute>
 0000:00000000       __arm64x_redirection_metadata 0000000000000000     <absolute>
 0000:00000000       __guard_iat_table          0000000000000000     <absolute>
 0000:00000000       __x64_code_ranges_to_entry_points 0000000000000000     <absolute>
 0000:00000000       __guard_iat_count          0000000000000000     <absolute>
 0000:00000000       __guard_longjmp_count      0000000000000000     <absolute>
 0000:00000000       __dynamic_value_reloc_table 0000000000000000     <absolute>
 0000:00000000       __guard_eh_cont_count      0000000000000000     <absolute>
 0000:00000000       __hybrid_auxiliary_iat     0000000000000000     <absolute>
 0000:00000000       __hybrid_auxiliary_iat_copy 0000000000000000     <absolute>
 0000:00000000       __AbsoluteZero             0000000000000000     <absolute>
 0000:00000000       __guard_check_icall_a64n_fptr 0000000000000000     <absolute>
 0000:00000000       __guard_fids_table         0000000000000000     <absolute>
 0000:00000000       __arm64x_redirection_metadata_count 0000000000000000     <absolute>
 0000:00000000       __enclave_config           0000000000000000     <absolute>
 0000:00000000       __guard_eh_cont_table      0000000000000000     <absolute>
 0000:00000000       __arm64x_native_entrypoint 0000000000000000     <absolute>
 0000:00000000       __hybrid_code_map_count    0000000000000000     <absolute>
 0000:00000100       __guard_flags              0000000000000100     <absolute>
 0000:00000000       __ImageBase                0000000180000000     <linker-defined>
 0001:00000000       __security_check_cookie    0000000180001000 f   LIBCMT:arm64secgs.obj
 0001:00000018       __gsfailure                0000000180001018 f   LIBCMT:arm64secgs.obj
 0001:00000048       _NLG_Notify                0000000180001048 f   libvcruntime:notify.obj
 0001:0000005c       __NLG_Dispatch2            000000018000105c     libvcruntime:notify.obj
 0001:00000064       __NLG_Return2              0000000180001064 f   libvcruntime:notify.obj
 0001:00000070       __C_ExecuteExceptionFilter 0000000180001070 f   libvcruntime:handler.obj
 0001:000000c4       __C_ExecuteTerminationHandler 00000001800010c4 f   libvcruntime:handler.obj
 0001:00000118       _CallSettingFrame          0000000180001118 f   libvcruntime:handlers.obj
 0001:000001c0       memmove                    00000001800011c0 f   libvcruntime:memcpy.obj
 0001:000001c0       memcpy                     00000001800011c0 f   libvcruntime:memcpy.obj
 0001:000001d0       __memcpy_forward           00000001800011d0     libvcruntime:memcpy.obj
 0001:000001d0       _memcpy_strict_align       00000001800011d0     libvcruntime:memcpy.obj
 0001:00000220       __memcpy_forward_large_neon 0000000180001220 f   libvcruntime:memcpy.obj
 0001:00000320       __memcpy_reverse           0000000180001320 f   libvcruntime:memcpy.obj
 0001:00000380       __memcpy_reverse_large_neon 0000000180001380 f   libvcruntime:memcpy.obj
 0001:000004a0       __security_push_cookie     00000001800014a0 f   LIBCMT:secpushpop.obj
 0001:000004c0       __security_pop_cookie      00000001800014c0 f   LIBCMT:secpushpop.obj
 0001:000004f0       __ppgsfailure              00000001800014f0 f   LIBCMT:secpushpop.obj
 0001:00000510       __chkstk                   0000000180001510 f   LIBCMT:chkstk.obj
 0001:00000510       _alloca_probe              0000000180001510 f   LIBCMT:chkstk.obj
 0001:00000540       memset                     0000000180001540 f   libvcruntime:memset.obj
 0001:000006e0       memcmp                     00000001800016e0 f   libvcruntime:memcmp.obj
 0001:00000ac8       ?SaveValue@PluginCheckBoxBinding@@UEAAXPEBUFarDialogItem@@H@Z 0000000180001ac8 f i FARCmds.obj
 0001:00000b68       ??_EPluginCheckBoxBinding@@UEAAPEAXI@Z 0000000180001b68 f i * CIL library *:* CIL module *
 0001:00000b68       ??_GPluginCheckBoxBinding@@UEAAPEAXI@Z 0000000180001b68 f i FARCmds.obj
 0001:00000b90       ?SaveValue@PluginRadioButtonBinding@@UEAAXPEBUFarDialogItem@@H@Z 0000000180001b90 f i FARCmds.obj
 0001:00000bd8       ??_EPluginRadioButtonBinding@@UEAAPEAXI@Z 0000000180001bd8 f i * CIL library *:* CIL module *
 0001:00000bd8       ??_GPluginRadioButtonBinding@@UEAAPEAXI@Z 0000000180001bd8 f i FARCmds.obj
 0001:00000c00       ?SaveValue@PluginUIntEditFieldBinding@@UEAAXPEBUFarDialogItem@@H@Z 0000000180001c00 f i FARCmds.obj
 0001:00000c50       ??_GPluginUIntEditFieldBinding@@UEAAPEAXI@Z 0000000180001c50 f i FARCmds.obj
 0001:00000c50       ??_EPluginUIntEditFieldBinding@@UEAAPEAXI@Z 0000000180001c50 f i * CIL library *:* CIL module *
 0001:00000c78       ?AddCheckbox@PluginDialogBuilder@@QEAAPEAUFarDialogItem@@HPEAHH_N@Z 0000000180001c78 f i FARCmds.obj
 0001:00000dd0       ?AddOKCancel@PluginDialogBuilder@@QEAAXHHH_N@Z 0000000180001dd0 f i FARCmds.obj
 0001:00000f98       ?ShowDialogEx@PluginDialogBuilder@@QEAA_JXZ 0000000180001f98 f i FARCmds.obj
 0001:00001120       ?AddDialogItem@PluginDialogBuilder@@AEAAPEAUFarDialogItem@@W4FARDIALOGITEMTYPES@@PEB_W@Z 0000000180002120 f i FARCmds.obj
 0001:000012c0       ?UpdateBorderSize@PluginDialogBuilder@@AEAAXXZ 00000001800022c0 f i FARCmds.obj
 0001:00001480       GetGlobalInfoW             0000000180002480 f   FARCmds.obj
 0001:00001518       SetStartupInfoW            0000000180002518 f   FARCmds.obj
 0001:00001790       OpenW                      0000000180002790 f   FARCmds.obj
 0001:00001a58       GetPluginInfoW             0000000180002a58 f   FARCmds.obj
 0001:00001ac8       ConfigureW                 0000000180002ac8 f   FARCmds.obj
 0001:00002408       ?ExpandEnv@@YAPEA_WPEB_WPEAK@Z 0000000180003408 f   Mix.obj
 0001:00002468       ?GetInt@@YAHPEB_WPEA_W@Z   0000000180003468 f   Mix.obj
 0001:00002698       ?ProcessOSAliases@@YAPEA_WPEB_W@Z 0000000180003698 f   Mix.obj
 0001:00002b70       ?GetShellLinkPath@@YAPEA_WPEB_W@Z 0000000180003b70 f   Mix.obj
 0001:00002ea8       ?GetCPBuffer@@YAIPEBX_KPEA_K@Z 0000000180003ea8 f   Mix.obj
 0001:00003018       ?ConvertBuffer@@YAPEA_WPEA_W_KHAEA_KPEA_N@Z 0000000180004018 f   Mix.obj
 0001:00003178       ??1ConsoleTitle@@QEAA@XZ   0000000180004178 f i OpenCmd.obj
 0001:000031b0       ??0MakeVETitle@@QEAA@PEB_W0@Z 00000001800041b0 f i OpenCmd.obj
 0001:00003258       ??1MakeVETitle@@QEAA@XZ    0000000180004258 f i OpenCmd.obj
 0001:00004308       ?__proc_WhereIs@@YAPEA_WHPEA_W_N@Z 0000000180005308 f   OpenCmd.obj
 0001:00004968       ?__proc_Link@@YA_NHPEA_W@Z 0000000180005968 f   OpenCmd.obj
 0001:00004c08       ?OpenFromCommandLine@@YAPEA_WPEB_W@Z 0000000180005c08 f   OpenCmd.obj
 0001:000061c0       ??_V@YAXPEAX@Z             00000001800071c0 f   LIBCMT:delete_array.obj
 0001:000061c0       ??3@YAXPEAX_K@Z            00000001800071c0 f   LIBCMT:delete_scalar_size.obj
 0001:000061c8       ??2@YAPEAX_K@Z             00000001800071c8 f   LIBCMT:new_scalar.obj
 0001:00006210       ??_U@YAPEAX_K@Z            0000000180007210 f   LIBCMT:new_array.obj
 0001:00006218       ??_Etype_info@@UEAAPEAXI@Z 0000000180007218 f i LIBCMT:std_type_info_static.obj
 0001:00006218       ??_Gtype_info@@UEAAPEAXI@Z 0000000180007218 f i LIBCMT:std_type_info_static.obj
 0001:00006618       _DllMainCRTStartup         0000000180007618 f   LIBCMT:dll_dllmain.obj
 0001:00006660       __report_gsfailure         0000000180007660 f   LIBCMT:gs_report.obj
 0001:00006678       __report_rangecheckfailure 0000000180007678 f   LIBCMT:gs_report.obj
 0001:00006690       __report_securityfailure   0000000180007690 f   LIBCMT:gs_report.obj
 0001:000066a8       ??3@YAXPEAX@Z              00000001800076a8 f   LIBCMT:delete_scalar.obj
 0001:000066b0       ??0bad_alloc@std@@QEAA@AEBV01@@Z 00000001800076b0 f i LIBCMT:throw_bad_alloc.obj
 0001:00006700       ??0bad_alloc@std@@QEAA@XZ  0000000180007700 f i LIBCMT:throw_bad_alloc.obj
 0001:00006720       ??0bad_array_new_length@std@@QEAA@AEBV01@@Z 0000000180007720 f i LIBCMT:throw_bad_alloc.obj
 0001:00006770       ??0bad_array_new_length@std@@QEAA@XZ 0000000180007770 f i LIBCMT:throw_bad_alloc.obj
 0001:00006790       ??0exception@std@@QEAA@AEBV01@@Z 0000000180007790 f i LIBCMT:throw_bad_alloc.obj
 0001:000067d0       ??1bad_exception@std@@UEAA@XZ 00000001800077d0 f i libvcruntime:frame.obj
 0001:000067d0       ??1bad_array_new_length@std@@UEAA@XZ 00000001800077d0 f i LIBCMT:throw_bad_alloc.obj
 0001:000067d0       ??1bad_alloc@std@@UEAA@XZ  00000001800077d0 f i LIBCMT:throw_bad_alloc.obj
 0001:000067e0       ??_Gbad_exception@std@@UEAAPEAXI@Z 00000001800077e0 f i libvcruntime:frame.obj
 0001:000067e0       ??_Ebad_array_new_length@std@@UEAAPEAXI@Z 00000001800077e0 f i LIBCMT:throw_bad_alloc.obj
 0001:000067e0       ??_Ebad_exception@std@@UEAAPEAXI@Z 00000001800077e0 f i libvcruntime:frame.obj
 0001:000067e0       ??_Gbad_alloc@std@@UEAAPEAXI@Z 00000001800077e0 f i LIBCMT:throw_bad_alloc.obj
 0001:000067e0       ??_Gexception@std@@UEAAPEAXI@Z 00000001800077e0 f i LIBCMT:throw_bad_alloc.obj
 0001:000067e0       ??_Gbad_array_new_length@std@@UEAAPEAXI@Z 00000001800077e0 f i LIBCMT:throw_bad_alloc.obj
 0001:000067e0       ??_Eexception@std@@UEAAPEAXI@Z 00000001800077e0 f i LIBCMT:throw_bad_alloc.obj
 0001:000067e0       ??_Ebad_alloc@std@@UEAAPEAXI@Z 00000001800077e0 f i LIBCMT:throw_bad_alloc.obj
 0001:00006828       ?__scrt_throw_std_bad_alloc@@YAXXZ 0000000180007828 f   LIBCMT:throw_bad_alloc.obj
 0001:00006848       ?__scrt_throw_std_bad_array_new_length@@YAXXZ 0000000180007848 f   LIBCMT:throw_bad_alloc.obj
 0001:00006868       ?what@exception@std@@UEBAPEBDXZ 0000000180007868 f i LIBCMT:throw_bad_alloc.obj
 0001:00006880       __security_init_cookie     0000000180007880 f   LIBCMT:gs_support.obj
 0001:00006970       __acrt_uninitialize_command_line 0000000180007970 f   libucrt:argv_data.obj
 0001:00006970       DllMain                    0000000180007970 f   LIBCMT:dll_dllmain_stub.obj
 0001:00006970       _get_startup_argv_mode     0000000180007970 f   LIBCMT:argv_mode.obj
 0001:00006978       ?__scrt_initialize_type_info@@YAXXZ 0000000180007978 f   LIBCMT:tncleanup.obj
 0001:00006990       ?__scrt_uninitialize_type_info@@YAXXZ 0000000180007990 f   LIBCMT:tncleanup.obj
 0001:000069a0       __local_stdio_printf_options 00000001800079a0 f i LIBCMT:default_local_stdio_options.obj
 0001:000069b0       __local_stdio_scanf_options 00000001800079b0 f i LIBCMT:default_local_stdio_options.obj
 0001:000069c0       __scrt_initialize_default_local_stdio_options 00000001800079c0 f   LIBCMT:default_local_stdio_options.obj
 0001:000069f8       __scrt_acquire_startup_lock 00000001800079f8 f   LIBCMT:utility.obj
 0001:00006a68       __scrt_dllmain_after_initialize_c 0000000180007a68 f   LIBCMT:utility.obj
 0001:00006aa8       __scrt_dllmain_before_initialize_c 0000000180007aa8 f   LIBCMT:utility.obj
 0001:00006ad0       __scrt_dllmain_crt_thread_attach 0000000180007ad0 f   LIBCMT:utility.obj
 0001:00006b10       __scrt_dllmain_crt_thread_detach 0000000180007b10 f   LIBCMT:utility.obj
 0001:00006b30       __scrt_dllmain_exception_filter 0000000180007b30 f   LIBCMT:utility.obj
 0001:00006bb0       __scrt_dllmain_uninitialize_c 0000000180007bb0 f   LIBCMT:utility.obj
 0001:00006be8       __scrt_dllmain_uninitialize_critical 0000000180007be8 f   LIBCMT:utility.obj
 0001:00006c08       __scrt_initialize_crt      0000000180007c08 f   LIBCMT:utility.obj
 0001:00006c68       __scrt_initialize_onexit_tables 0000000180007c68 f   LIBCMT:utility.obj
 0001:00006d08       __scrt_is_nonwritable_in_current_image 0000000180007d08 f   LIBCMT:utility.obj
 0001:00006dd8       __scrt_release_startup_lock 0000000180007dd8 f   LIBCMT:utility.obj
 0001:00006e10       __scrt_uninitialize_crt    0000000180007e10 f   LIBCMT:utility.obj
 0001:00006e58       __scrt_get_dyn_tls_init_callback 0000000180007e58 f   LIBCMT:dyn_tls_init.obj
 0001:00006e68       __scrt_fastfail            0000000180007e68 f   LIBCMT:utility_desktop.obj
 0001:00006e68       _invoke_watson             0000000180007e68 f   libucrt:invalid_parameter.obj
 0001:00006e70       _RTC_Initialize            0000000180007e70 f   LIBCMT:initsect.obj
 0001:00006ed8       _RTC_Terminate             0000000180007ed8 f   LIBCMT:initsect.obj
 0001:00006f40       _guard_check_icall_nop     0000000180007f40 f i LIBCMT:guard_support.obj
 0001:00006f48       __isa_available_init       0000000180007f48 f   LIBCMT:cpu_disp.obj
 0001:00006f50       __scrt_is_ucrt_dll_in_use  0000000180007f50 f   LIBCMT:ucrt_detection.obj
 0001:00006f68       ??$_CallSETranslator@V__FrameHandler3@@@@YAHPEAUEHExceptionRecord@@PEA_KPEAU_CONTEXT@@PEAU_xDISPATCHER_CONTEXT@@PEBU_s_FuncInfo@@K1H@Z 0000000180007f68 f i libvcruntime:risctrnsctrl.obj
 0001:00006fd8       ?CatchTryBlock@__FrameHandler3@@SAPEBU_s_TryBlockMapEntry@@PEBU_s_FuncInfo@@H@Z 0000000180007fd8 f   libvcruntime:risctrnsctrl.obj
 0001:00007048       ?ExecutionInCatch@__FrameHandler3@@SA_NPEAU_xDISPATCHER_CONTEXT@@PEBU_s_FuncInfo@@@Z 0000000180008048 f   libvcruntime:risctrnsctrl.obj
 0001:00007088       ?FrameUnwindToEmptyState@__FrameHandler3@@SAXPEA_KPEAU_xDISPATCHER_CONTEXT@@PEBU_s_FuncInfo@@@Z 0000000180008088 f   libvcruntime:risctrnsctrl.obj
 0001:000070f8       ?GetEstablisherFrame@__FrameHandler3@@SAPEA_KPEA_KPEAU_xDISPATCHER_CONTEXT@@PEBU_s_FuncInfo@@0@Z 00000001800080f8 f   libvcruntime:risctrnsctrl.obj
 0001:00007200       ?GetRangeOfTrysToCheck@__FrameHandler3@@SA?AU?$pair@Viterator@TryBlockMap@__FrameHandler3@@V123@@std@@AEAVTryBlockMap@1@HPEAU_xDISPATCHER_CONTEXT@@PEBU_s_FuncInfo@@H@Z 0000000180008200 f   libvcruntime:risctrnsctrl.obj
 0001:00007360       ?UnwindNestedFrames@__FrameHandler3@@SAXPEA_KPEAUEHExceptionRecord@@PEAU_CONTEXT@@0PEAXPEBU_s_FuncInfo@@HHPEBU_s_HandlerType@@PEAU_xDISPATCHER_CONTEXT@@E@Z 0000000180008360 f   libvcruntime:risctrnsctrl.obj
 0001:00007410       _CreateFrameInfo           0000000180008410 f   libvcruntime:risctrnsctrl.obj
 0001:00007460       _FindAndUnlinkFrame        0000000180008460 f   libvcruntime:risctrnsctrl.obj
 0001:000074c0       _GetImageBase              00000001800084c0 f   libvcruntime:risctrnsctrl.obj
 0001:000074d8       _GetThrowImageBase         00000001800084d8 f   libvcruntime:risctrnsctrl.obj
 0001:000074f0       _SetImageBase              00000001800084f0 f   libvcruntime:risctrnsctrl.obj
 0001:00007518       _SetThrowImageBase         0000000180008518 f   libvcruntime:risctrnsctrl.obj
 0001:00007540       __CxxFrameHandler3         0000000180008540 f   libvcruntime:risctrnsctrl.obj
 0001:000075c0       __DestructExceptionObject  00000001800085c0 f   libvcruntime:ehhelpers.obj
 0001:00007678       ?_CallMemberFunction0@@YAXQEAX0@Z 0000000180008678 f i libvcruntime:ehhelpers.obj
 0001:00007680       _IsExceptionObjectToBeDestroyed 0000000180008680 f   libvcruntime:ehhelpers.obj
 0001:000076c8       __AdjustPointer            00000001800086c8 f   libvcruntime:ehhelpers.obj
 0001:000076f0       __FrameUnwindFilter        00000001800086f0 f   libvcruntime:ehhelpers.obj
 0001:00007788       __std_terminate            0000000180008788 f   libvcruntime:ehhelpers.obj
 0001:00007790       wcschr                     0000000180008790 f   libvcruntime:wcschr.obj
 0001:00007978       wcsstr                     0000000180008978 f   libvcruntime:wcsstr.obj
 0001:00007a98       __C_specific_handler       0000000180008a98 f   libvcruntime:riscchandler.obj
 0001:00007d40       __std_exception_copy       0000000180008d40 f   libvcruntime:std_exception.obj
 0001:00007dd8       __std_exception_destroy    0000000180008dd8 f   libvcruntime:std_exception.obj
 0001:00007e10       _CxxThrowException         0000000180008e10 f   libvcruntime:throw.obj
 0001:00007ee8       __std_type_info_compare    0000000180008ee8 f   libvcruntime:std_type_info.obj
 0001:00007f08       __std_type_info_destroy_list 0000000180008f08 f   libvcruntime:std_type_info.obj
 0001:00007f48       __vcrt_initialize          0000000180008f48 f   libvcruntime:initialization.obj
 0001:00007f88       __vcrt_thread_attach       0000000180008f88 f   libvcruntime:initialization.obj
 0001:00007fa8       __vcrt_thread_detach       0000000180008fa8 f   libvcruntime:initialization.obj
 0001:00007fc8       __vcrt_uninitialize        0000000180008fc8 f   libvcruntime:initialization.obj
 0001:00007ff0       __vcrt_uninitialize_critical 0000000180008ff0 f   libvcruntime:initialization.obj
 0001:00008008       __vcrt_freefls             0000000180009008 f   libvcruntime:per_thread_data.obj
 0001:00008028       __vcrt_freeptd             0000000180009028 f   libvcruntime:per_thread_data.obj
 0001:000080a0       __vcrt_getptd              00000001800090a0 f   libvcruntime:per_thread_data.obj
 0001:000080c0       __vcrt_getptd_noexit       00000001800090c0 f   libvcruntime:per_thread_data.obj
 0001:000081d8       __vcrt_initialize_ptd      00000001800091d8 f   libvcruntime:per_thread_data.obj
 0001:00008250       __vcrt_uninitialize_ptd    0000000180009250 f   libvcruntime:per_thread_data.obj
 0001:00008298       ?GetCurrentState@__FrameHandler3@@SAHPEA_KPEAU_xDISPATCHER_CONTEXT@@PEBU_s_FuncInfo@@@Z 0000000180009298 f   libvcruntime:ehstate.obj
 0001:000082c0       ?GetUnwindTryBlock@__FrameHandler3@@SAHPEA_KPEAU_xDISPATCHER_CONTEXT@@PEBU_s_FuncInfo@@@Z 00000001800092c0 f   libvcruntime:ehstate.obj
 0001:000082f8       ?SetState@__FrameHandler3@@SAXPEA_KPEBU_s_FuncInfo@@H@Z 00000001800092f8 f   libvcruntime:ehstate.obj
 0001:00008308       ?SetUnwindTryBlock@__FrameHandler3@@SAXPEA_KPEAU_xDISPATCHER_CONTEXT@@PEBU_s_FuncInfo@@H@Z 0000000180009308 f   libvcruntime:ehstate.obj
 0001:00008350       ?StateFromControlPc@__FrameHandler3@@SAHPEBU_s_FuncInfo@@PEAU_xDISPATCHER_CONTEXT@@@Z 0000000180009350 f   libvcruntime:ehstate.obj
 0001:00008358       ?StateFromIp@__FrameHandler3@@SAHPEBU_s_FuncInfo@@PEAU_xDISPATCHER_CONTEXT@@_K@Z 0000000180009358 f   libvcruntime:ehstate.obj
 0001:00008f00       ??$TypeMatchHelper@V__FrameHandler3@@@@YAHPEBU_s_HandlerType@@PEBU_s_CatchableType@@PEBU_s_ThrowInfo@@@Z 0000000180009f00 f i libvcruntime:frame.obj
 0001:00009020       ??$__InternalCxxFrameHandler@V__FrameHandler3@@@@YA?AW4_EXCEPTION_DISPOSITION@@PEAUEHExceptionRecord@@PEA_KPEAU_CONTEXT@@PEAU_xDISPATCHER_CONTEXT@@PEBU_s_FuncInfo@@H1E@Z 000000018000a020 f i libvcruntime:frame.obj
 0001:000092a8       ??0bad_exception@std@@QEAA@AEBV01@@Z 000000018000a2a8 f i libvcruntime:frame.obj
 0001:000092f8       ??0bad_exception@std@@QEAA@XZ 000000018000a2f8 f i libvcruntime:frame.obj
 0001:00009318       ?CxxCallCatchBlock@__FrameHandler3@@SAPEAXPEAU_EXCEPTION_RECORD@@@Z 000000018000a318 f   libvcruntime:frame.obj
 0001:000095e8       ?FrameUnwindToState@__FrameHandler3@@SAXPEA_KPEAU_xDISPATCHER_CONTEXT@@PEBU_s_FuncInfo@@H@Z 000000018000a5e8 f   libvcruntime:frame.obj
 0001:000097c8       ?GetHandlerSearchState@__FrameHandler3@@SAHPEA_KPEAU_xDISPATCHER_CONTEXT@@PEBU_s_FuncInfo@@@Z 000000018000a7c8 f i libvcruntime:frame.obj
 0001:00009960       ?_CallMemberFunction1@@YAXQEAX00@Z 000000018000a960 f i libvcruntime:frame.obj
 0001:00009970       ?_CallMemberFunction2@@YAXQEAX00H@Z 000000018000a970 f i libvcruntime:frame.obj
 0001:00009980       __vcrt_initialize_locks    000000018000a980 f   libvcruntime:locks.obj
 0001:000099d8       __vcrt_uninitialize_locks  000000018000a9d8 f   libvcruntime:locks.obj
 0001:00009a48       __except_validate_context_record 000000018000aa48 f   libvcruntime:jbcxrval.obj
 0001:00009a88       free                       000000018000aa88 f   libucrt:free.obj
 0001:00009aa0       malloc                     000000018000aaa0 f   libucrt:malloc.obj
 0001:00009aa8       realloc                    000000018000aaa8 f   libucrt:realloc.obj
 0001:00009ab0       ??0_LocaleUpdate@@QEAA@QEAU__crt_locale_pointers@@@Z 000000018000aab0 f i libucrt:memicmp.obj
 0001:00009b50       __ascii_memicmp            000000018000ab50 f   libucrt:memicmp.obj
 0001:00009ba8       _memicmp                   000000018000aba8 f   libucrt:memicmp.obj
 0001:00009c00       _memicmp_l                 000000018000ac00 f   libucrt:memicmp.obj
 0001:00009cb0       wcsncmp                    000000018000acb0 f   libucrt:wcsncmp.obj
 0001:00009cf8       __acrt_initialize_new_handler 000000018000acf8 f   libucrt:new_handler.obj
 0001:00009d08       _callnewh                  000000018000ad08 f   libucrt:new_handler.obj
 0001:00009d58       _query_new_handler         000000018000ad58 f   libucrt:new_handler.obj
 0001:00009da0       _initterm                  000000018000ada0 f   libucrt:initterm.obj
 0001:00009e10       _initterm_e                000000018000ae10 f   libucrt:initterm.obj
 0001:00009e70       _seh_filter_dll            000000018000ae70 f   libucrt:exception_filter.obj
 0001:00009e98       _seh_filter_exe            000000018000ae98 f   libucrt:exception_filter.obj
 0001:0000a410       __acrt_initialize_thread_local_exit_callback 000000018000b410 f   libucrt:exit.obj
 0001:0000a420       _cexit                     000000018000b420 f   libucrt:exit.obj
 0001:0000a430       _exit                      000000018000b430 f   libucrt:exit.obj
 0001:0000a440       _is_c_termination_complete 000000018000b440 f   libucrt:exit.obj
 0001:0000a6a0       __acrt_allocate_buffer_for_argv 000000018000b6a0 f   libucrt:argv_parsing.obj
 0001:0000a710       _configure_narrow_argv     000000018000b710 f   libucrt:argv_parsing.obj
 0001:0000ab00       __dcrt_uninitialize_environments_nolock 000000018000bb00 f   libucrt:environment_initialization.obj
 0001:0000ab90       _initialize_narrow_environment 000000018000bb90 f   libucrt:environment_initialization.obj
 0001:0000ad28       _execute_onexit_table      000000018000bd28 f   libucrt:onexit.obj
 0001:0000ad68       _initialize_onexit_table   000000018000bd68 f   libucrt:onexit.obj
 0001:0000af30       __acrt_initialize          000000018000bf30 f   libucrt:initialization.obj
 0001:0000af58       __acrt_thread_attach       000000018000bf58 f   libucrt:initialization.obj
 0001:0000af78       __acrt_thread_detach       000000018000bf78 f   libucrt:initialization.obj
 0001:0000af90       __acrt_uninitialize        000000018000bf90 f   libucrt:initialization.obj
 0001:0000afd8       __acrt_uninitialize_critical 000000018000bfd8 f   libucrt:initialization.obj
 0001:0000aff8       terminate                  000000018000bff8 f   libucrt:terminate.obj
 0001:0000b030       swab                       000000018000c030 f   libucrt:swab.obj
 0001:0000b030       _swab                      000000018000c030 f   libucrt:swab.obj
 0001:0000b098       abort                      000000018000c098 f   libucrt:abort.obj
 0001:0000b0c8       strcmp                     000000018000c0c8 f   libucrt:strcmp.obj
 0001:0000b108       strcpy_s                   000000018000c108 f   libucrt:strcpy_s.obj
 0001:0000b188       calloc                     000000018000c188 f   libucrt:calloc.obj
 0001:0000b190       _free_base                 000000018000c190 f   libucrt:free_base.obj
 0001:0000b1f0       _malloc_base               000000018000c1f0 f   libucrt:malloc_base.obj
 0001:0000b290       _realloc_base              000000018000c290 f   libucrt:realloc_base.obj
 0001:0000b358       __acrt_initialize_invalid_parameter_handler 000000018000c358 f   libucrt:invalid_parameter.obj
 0001:0000b368       _invalid_parameter         000000018000c368 f   libucrt:invalid_parameter.obj
 0001:0000b418       _invalid_parameter_noinfo  000000018000c418 f   libucrt:invalid_parameter.obj
 0001:0000b430       __acrt_errno_from_os_error 000000018000c430 f   libucrt:errno.obj
 0001:0000b498       __acrt_errno_map_os_error  000000018000c498 f   libucrt:errno.obj
 0001:0000b4f8       __doserrno                 000000018000c4f8 f   libucrt:errno.obj
 0001:0000b520       _errno                     000000018000c520 f   libucrt:errno.obj
 0001:0000b938       __acrt_freeptd             000000018000c938 f   libucrt:per_thread_data.obj
 0001:0000b988       __acrt_getptd              000000018000c988 f   libucrt:per_thread_data.obj
 0001:0000ba78       __acrt_getptd_head         000000018000ca78 f   libucrt:per_thread_data.obj
 0001:0000bb30       __acrt_getptd_noexit       000000018000cb30 f   libucrt:per_thread_data.obj
 0001:0000bc18       __acrt_initialize_ptd      000000018000cc18 f   libucrt:per_thread_data.obj
 0001:0000bc68       __acrt_uninitialize_ptd    000000018000cc68 f   libucrt:per_thread_data.obj
 0001:0000bca0       __acrt_update_locale_info  000000018000cca0 f   libucrt:locale_update.obj
 0001:0000bcf0       __acrt_update_multibyte_info 000000018000ccf0 f   libucrt:locale_update.obj
 0001:0000bdc0       __acrt_set_locale_changed  000000018000cdc0 f   libucrt:wsetlocale.obj
 0001:0000bdd8       __acrt_uninitialize_locale 000000018000cdd8 f   libucrt:wsetlocale.obj
 0001:0000be08       __acrt_initialize_locks    000000018000ce08 f   libucrt:locks.obj
 0001:0000be80       __acrt_lock                000000018000ce80 f   libucrt:locks.obj
 0001:0000bea8       __acrt_uninitialize_locks  000000018000cea8 f   libucrt:locks.obj
 0001:0000bf18       __acrt_unlock              000000018000cf18 f   libucrt:locks.obj
 0001:0000bf40       __acrt_get_process_end_policy 000000018000cf40 f   libucrt:win_policies.obj
 0001:0000bf88       _calloc_base               000000018000cf88 f   libucrt:calloc_base.obj
 0001:0000c058       ??$__acrt_mbs_to_wcs_cp@U__crt_win32_buffer_internal_dynamic_resizing@@@@YAHQEBDAEAV?$__crt_win32_buffer@_WU__crt_win32_buffer_internal_dynamic_resizing@@@@I@Z 000000018000d058 f i libucrt:argv_wildcards.obj
 0001:0000c1e0       ??$__acrt_wcs_to_mbs_cp@U__crt_win32_buffer_internal_dynamic_resizing@@@@YAHQEB_WAEAV?$__crt_win32_buffer@DU__crt_win32_buffer_internal_dynamic_resizing@@@@I@Z 000000018000d1e0 f i libucrt:argv_wildcards.obj
 0001:0000cab0       __acrt_expand_narrow_argv_wildcards 000000018000dab0 f   libucrt:argv_wildcards.obj
 0001:0000cab8       ??$__acrt_wcs_to_mbs_cp@U__crt_win32_buffer_no_resizing@@@@YAHQEB_WAEAV?$__crt_win32_buffer@DU__crt_win32_buffer_no_resizing@@@@I@Z 000000018000dab8 f i libucrt:getmodulefilenamea.obj
 0001:0000cbe0       __acrt_GetModuleFileNameA  000000018000dbe0 f   libucrt:getmodulefilenamea.obj
 0001:0000d408       __acrt_initialize_multibyte 000000018000e408 f   libucrt:mbctype.obj
 0001:0000d478       __acrt_update_thread_multibyte_data 000000018000e478 f   libucrt:mbctype.obj
 0001:0000d498       _setmbcp_nolock            000000018000e498 f   libucrt:mbctype.obj
 0001:0000d7c0       _ismbblead                 000000018000e7c0 f   libucrt:ismbbyte.obj
 0001:0000d7d8       __acrt_initialize_command_line 000000018000e7d8 f   libucrt:argv_data.obj
 0001:0000d820       __acrt_MultiByteToWideChar 000000018000e820 f   libucrt:multibytetowidechar.obj
 0001:0000d8a8       __acrt_WideCharToMultiByte 000000018000e8a8 f   libucrt:widechartomultibyte.obj
 0001:0000d950       __dcrt_get_narrow_environment_from_os 000000018000e950 f   libucrt:get_environment_from_os.obj
 0001:0000da78       _recalloc_base             000000018000ea78 f   libucrt:recalloc.obj
 0001:0000dd40       __acrt_AppPolicyGetProcessTerminationMethodInternal 000000018000ed40 f   libucrt:winapi_thunks.obj
 0001:0000ddb0       __acrt_AreFileApisANSI     000000018000edb0 f   libucrt:winapi_thunks.obj
 0001:0000de08       __acrt_FlsAlloc            000000018000ee08 f   libucrt:winapi_thunks.obj
 0001:0000de78       __acrt_FlsFree             000000018000ee78 f   libucrt:winapi_thunks.obj
 0001:0000dee8       __acrt_FlsGetValue         000000018000eee8 f   libucrt:winapi_thunks.obj
 0001:0000df58       __acrt_FlsSetValue         000000018000ef58 f   libucrt:winapi_thunks.obj
 0001:0000dfe0       __acrt_InitializeCriticalSectionEx 000000018000efe0 f   libucrt:winapi_thunks.obj
 0001:0000e070       __acrt_LCMapStringEx       000000018000f070 f   libucrt:winapi_thunks.obj
 0001:0000e168       __acrt_LocaleNameToLCID    000000018000f168 f   libucrt:winapi_thunks.obj
 0001:0000e1e0       __acrt_initialize_winapi_thunks 000000018000f1e0 f   libucrt:winapi_thunks.obj
 0001:0000e220       __acrt_uninitialize_winapi_thunks 000000018000f220 f   libucrt:winapi_thunks.obj
 0001:0000e288       __acrt_initialize_heap     000000018000f288 f   libucrt:heap_handle.obj
 0001:0000e2b8       __acrt_uninitialize_heap   000000018000f2b8 f   libucrt:heap_handle.obj
 0001:0000e510       __acrt_initialize_lowio    000000018000f510 f   libucrt:ioinit.obj
 0001:0000e558       __acrt_uninitialize_lowio  000000018000f558 f   libucrt:ioinit.obj
 0001:0000e5a0       __acrt_execute_initializers 000000018000f5a0 f   libucrt:shared_initialization.obj
 0001:0000e660       __acrt_execute_uninitializers 000000018000f660 f   libucrt:shared_initialization.obj
 0001:0000e778       __acrt_get_sigabrt_handler 000000018000f778 f   libucrt:signal.obj
 0001:0000e7a8       __acrt_initialize_signal_handlers 000000018000f7a8 f   libucrt:signal.obj
 0001:0000e7c0       raise                      000000018000f7c0 f   libucrt:signal.obj
 0001:0000ea30       __acrt_initialize_user_matherr 000000018000fa30 f   libucrt:matherr.obj
 0001:0000ec58       __acrt_stdio_flush_nolock  000000018000fc58 f   libucrt:fflush.obj
 0001:0000ed10       _fflush_nolock             000000018000fd10 f   libucrt:fflush.obj
 0001:0000ed78       _flushall                  000000018000fd78 f   libucrt:fflush.obj
 0001:0000ed80       __acrt_initialize_stdio    000000018000fd80 f   libucrt:_file.obj
 0001:0000eea0       __acrt_uninitialize_stdio  000000018000fea0 f   libucrt:_file.obj
 0001:0000ef18       _lock_file                 000000018000ff18 f   libucrt:_file.obj
 0001:0000ef30       _unlock_file               000000018000ff30 f   libucrt:_file.obj
 0001:0000ef48       _mbtowc_l                  000000018000ff48 f   libucrt:mbtowc.obj
 0001:0000f0c0       mbtowc                     00000001800100c0 f   libucrt:mbtowc.obj
 0001:0000f0c8       _fileno                    00000001800100c8 f   libucrt:fileno.obj
 0001:0000f100       __pctype_func              0000000180010100 f   libucrt:ctype.obj
 0001:0000f130       _query_new_mode            0000000180010130 f   libucrt:new_mode.obj
 0001:0000f140       __acrt_add_locale_ref      0000000180010140 f   libucrt:locale_refcounting.obj
 0001:0000f238       __acrt_free_locale         0000000180010238 f   libucrt:locale_refcounting.obj
 0001:0000f388       __acrt_locale_add_lc_time_reference 0000000180010388 f   libucrt:locale_refcounting.obj
 0001:0000f3c8       __acrt_locale_free_lc_time_if_unreferenced 00000001800103c8 f   libucrt:locale_refcounting.obj
 0001:0000f410       __acrt_locale_release_lc_time_reference 0000000180010410 f   libucrt:locale_refcounting.obj
 0001:0000f450       __acrt_release_locale_ref  0000000180010450 f   libucrt:locale_refcounting.obj
 0001:0000f550       __acrt_update_thread_locale_data 0000000180010550 f   libucrt:locale_refcounting.obj
 0001:0000f5c0       _updatetlocinfoEx_nolock   00000001800105c0 f   libucrt:locale_refcounting.obj
 0001:0000f638       __acrt_locale_free_monetary 0000000180010638 f   libucrt:initmon.obj
 0001:0000f768       __acrt_locale_free_numeric 0000000180010768 f   libucrt:initnum.obj
 0001:0000f848       __acrt_locale_free_time    0000000180010848 f   libucrt:inittime.obj
 0001:0000f918       __acrt_GetStringTypeA      0000000180010918 f   libucrt:getstringtypea.obj
 0001:0000fad8       qsort                      0000000180010ad8 f   libucrt:qsort.obj
 0001:0000ff00       strncpy_s                  0000000180010f00 f   libucrt:strncpy_s.obj
 0001:0000ffe0       strpbrk                    0000000180010fe0 f   libucrt:strpbrk.obj
 0001:00010090       _mbsdec                    0000000180011090 f   libucrt:mbsdec.obj
 0001:00010098       _mbsdec_l                  0000000180011098 f   libucrt:mbsdec.obj
 0001:00010450       __acrt_LCMapStringA        0000000180011450 f   libucrt:lcmapstringa.obj
 0001:00010518       _msize_base                0000000180011518 f   libucrt:msize.obj
 0001:00010568       __acrt_DownlevelLocaleNameToLCID 0000000180011568 f   libucrt:lcidtoname_downlevel.obj
 0001:00010620       __acrt_lowio_create_handle_array 0000000180011620 f   libucrt:osfinfo.obj
 0001:000106f0       __acrt_lowio_destroy_handle_array 00000001800116f0 f   libucrt:osfinfo.obj
 0001:00010758       __acrt_lowio_ensure_fh_exists 0000000180011758 f   libucrt:osfinfo.obj
 0001:00010810       __acrt_lowio_lock_fh       0000000180011810 f   libucrt:osfinfo.obj
 0001:00010840       __acrt_lowio_unlock_fh     0000000180011840 f   libucrt:osfinfo.obj
 0001:00010870       _free_osfhnd               0000000180011870 f   libucrt:osfinfo.obj
 0001:00010960       _get_osfhandle             0000000180011960 f   libucrt:osfinfo.obj
 0001:00010aa8       _commit                    0000000180011aa8 f   libucrt:commit.obj
 0001:00011450       _write                     0000000180012450 f   libucrt:write.obj
 0001:00011568       _write_nolock              0000000180012568 f   libucrt:write.obj
 0001:000118a8       _fcloseall                 00000001800128a8 f   libucrt:closeall.obj
 0001:00011980       __acrt_stdio_free_buffer_nolock 0000000180012980 f   libucrt:_freebuf.obj
 0001:000119e8       _isatty                    00000001800129e8 f   libucrt:isatty.obj
 0001:00011a68       _isleadbyte_l              0000000180012a68 f i libucrt:_wctype.obj
 0001:00011ac8       ?__mbrtowc_utf8@__crt_mbstring@@YA_KPEA_WPEBD_KPEAU_Mbstatet@@@Z 0000000180012ac8 f   libucrt:mbrtowc.obj
 0001:00011b10       ?__mbsrtowcs_utf8@__crt_mbstring@@YA_KPEA_WPEAPEBD_KPEAU_Mbstatet@@@Z 0000000180012b10 f   libucrt:mbrtowc.obj
 0001:00011cb8       __ascii_wcsnicmp           0000000180012cb8 f   libucrt:wcsnicmp.obj
 0001:00011d08       __strncnt                  0000000180012d08 f   libucrt:strncnt.obj
 0001:00011d30       _query_app_type            0000000180012d30 f   libucrt:report_runtime_error.obj
 0001:00011e00       _lseeki64_nolock           0000000180012e00 f   libucrt:lseek.obj
 0001:00011e08       _putwch_nolock             0000000180012e08 f   libucrt:putwch.obj
 0001:00011e48       _fclose_nolock             0000000180012e48 f   libucrt:fclose.obj
 0001:00011ee0       fclose                     0000000180012ee0 f   libucrt:fclose.obj
 0001:00011f58       ?__mbrtoc32_utf8@__crt_mbstring@@YA_KPEA_UPEBD_KPEAU_Mbstatet@@@Z 0000000180012f58 f   libucrt:mbrtoc32.obj
 0001:00012120       __dcrt_lowio_ensure_console_output_initialized 0000000180013120 f   libucrt:initcon.obj
 0001:00012188       __dcrt_terminate_console_output 0000000180013188 f   libucrt:initcon.obj
 0001:000121b0       __dcrt_write_console       00000001800131b0 f   libucrt:initcon.obj
 0001:00012330       _close                     0000000180013330 f   libucrt:close.obj
 0001:000123e0       _close_nolock              00000001800133e0 f   libucrt:close.obj
 0001:000124d0       ?__acrt_stdio_free_stream@@YAXV__crt_stdio_stream@@@Z 00000001800134d0 f   libucrt:stream.obj
 0001:000124f8       __GSHandlerCheck           00000001800134f8 f   LIBCMT:gshandler.obj
 0001:00012530       __GSHandlerCheckCommon     0000000180013530 f   LIBCMT:gshandler.obj
 0001:00012550       _FindPESection             0000000180013550 f   LIBCMT:pesect.obj
 0001:000125b0       _IsNonwritableInCurrentImage 00000001800135b0 f   LIBCMT:pesect.obj
 0001:00012618       _ValidateImageBase         0000000180013618 f   LIBCMT:pesect.obj
 0001:00012658       __GSHandlerCheck_EH        0000000180013658 f   LIBCMT:gshandlereh.obj
 0002:00000000       __imp_RegOpenKeyExW        0000000180014000     advapi32:ADVAPI32.dll
 0002:00000008       __imp_RegQueryValueExW     0000000180014008     advapi32:ADVAPI32.dll
 0002:00000010       __imp_IsTextUnicode        0000000180014010     advapi32:ADVAPI32.dll
 0002:00000018       __imp_RegCloseKey          0000000180014018     advapi32:ADVAPI32.dll
 0002:00000020       \177ADVAPI32_NULL_THUNK_DATA 0000000180014020     advapi32:ADVAPI32.dll
 0002:00000028       __imp_GetConsoleOutputCP   0000000180014028     kernel32:KERNEL32.dll
 0002:00000030       __imp_ExpandEnvironmentStringsW 0000000180014030     kernel32:KERNEL32.dll
 0002:00000038       __imp_GetModuleFileNameW   0000000180014038     kernel32:KERNEL32.dll
 0002:00000040       __imp_CreateFileW          0000000180014040     kernel32:KERNEL32.dll
 0002:00000048       __imp_GetFileAttributesW   0000000180014048     kernel32:KERNEL32.dll
 0002:00000050       __imp_GetACP               0000000180014050     kernel32:KERNEL32.dll
 0002:00000058       __imp_MultiByteToWideChar  0000000180014058     kernel32:KERNEL32.dll
 0002:00000060       __imp_GetLastError         0000000180014060     kernel32:KERNEL32.dll
 0002:00000068       __imp_GetConsoleAliasesLengthW 0000000180014068     kernel32:KERNEL32.dll
 0002:00000070       __imp_lstrcatW             0000000180014070     kernel32:KERNEL32.dll
 0002:00000078       __imp_CloseHandle          0000000180014078     kernel32:KERNEL32.dll
 0002:00000080       __imp_CreateDirectoryW     0000000180014080     kernel32:KERNEL32.dll
 0002:00000088       __imp_SearchPathW          0000000180014088     kernel32:KERNEL32.dll
 0002:00000090       __imp_GetConsoleScreenBufferInfo 0000000180014090     kernel32:KERNEL32.dll
 0002:00000098       __imp_GetStdHandle         0000000180014098     kernel32:KERNEL32.dll
 0002:000000a0       __imp_GetConsoleAliasesW   00000001800140a0     kernel32:KERNEL32.dll
 0002:000000a8       __imp_RemoveDirectoryW     00000001800140a8     kernel32:KERNEL32.dll
 0002:000000b0       __imp_GetEnvironmentVariableW 00000001800140b0     kernel32:KERNEL32.dll
 0002:000000b8       __imp_WaitForSingleObject  00000001800140b8     kernel32:KERNEL32.dll
 0002:000000c0       __imp_GetConsoleMode       00000001800140c0     kernel32:KERNEL32.dll
 0002:000000c8       __imp_DeleteFileW          00000001800140c8     kernel32:KERNEL32.dll
 0002:000000d0       __imp_GetCurrentDirectoryW 00000001800140d0     kernel32:KERNEL32.dll
 0002:000000d8       __imp_SetCurrentDirectoryW 00000001800140d8     kernel32:KERNEL32.dll
 0002:000000e0       __imp_WriteConsoleW        00000001800140e0     kernel32:KERNEL32.dll
 0002:000000e8       __imp_GetFileSize          00000001800140e8     kernel32:KERNEL32.dll
 0002:000000f0       __imp_CreateProcessW       00000001800140f0     kernel32:KERNEL32.dll
 0002:000000f8       __imp_GetConsoleWindow     00000001800140f8     kernel32:KERNEL32.dll
 0002:00000100       __imp_GetTempFileNameW     0000000180014100     kernel32:KERNEL32.dll
 0002:00000108       __imp_SetConsoleCursorPosition 0000000180014108     kernel32:KERNEL32.dll
 0002:00000110       __imp_SetConsoleTitleW     0000000180014110     kernel32:KERNEL32.dll
 0002:00000118       __imp_ReadFile             0000000180014118     kernel32:KERNEL32.dll
 0002:00000120       __imp_lstrcpyW             0000000180014120     kernel32:KERNEL32.dll
 0002:00000128       __imp_lstrcpynW            0000000180014128     kernel32:KERNEL32.dll
 0002:00000130       __imp_SetConsoleMode       0000000180014130     kernel32:KERNEL32.dll
 0002:00000138       __imp_lstrlenW             0000000180014138     kernel32:KERNEL32.dll
 0002:00000140       __imp_SetFilePointerEx     0000000180014140     kernel32:KERNEL32.dll
 0002:00000148       __imp_GetConsoleCP         0000000180014148     kernel32:KERNEL32.dll
 0002:00000150       __imp_WriteFile            0000000180014150     kernel32:KERNEL32.dll
 0002:00000158       __imp_FlushFileBuffers     0000000180014158     kernel32:KERNEL32.dll
 0002:00000160       __imp_SetStdHandle         0000000180014160     kernel32:KERNEL32.dll
 0002:00000168       __imp_HeapSize             0000000180014168     kernel32:KERNEL32.dll
 0002:00000170       __imp_QueryPerformanceCounter 0000000180014170     kernel32:KERNEL32.dll
 0002:00000178       __imp_GetCurrentProcessId  0000000180014178     kernel32:KERNEL32.dll
 0002:00000180       __imp_GetCurrentThreadId   0000000180014180     kernel32:KERNEL32.dll
 0002:00000188       __imp_GetSystemTimeAsFileTime 0000000180014188     kernel32:KERNEL32.dll
 0002:00000190       __imp_InitializeSListHead  0000000180014190     kernel32:KERNEL32.dll
 0002:00000198       __imp_GetStartupInfoW      0000000180014198     kernel32:KERNEL32.dll
 0002:000001a0       __imp_GetModuleHandleW     00000001800141a0     kernel32:KERNEL32.dll
 0002:000001a8       __imp_RtlLookupFunctionEntry 00000001800141a8     kernel32:KERNEL32.dll
 0002:000001b0       __imp_RtlUnwindEx          00000001800141b0     kernel32:KERNEL32.dll
 0002:000001b8       __imp_RtlPcToFileHeader    00000001800141b8     kernel32:KERNEL32.dll
 0002:000001c0       __imp_RaiseException       00000001800141c0     kernel32:KERNEL32.dll
 0002:000001c8       __imp_InterlockedFlushSList 00000001800141c8     kernel32:KERNEL32.dll
 0002:000001d0       __imp_SetLastError         00000001800141d0     kernel32:KERNEL32.dll
 0002:000001d8       __imp_FlsAlloc             00000001800141d8     kernel32:KERNEL32.dll
 0002:000001e0       __imp_FlsGetValue          00000001800141e0     kernel32:KERNEL32.dll
 0002:000001e8       __imp_FlsSetValue          00000001800141e8     kernel32:KERNEL32.dll
 0002:000001f0       __imp_FlsFree              00000001800141f0     kernel32:KERNEL32.dll
 0002:000001f8       __imp_EncodePointer        00000001800141f8     kernel32:KERNEL32.dll
 0002:00000200       __imp_EnterCriticalSection 0000000180014200     kernel32:KERNEL32.dll
 0002:00000208       __imp_LeaveCriticalSection 0000000180014208     kernel32:KERNEL32.dll
 0002:00000210       __imp_InitializeCriticalSectionEx 0000000180014210     kernel32:KERNEL32.dll
 0002:00000218       __imp_DeleteCriticalSection 0000000180014218     kernel32:KERNEL32.dll
 0002:00000220       __imp_GetCurrentProcess    0000000180014220     kernel32:KERNEL32.dll
 0002:00000228       __imp_ExitProcess          0000000180014228     kernel32:KERNEL32.dll
 0002:00000230       __imp_TerminateProcess     0000000180014230     kernel32:KERNEL32.dll
 0002:00000238       __imp_FreeLibrary          0000000180014238     kernel32:KERNEL32.dll
 0002:00000240       __imp_GetModuleHandleExW   0000000180014240     kernel32:KERNEL32.dll
 0002:00000248       __imp_GetProcAddress       0000000180014248     kernel32:KERNEL32.dll
 0002:00000250       __imp_HeapFree             0000000180014250     kernel32:KERNEL32.dll
 0002:00000258       __imp_HeapAlloc            0000000180014258     kernel32:KERNEL32.dll
 0002:00000260       __imp_HeapReAlloc          0000000180014260     kernel32:KERNEL32.dll
 0002:00000268       __imp_FindClose            0000000180014268     kernel32:KERNEL32.dll
 0002:00000270       __imp_FindFirstFileExW     0000000180014270     kernel32:KERNEL32.dll
 0002:00000278       __imp_FindNextFileW        0000000180014278     kernel32:KERNEL32.dll
 0002:00000280       __imp_IsValidCodePage      0000000180014280     kernel32:KERNEL32.dll
 0002:00000288       __imp_GetOEMCP             0000000180014288     kernel32:KERNEL32.dll
 0002:00000290       __imp_GetCPInfo            0000000180014290     kernel32:KERNEL32.dll
 0002:00000298       __imp_GetCommandLineA      0000000180014298     kernel32:KERNEL32.dll
 0002:000002a0       __imp_GetCommandLineW      00000001800142a0     kernel32:KERNEL32.dll
 0002:000002a8       __imp_WideCharToMultiByte  00000001800142a8     kernel32:KERNEL32.dll
 0002:000002b0       __imp_GetEnvironmentStringsW 00000001800142b0     kernel32:KERNEL32.dll
 0002:000002b8       __imp_FreeEnvironmentStringsW 00000001800142b8     kernel32:KERNEL32.dll
 0002:000002c0       __imp_InitializeCriticalSectionAndSpinCount 00000001800142c0     kernel32:KERNEL32.dll
 0002:000002c8       __imp_TlsAlloc             00000001800142c8     kernel32:KERNEL32.dll
 0002:000002d0       __imp_TlsGetValue          00000001800142d0     kernel32:KERNEL32.dll
 0002:000002d8       __imp_TlsSetValue          00000001800142d8     kernel32:KERNEL32.dll
 0002:000002e0       __imp_TlsFree              00000001800142e0     kernel32:KERNEL32.dll
 0002:000002e8       __imp_LoadLibraryExW       00000001800142e8     kernel32:KERNEL32.dll
 0002:000002f0       __imp_LCMapStringW         00000001800142f0     kernel32:KERNEL32.dll
 0002:000002f8       __imp_GetProcessHeap       00000001800142f8     kernel32:KERNEL32.dll
 0002:00000300       __imp_GetFileType          0000000180014300     kernel32:KERNEL32.dll
 0002:00000308       __imp_GetStringTypeW       0000000180014308     kernel32:KERNEL32.dll
 0002:00000310       \177KERNEL32_NULL_THUNK_DATA 0000000180014310     kernel32:KERNEL32.dll
 0002:00000318       __imp_UuidFromStringW      0000000180014318     rpcrt4:RPCRT4.dll
 0002:00000320       \177RPCRT4_NULL_THUNK_DATA 0000000180014320     rpcrt4:RPCRT4.dll
 0002:00000328       __imp_GetWindowTextLengthW 0000000180014328     user32:USER32.dll
 0002:00000330       __imp_GetWindowTextW       0000000180014330     user32:USER32.dll
 0002:00000338       \177USER32_NULL_THUNK_DATA 0000000180014338     user32:USER32.dll
 0002:00000340       __imp_CoCreateInstance     0000000180014340     ole32:ole32.dll
 0002:00000348       __imp_CoInitialize         0000000180014348     ole32:ole32.dll
 0002:00000350       __imp_CoUninitialize       0000000180014350     ole32:ole32.dll
 0002:00000358       \177ole32_NULL_THUNK_DATA  0000000180014358     ole32:ole32.dll
 0002:00000360       __guard_check_icall_fptr   0000000180014360     LIBCMT:guard_support.obj
 0002:00000368       __xc_a                     0000000180014368     LIBCMT:initializers.obj
 0002:00000370       __xc_z                     0000000180014370     LIBCMT:initializers.obj
 0002:00000378       __xi_a                     0000000180014378     LIBCMT:initializers.obj
 0002:00000380       __acrt_multibyte_initializer 0000000180014380     libucrt:multibyte_initializer.obj
 0002:00000388       __acrt_stdio_initializer   0000000180014388     libucrt:stdio_initializer.obj
 0002:00000390       __xi_z                     0000000180014390     LIBCMT:initializers.obj
 0002:00000398       __xp_a                     0000000180014398     LIBCMT:initializers.obj
 0002:000003a0       __acrt_locale_terminator   00000001800143a0     libucrt:locale_initializer.obj
 0002:000003a8       __dcrt_console_output_terminator 00000001800143a8     libucrt:console_output_initializer.obj
 0002:000003b0       __acrt_stdio_terminator    00000001800143b0     libucrt:stdio_initializer.obj
 0002:000003b8       __xp_z                     00000001800143b8     LIBCMT:initializers.obj
 0002:000003c0       __xt_a                     00000001800143c0     LIBCMT:initializers.obj
 0002:000003c8       __xt_z                     00000001800143c8     LIBCMT:initializers.obj
 0002:000003d0       IID_IShellLinkW            00000001800143d0     shell32:shguid.obj
 0002:000003e0       IID_IPersistFile           00000001800143e0     uuid:objidl_i.obj
 0002:000003f0       CLSID_ShellLink            00000001800143f0     uuid:shguids.obj
 0002:00000408       ??_7type_info@@6B@         0000000180014408     LIBCMT:std_type_info_static.obj
 0002:00000410       _pRawDllMain               0000000180014410     LIBCMT:dll_dllmain.obj
 0002:00000410       _pDefaultRawDllMain        0000000180014410     LIBCMT:dll_dllmain.obj
 0002:00000430       ??_7exception@std@@6B@     0000000180014430     LIBCMT:throw_bad_alloc.obj
 0002:00000440       ??_C@_0BC@EOODALEL@Unknown?5exception@ 0000000180014440     LIBCMT:throw_bad_alloc.obj
 0002:00000460       ??_7bad_alloc@std@@6B@     0000000180014460     LIBCMT:throw_bad_alloc.obj
 0002:00000470       ??_C@_0P@GHFPNOJB@bad?5allocation@ 0000000180014470     LIBCMT:throw_bad_alloc.obj
 0002:00000488       ??_7bad_array_new_length@std@@6B@ 0000000180014488     LIBCMT:throw_bad_alloc.obj
 0002:00000498       ??_C@_0BF@KINCDENJ@bad?5array?5new?5length@ 0000000180014498     LIBCMT:throw_bad_alloc.obj
 0002:00000548       _pDestructExceptionObject  0000000180014548     libvcruntime:ehhelpers.obj
 0002:00000558       ??_7bad_exception@std@@6B@ 0000000180014558     libvcruntime:frame.obj
 0002:00000568       ??_C@_0O@DPKOEFFH@bad?5exception@ 0000000180014568     libvcruntime:frame.obj
 0002:00000c80       ??_C@_08EHJDFFNH@__based?$CI@ 0000000180014c80     libvcruntime:undname.obj
 0002:00000c90       ??_C@_07KOLFKCDI@__cdecl@  0000000180014c90     libvcruntime:undname.obj
 0002:00000c98       ??_C@_08GHMPAG@__pascal@   0000000180014c98     libvcruntime:undname.obj
 0002:00000ca8       ??_C@_09IFJBGAPI@__stdcall@ 0000000180014ca8     libvcruntime:undname.obj
 0002:00000cb8       ??_C@_0L@NPHFGOKO@__thiscall@ 0000000180014cb8     libvcruntime:undname.obj
 0002:00000cc8       ??_C@_0L@JMKHOMEK@__fastcall@ 0000000180014cc8     libvcruntime:undname.obj
 0002:00000cd8       ??_C@_0N@BCKKPABJ@__vectorcall@ 0000000180014cd8     libvcruntime:undname.obj
 0002:00000ce8       ??_C@_09HIJEGCPM@__clrcall@ 0000000180014ce8     libvcruntime:undname.obj
 0002:00000cf4       ??_C@_06GHPCKEAG@__eabi@   0000000180014cf4     libvcruntime:undname.obj
 0002:00000d00       ??_C@_09IOPIDJLG@__swift_1@ 0000000180014d00     libvcruntime:undname.obj
 0002:00000d10       ??_C@_09KFNFGKHF@__swift_2@ 0000000180014d10     libvcruntime:undname.obj
 0002:00000d20       ??_C@_07JOMMBBKO@__ptr64@  0000000180014d20     libvcruntime:undname.obj
 0002:00000d28       ??_C@_0L@PILCLIHE@__restrict@ 0000000180014d28     libvcruntime:undname.obj
 0002:00000d38       ??_C@_0M@GFIIJFMG@__unaligned@ 0000000180014d38     libvcruntime:undname.obj
 0002:00000d48       ??_C@_09DHDLOLLB@restrict?$CI@ 0000000180014d48     libvcruntime:undname.obj
 0002:00000d52       ??_C@_00CNPNBAHC@@         0000000180014d52     libvcruntime:undname.obj
 0002:00000d54       ??_C@_04NIHEBCM@?5new@     0000000180014d54     libvcruntime:undname.obj
 0002:00000d60       ??_C@_07FPCDHGMM@?5delete@ 0000000180014d60     libvcruntime:undname.obj
 0002:00000d68       ??_C@_01NEMOKFLO@?$DN@     0000000180014d68     libvcruntime:undname.obj
 0002:00000d6c       ??_C@_02GPIOPFAK@?$DO?$DO@ 0000000180014d6c     libvcruntime:undname.obj
 0002:00000d70       ??_C@_02FODMEDOG@?$DM?$DM@ 0000000180014d70     libvcruntime:undname.obj
 0002:00000d74       ??_C@_01DCLJPIOD@?$CB@     0000000180014d74     libvcruntime:undname.obj
 0002:00000d78       ??_C@_02EGOFBIJA@?$DN?$DN@ 0000000180014d78     libvcruntime:undname.obj
 0002:00000d7c       ??_C@_02FDNJECIE@?$CB?$DN@ 0000000180014d7c     libvcruntime:undname.obj
 0002:00000d80       ??_C@_02GPECMEKF@?$FL?$FN@ 0000000180014d80     libvcruntime:undname.obj
 0002:00000d88       ??_C@_08LHJFAFGD@operator@ 0000000180014d88     libvcruntime:undname.obj
 0002:00000d94       ??_C@_02HBOOOICD@?9?$DO@   0000000180014d94     libvcruntime:undname.obj
 0002:00000d98       ??_C@_01NBENCBCI@?$CK@     0000000180014d98     libvcruntime:undname.obj
 0002:00000d9c       ??_C@_02ECNGHCIF@?$CL?$CL@ 0000000180014d9c     libvcruntime:undname.obj
 0002:00000da0       ??_C@_02BAABKJLB@?9?9@     0000000180014da0     libvcruntime:undname.obj
 0002:00000da4       ??_C@_01JOAMLHOP@?9@       0000000180014da4     libvcruntime:undname.obj
 0002:00000da8       ??_C@_01MIFGBAGJ@?$CL@     0000000180014da8     libvcruntime:undname.obj
 0002:00000dac       ??_C@_01HNPIGOCE@?$CG@     0000000180014dac     libvcruntime:undname.obj
 0002:00000db0       ??_C@_03MNHNFDLC@?9?$DO?$CK@ 0000000180014db0     libvcruntime:undname.obj
 0002:00000db4       ??_C@_01KMDKNFGN@?1@       0000000180014db4     libvcruntime:undname.obj
 0002:00000db8       ??_C@_01FGNFDNOH@?$CF@     0000000180014db8     libvcruntime:undname.obj
 0002:00000dbc       ??_C@_01MNNFJEPP@?$DM@     0000000180014dbc     libvcruntime:undname.obj
 0002:00000dc0       ??_C@_02EHCHHCKH@?$DM?$DN@ 0000000180014dc0     libvcruntime:undname.obj
 0002:00000dc4       ??_C@_01PPODPGHN@?$DO@     0000000180014dc4     libvcruntime:undname.obj
 0002:00000dc8       ??_C@_02EEKDKGMJ@?$DO?$DN@ 0000000180014dc8     libvcruntime:undname.obj
 0002:00000dcc       ??_C@_01IHBHIGKO@?0@       0000000180014dcc     libvcruntime:undname.obj
 0002:00000dd0       ??_C@_02HCKGKOFO@?$CI?$CJ@ 0000000180014dd0     libvcruntime:undname.obj
 0002:00000dd4       ??_C@_01PJKLJHI@?$HO@      0000000180014dd4     libvcruntime:undname.obj
 0002:00000dd8       ??_C@_01JKBOJNNK@?$FO@     0000000180014dd8     libvcruntime:undname.obj
 0002:00000ddc       ??_C@_01DNKMNLPK@?$HM@     0000000180014ddc     libvcruntime:undname.obj
 0002:00000de0       ??_C@_02PPKAJPJL@?$CG?$CG@ 0000000180014de0     libvcruntime:undname.obj
 0002:00000de4       ??_C@_02NONPIBCD@?$HM?$HM@ 0000000180014de4     libvcruntime:undname.obj
 0002:00000de8       ??_C@_02FPIMKNGF@?$CK?$DN@ 0000000180014de8     libvcruntime:undname.obj
 0002:00000dec       ??_C@_02FOEOMHFC@?$CL?$DN@ 0000000180014dec     libvcruntime:undname.obj
 0002:00000df0       ??_C@_02FKMDLLOA@?9?$DN@   0000000180014df0     libvcruntime:undname.obj
 0002:00000df4       ??_C@_02FJEHGPIO@?1?$DN@   0000000180014df4     libvcruntime:undname.obj
 0002:00000df8       ??_C@_02FENAOKFI@?$CF?$DN@ 0000000180014df8     libvcruntime:undname.obj
 0002:00000dfc       ??_C@_03IKFCCPFF@?$DO?$DO?$DN@ 0000000180014dfc     libvcruntime:undname.obj
 0002:00000e00       ??_C@_03CDNPDDLA@?$DM?$DM?$DN@ 0000000180014e00     libvcruntime:undname.obj
 0002:00000e04       ??_C@_02FGJGFEAB@?$CG?$DN@ 0000000180014e04     libvcruntime:undname.obj
 0002:00000e08       ??_C@_02DHLNPPGH@?$HM?$DN@ 0000000180014e08     libvcruntime:undname.obj
 0002:00000e0c       ??_C@_02MHEGNOJ@?$FO?$DN@  0000000180014e0c     libvcruntime:undname.obj
 0002:00000e10       ??_C@_09IFPLHPGF@?$GAvftable?8@ 0000000180014e10     libvcruntime:undname.obj
 0002:00000e20       ??_C@_09BLBHBJP@?$GAvbtable?8@ 0000000180014e20     libvcruntime:undname.obj
 0002:00000e30       ??_C@_07FEEIOKP@?$GAvcall?8@ 0000000180014e30     libvcruntime:undname.obj
 0002:00000e38       ??_C@_08LLFFHHDJ@?$GAtypeof?8@ 0000000180014e38     libvcruntime:undname.obj
 0002:00000e48       ??_C@_0BF@KDPPACIK@?$GAlocal?5static?5guard?8@ 0000000180014e48     libvcruntime:undname.obj
 0002:00000e60       ??_C@_08OBABFOLI@?$GAstring?8@ 0000000180014e60     libvcruntime:undname.obj
 0002:00000e70       ??_C@_0BD@JDLKDPAB@?$GAvbase?5destructor?8@ 0000000180014e70     libvcruntime:undname.obj
 0002:00000e88       ??_C@_0BN@DEGPLNFK@?$GAvector?5deleting?5destructor?8@ 0000000180014e88     libvcruntime:undname.obj
 0002:00000ea8       ??_C@_0BO@OBMKPJIG@?$GAdefault?5constructor?5closure?8@ 0000000180014ea8     libvcruntime:undname.obj
 0002:00000ec8       ??_C@_0BN@IMDCHIKM@?$GAscalar?5deleting?5destructor?8@ 0000000180014ec8     libvcruntime:undname.obj
 0002:00000ee8       ??_C@_0BO@PFGOCPJJ@?$GAvector?5constructor?5iterator?8@ 0000000180014ee8     libvcruntime:undname.obj
 0002:00000f08       ??_C@_0BN@LFPFMEDL@?$GAvector?5destructor?5iterator?8@ 0000000180014f08     libvcruntime:undname.obj
 0002:00000f28       ??_C@_0CE@IKBNEHA@?$GAvector?5vbase?5constructor?5itera@ 0000000180014f28     libvcruntime:undname.obj
 0002:00000f50       ??_C@_0BL@NILFHHPC@?$GAvirtual?5displacement?5map?8@ 0000000180014f50     libvcruntime:undname.obj
 0002:00000f70       ??_C@_0CB@JONCMFFK@?$GAeh?5vector?5constructor?5iterator@ 0000000180014f70     libvcruntime:undname.obj
 0002:00000f98       ??_C@_0CA@GCEOPDGL@?$GAeh?5vector?5destructor?5iterator?8@ 0000000180014f98     libvcruntime:undname.obj
 0002:00000fb8       ??_C@_0CH@OOJPLCPH@?$GAeh?5vector?5vbase?5constructor?5it@ 0000000180014fb8     libvcruntime:undname.obj
 0002:00000fe0       ??_C@_0BL@LLKPOHJI@?$GAcopy?5constructor?5closure?8@ 0000000180014fe0     libvcruntime:undname.obj
 0002:00001000       ??_C@_0BA@KBCDOMBN@?$GAudt?5returning?8@ 0000000180015000     libvcruntime:undname.obj
 0002:00001010       ??_C@_03KLGMFNMG@?$GAEH@   0000000180015010     libvcruntime:undname.obj
 0002:00001014       ??_C@_05KHLCHHI@?$GARTTI@  0000000180015014     libvcruntime:undname.obj
 0002:00001020       ??_C@_0BA@KKLDJDLB@?$GAlocal?5vftable?8@ 0000000180015020     libvcruntime:undname.obj
 0002:00001030       ??_C@_0CE@IIHCMGGL@?$GAlocal?5vftable?5constructor?5clos@ 0000000180015030     libvcruntime:undname.obj
 0002:00001054       ??_C@_06FHBGPFGH@?5new?$FL?$FN@ 0000000180015054     libvcruntime:undname.obj
 0002:00001060       ??_C@_09LBNFPBCA@?5delete?$FL?$FN@ 0000000180015060     libvcruntime:undname.obj
 0002:00001070       ??_C@_0P@HJKNJFNN@?$GAomni?5callsig?8@ 0000000180015070     libvcruntime:undname.obj
 0002:00001080       ??_C@_0BL@CNOONJFP@?$GAplacement?5delete?5closure?8@ 0000000180015080     libvcruntime:undname.obj
 0002:000010a0       ??_C@_0BN@CKNJLHMB@?$GAplacement?5delete?$FL?$FN?5closure?8@ 00000001800150a0     libvcruntime:undname.obj
 0002:000010c0       ??_C@_0CG@CFDHKGGD@?$GAmanaged?5vector?5constructor?5ite@ 00000001800150c0     libvcruntime:undname.obj
 0002:000010e8       ??_C@_0CF@IMGKMJNO@?$GAmanaged?5vector?5destructor?5iter@ 00000001800150e8     libvcruntime:undname.obj
 0002:00001110       ??_C@_0CG@HLDDJMAG@?$GAeh?5vector?5copy?5constructor?5ite@ 0000000180015110     libvcruntime:undname.obj
 0002:00001138       ??_C@_0CM@FCBBDIGB@?$GAeh?5vector?5vbase?5copy?5construct@ 0000000180015138     libvcruntime:undname.obj
 0002:00001168       ??_C@_0BL@CLIPGLGB@?$GAdynamic?5initializer?5for?5?8@ 0000000180015168     libvcruntime:undname.obj
 0002:00001188       ??_C@_0CB@PDBIFEP@?$GAdynamic?5atexit?5destructor?5for?5@ 0000000180015188     libvcruntime:undname.obj
 0002:000011b0       ??_C@_0CD@CGAJBKEJ@?$GAvector?5copy?5constructor?5iterat@ 00000001800151b0     libvcruntime:undname.obj
 0002:000011d8       ??_C@_0CJ@GJELGAMM@?$GAvector?5vbase?5copy?5constructor?5@ 00000001800151d8     libvcruntime:undname.obj
 0002:00001208       ??_C@_0CL@FGIJHLCE@?$GAmanaged?5vector?5copy?5constructo@ 0000000180015208     libvcruntime:undname.obj
 0002:00001238       ??_C@_0BM@PMGGMLDN@?$GAlocal?5static?5thread?5guard?8@ 0000000180015238     libvcruntime:undname.obj
 0002:00001258       ??_C@_0N@BDNMDMOL@operator?5?$CC?$CC?5@ 0000000180015258     libvcruntime:undname.obj
 0002:00001268       ??_C@_0BC@GGEBGALA@operator?5co_await@ 0000000180015268     libvcruntime:undname.obj
 0002:00001280       ??_C@_0M@GAAIMMOH@operator?$DM?$DN?$DO@ 0000000180015280     libvcruntime:undname.obj
 0002:00001290       ??_C@_0BC@DAFEJGAK@?5Type?5Descriptor?8@ 0000000180015290     libvcruntime:undname.obj
 0002:000012a8       ??_C@_0BM@LDKODKLH@?5Base?5Class?5Descriptor?5at?5?$CI@ 00000001800152a8     libvcruntime:undname.obj
 0002:000012c8       ??_C@_0BD@LGICGFMM@?5Base?5Class?5Array?8@ 00000001800152c8     libvcruntime:undname.obj
 0002:000012e0       ??_C@_0BN@MECKDCOJ@?5Class?5Hierarchy?5Descriptor?8@ 00000001800152e0     libvcruntime:undname.obj
 0002:00001300       ??_C@_0BK@CFCOFLF@?5Complete?5Object?5Locator?8@ 0000000180015300     libvcruntime:undname.obj
 0002:00001320       ??_C@_0BG@JNJLAMPM@?$GAanonymous?5namespace?8@ 0000000180015320     libvcruntime:undname.obj
 0002:00001340       __acrt_exception_action_table 0000000180015340     libucrt:exception_filter.obj
 0002:00001400       __acrt_signal_action_table_count 0000000180015400     libucrt:exception_filter.obj
 0002:00001408       __acrt_signal_action_first_fpe_index 0000000180015408     libucrt:exception_filter.obj
 0002:00001410       __acrt_signal_action_fpe_count 0000000180015410     libucrt:exception_filter.obj
 0002:00001418       ??_C@_1BI@BGOHAHKC@?$AAm?$AAs?$AAc?$AAo?$AAr?$AAe?$AAe?$AA?4?$AAd?$AAl?$AAl@ 0000000180015418     libucrt:exit.obj
 0002:00001430       ??_C@_0P@MIGLKIOC@CorExitProcess@ 0000000180015430     libucrt:exit.obj
 0002:000016b0       __lc_time_c                00000001800156b0     libucrt:nlsdata.obj
 0002:00001970       ??_C@_03KOEHGMDN@Sun@      0000000180015970     libucrt:nlsdata.obj
 0002:00001974       ??_C@_03PDAGKDH@Mon@       0000000180015974     libucrt:nlsdata.obj
 0002:00001978       ??_C@_03NAGEINEP@Tue@      0000000180015978     libucrt:nlsdata.obj
 0002:0000197c       ??_C@_03MHOMLAJA@Wed@      000000018001597c     libucrt:nlsdata.obj
 0002:00001980       ??_C@_03IOFIKPDN@Thu@      0000000180015980     libucrt:nlsdata.obj
 0002:00001984       ??_C@_03IDIOELNC@Fri@      0000000180015984     libucrt:nlsdata.obj
 0002:00001988       ??_C@_03FEFJNEK@Sat@       0000000180015988     libucrt:nlsdata.obj
 0002:0000198c       ??_C@_06OOPIFAJ@Sunday@    000000018001598c     libucrt:nlsdata.obj
 0002:00001994       ??_C@_06JLEDEDGH@Monday@   0000000180015994     libucrt:nlsdata.obj
 0002:000019a0       ??_C@_07BAAGCFCM@Tuesday@  00000001800159a0     libucrt:nlsdata.obj
 0002:000019a8       ??_C@_09DLIGFAKA@Wednesday@ 00000001800159a8     libucrt:nlsdata.obj
 0002:000019b8       ??_C@_08HACCIKIA@Thursday@ 00000001800159b8     libucrt:nlsdata.obj
 0002:000019c4       ??_C@_06JECMNKMI@Friday@   00000001800159c4     libucrt:nlsdata.obj
 0002:000019d0       ??_C@_08INBOOONO@Saturday@ 00000001800159d0     libucrt:nlsdata.obj
 0002:000019dc       ??_C@_03JIHJHPIE@Jan@      00000001800159dc     libucrt:nlsdata.obj
 0002:000019e0       ??_C@_03HJBDCHOM@Feb@      00000001800159e0     libucrt:nlsdata.obj
 0002:000019e4       ??_C@_03ODNJBKGA@Mar@      00000001800159e4     libucrt:nlsdata.obj
 0002:000019e8       ??_C@_03LEOLGMJP@Apr@      00000001800159e8     libucrt:nlsdata.obj
 0002:000019ec       ??_C@_03CNMDKL@May@        00000001800159ec     libucrt:nlsdata.obj
 0002:000019f0       ??_C@_03IDFGHECI@Jun@      00000001800159f0     libucrt:nlsdata.obj
 0002:000019f4       ??_C@_03LBGABGKK@Jul@      00000001800159f4     libucrt:nlsdata.obj
 0002:000019f8       ??_C@_03IFJFEIGA@Aug@      00000001800159f8     libucrt:nlsdata.obj
 0002:000019fc       ??_C@_03GGCAPAJC@Sep@      00000001800159fc     libucrt:nlsdata.obj
 0002:00001a00       ??_C@_03BMAOKBAD@Oct@      0000000180015a00     libucrt:nlsdata.obj
 0002:00001a04       ??_C@_03JPJOFNIA@Nov@      0000000180015a04     libucrt:nlsdata.obj
 0002:00001a08       ??_C@_03MKABNOCG@Dec@      0000000180015a08     libucrt:nlsdata.obj
 0002:00001a10       ??_C@_07CGJPFGJA@January@  0000000180015a10     libucrt:nlsdata.obj
 0002:00001a18       ??_C@_08GNJGEPFN@February@ 0000000180015a18     libucrt:nlsdata.obj
 0002:00001a24       ??_C@_05HPCKOFNC@March@    0000000180015a24     libucrt:nlsdata.obj
 0002:00001a2c       ??_C@_05DMJDNLEJ@April@    0000000180015a2c     libucrt:nlsdata.obj
 0002:00001a34       ??_C@_04CNLMGBGM@June@     0000000180015a34     libucrt:nlsdata.obj
 0002:00001a3c       ??_C@_04MIEPOIFP@July@     0000000180015a3c     libucrt:nlsdata.obj
 0002:00001a44       ??_C@_06LBBHFDDG@August@   0000000180015a44     libucrt:nlsdata.obj
 0002:00001a50       ??_C@_09BHHEALKD@September@ 0000000180015a50     libucrt:nlsdata.obj
 0002:00001a60       ??_C@_07JJNFCEND@October@  0000000180015a60     libucrt:nlsdata.obj
 0002:00001a68       ??_C@_08HCHEGEOA@November@ 0000000180015a68     libucrt:nlsdata.obj
 0002:00001a78       ??_C@_08EDHMEBNP@December@ 0000000180015a78     libucrt:nlsdata.obj
 0002:00001a84       ??_C@_02DEDBPAFC@AM@       0000000180015a84     libucrt:nlsdata.obj
 0002:00001a88       ??_C@_02CJNFDJBF@PM@       0000000180015a88     libucrt:nlsdata.obj
 0002:00001a90       ??_C@_08BPBNCDIB@MM?1dd?1yy@ 0000000180015a90     libucrt:nlsdata.obj
 0002:00001aa0       ??_C@_0BE@CKGJFCPC@dddd?0?5MMMM?5dd?0?5yyyy@ 0000000180015aa0     libucrt:nlsdata.obj
 0002:00001ab8       ??_C@_08JCCMCCIL@HH?3mm?3ss@ 0000000180015ab8     libucrt:nlsdata.obj
 0002:00001ac8       ??_C@_17MBGCMIPB@?$AAS?$AAu?$AAn@ 0000000180015ac8     libucrt:nlsdata.obj
 0002:00001ad0       ??_C@_17KBOMKBF@?$AAM?$AAo?$AAn@ 0000000180015ad0     libucrt:nlsdata.obj
 0002:00001ad8       ??_C@_17BMKGEGOJ@?$AAT?$AAu?$AAe@ 0000000180015ad8     libucrt:nlsdata.obj
 0002:00001ae0       ??_C@_17CJEDCEPE@?$AAW?$AAe?$AAd@ 0000000180015ae0     libucrt:nlsdata.obj
 0002:00001ae8       ??_C@_17PDPHAADD@?$AAT?$AAh?$AAu@ 0000000180015ae8     libucrt:nlsdata.obj
 0002:00001af0       ??_C@_17HFOLPPLP@?$AAF?$AAr?$AAi@ 0000000180015af0     libucrt:nlsdata.obj
 0002:00001af8       ??_C@_17GGIBDPIH@?$AAS?$AAa?$AAt@ 0000000180015af8     libucrt:nlsdata.obj
 0002:00001b00       ??_C@_1O@IHNHDHPB@?$AAS?$AAu?$AAn?$AAd?$AAa?$AAy@ 0000000180015b00     libucrt:nlsdata.obj
 0002:00001b10       ??_C@_1O@MMNBFLIA@?$AAM?$AAo?$AAn?$AAd?$AAa?$AAy@ 0000000180015b10     libucrt:nlsdata.obj
 0002:00001b20       ??_C@_1BA@ENFBFFEK@?$AAT?$AAu?$AAe?$AAs?$AAd?$AAa?$AAy@ 0000000180015b20     libucrt:nlsdata.obj
 0002:00001b30       ??_C@_1BE@EBOGMDOH@?$AAW?$AAe?$AAd?$AAn?$AAe?$AAs?$AAd?$AAa?$AAy@ 0000000180015b30     libucrt:nlsdata.obj
 0002:00001b48       ??_C@_1BC@HHMNLIHE@?$AAT?$AAh?$AAu?$AAr?$AAs?$AAd?$AAa?$AAy@ 0000000180015b48     libucrt:nlsdata.obj
 0002:00001b60       ??_C@_1O@PDICJHAG@?$AAF?$AAr?$AAi?$AAd?$AAa?$AAy@ 0000000180015b60     libucrt:nlsdata.obj
 0002:00001b70       ??_C@_1BC@ENMNNPAJ@?$AAS?$AAa?$AAt?$AAu?$AAr?$AAd?$AAa?$AAy@ 0000000180015b70     libucrt:nlsdata.obj
 0002:00001b88       ??_C@_17DKNBKCHM@?$AAJ?$AAa?$AAn@ 0000000180015b88     libucrt:nlsdata.obj
 0002:00001b90       ??_C@_17LMDJEKJN@?$AAF?$AAe?$AAb@ 0000000180015b90     libucrt:nlsdata.obj
 0002:00001b98       ??_C@_17CKNLEDEC@?$AAM?$AAa?$AAr@ 0000000180015b98     libucrt:nlsdata.obj
 0002:00001ba0       ??_C@_17LFPOIHDD@?$AAA?$AAp?$AAr@ 0000000180015ba0     libucrt:nlsdata.obj
 0002:00001ba8       ??_C@_17PNNKMEED@?$AAM?$AAa?$AAy@ 0000000180015ba8     libucrt:nlsdata.obj
 0002:00001bb0       ??_C@_17KCJGOCPB@?$AAJ?$AAu?$AAn@ 0000000180015bb0     libucrt:nlsdata.obj
 0002:00001bb8       ??_C@_17IJPCKHK@?$AAJ?$AAu?$AAl@ 0000000180015bb8     libucrt:nlsdata.obj
 0002:00001bc0       ??_C@_17ICPELBCN@?$AAA?$AAu?$AAg@ 0000000180015bc0     libucrt:nlsdata.obj
 0002:00001bc8       ??_C@_17HCHCOKMG@?$AAS?$AAe?$AAp@ 0000000180015bc8     libucrt:nlsdata.obj
 0002:00001bd0       ??_C@_17FNLKOI@?$AAO?$AAc?$AAt@ 0000000180015bd0     libucrt:nlsdata.obj
 0002:00001bd8       ??_C@_17BBDMLCIG@?$AAN?$AAo?$AAv@ 0000000180015bd8     libucrt:nlsdata.obj
 0002:00001be0       ??_C@_17EGKACKIF@?$AAD?$AAe?$AAc@ 0000000180015be0     libucrt:nlsdata.obj
 0002:00001be8       ??_C@_1BA@EFMEIEBA@?$AAJ?$AAa?$AAn?$AAu?$AAa?$AAr?$AAy@ 0000000180015be8     libucrt:nlsdata.obj
 0002:00001bf8       ??_C@_1BC@JGDDFFAM@?$AAF?$AAe?$AAb?$AAr?$AAu?$AAa?$AAr?$AAy@ 0000000180015bf8     libucrt:nlsdata.obj
 0002:00001c10       ??_C@_1M@IKEENEDF@?$AAM?$AAa?$AAr?$AAc?$AAh@ 0000000180015c10     libucrt:nlsdata.obj
 0002:00001c20       ??_C@_1M@GJNLMHFD@?$AAA?$AAp?$AAr?$AAi?$AAl@ 0000000180015c20     libucrt:nlsdata.obj
 0002:00001c30       ??_C@_19EPFLPGAP@?$AAJ?$AAu?$AAn?$AAe@ 0000000180015c30     libucrt:nlsdata.obj
 0002:00001c40       ??_C@_19BIFMLPCD@?$AAJ?$AAu?$AAl?$AAy@ 0000000180015c40     libucrt:nlsdata.obj
 0002:00001c50       ??_C@_1O@PAHLKOAC@?$AAA?$AAu?$AAg?$AAu?$AAs?$AAt@ 0000000180015c50     libucrt:nlsdata.obj
 0002:00001c60       ??_C@_1BE@DKAAMBJL@?$AAS?$AAe?$AAp?$AAt?$AAe?$AAm?$AAb?$AAe?$AAr@ 0000000180015c60     libucrt:nlsdata.obj
 0002:00001c78       ??_C@_1BA@EPANDLNG@?$AAO?$AAc?$AAt?$AAo?$AAb?$AAe?$AAr@ 0000000180015c78     libucrt:nlsdata.obj
 0002:00001c88       ??_C@_1BC@BGLIFPF@?$AAN?$AAo?$AAv?$AAe?$AAm?$AAb?$AAe?$AAr@ 0000000180015c88     libucrt:nlsdata.obj
 0002:00001ca0       ??_C@_1BC@FEMKIFH@?$AAD?$AAe?$AAc?$AAe?$AAm?$AAb?$AAe?$AAr@ 0000000180015ca0     libucrt:nlsdata.obj
 0002:00001cb4       ??_C@_15ODEHAHHF@?$AAA?$AAM@ 0000000180015cb4     libucrt:nlsdata.obj
 0002:00001cbc       ??_C@_15CLMNNGEL@?$AAP?$AAM@ 0000000180015cbc     libucrt:nlsdata.obj
 0002:00001cc8       ??_C@_1BC@IEBCMHCM@?$AAM?$AAM?$AA?1?$AAd?$AAd?$AA?1?$AAy?$AAy@ 0000000180015cc8     libucrt:nlsdata.obj
 0002:00001ce0       ??_C@_1CI@KNAKOEBC@?$AAd?$AAd?$AAd?$AAd?$AA?0?$AA?5?$AAM?$AAM?$AAM?$AAM?$AA?5?$AAd?$AAd?$AA?0?$AA?5@ 0000000180015ce0     libucrt:nlsdata.obj
 0002:00001d08       ??_C@_1BC@GDGBMEMK@?$AAH?$AAH?$AA?3?$AAm?$AAm?$AA?3?$AAs?$AAs@ 0000000180015d08     libucrt:nlsdata.obj
 0002:00001d20       ??_C@_1M@BMHNFIME@?$AAe?$AAn?$AA?9?$AAU?$AAS@ 0000000180015d20     libucrt:nlsdata.obj
 0002:00001d30       ??_C@_1M@HPNHIDJI@?$AAj?$AAa?$AA?9?$AAJ?$AAP@ 0000000180015d30     libucrt:mbctype.obj
 0002:00001d40       ??_C@_1M@BIBDDEMK@?$AAz?$AAh?$AA?9?$AAC?$AAN@ 0000000180015d40     libucrt:mbctype.obj
 0002:00001d50       ??_C@_1M@JLOOOEGK@?$AAk?$AAo?$AA?9?$AAK?$AAR@ 0000000180015d50     libucrt:mbctype.obj
 0002:00001d60       ??_C@_1M@CLNBBOPM@?$AAz?$AAh?$AA?9?$AAT?$AAW@ 0000000180015d60     libucrt:mbctype.obj
 0002:00001e10       ??_C@_1EA@JGEFHKEI@?$AAa?$AAp?$AAi?$AA?9?$AAm?$AAs?$AA?9?$AAw?$AAi?$AAn?$AA?9?$AAc?$AAo?$AAr?$AAe@ 0000000180015e10     libucrt:winapi_thunks.obj
 0002:00001e50       ??_C@_1DM@KHCHBNEB@?$AAa?$AAp?$AAi?$AA?9?$AAm?$AAs?$AA?9?$AAw?$AAi?$AAn?$AA?9?$AAc?$AAo?$AAr?$AAe@ 0000000180015e50     libucrt:winapi_thunks.obj
 0002:00001e90       ??_C@_1DI@IJCEHOCB@?$AAa?$AAp?$AAi?$AA?9?$AAm?$AAs?$AA?9?$AAw?$AAi?$AAn?$AA?9?$AAc?$AAo?$AAr?$AAe@ 0000000180015e90     libucrt:winapi_thunks.obj
 0002:00001ed0       ??_C@_1EI@MPIAOHOC@?$AAa?$AAp?$AAi?$AA?9?$AAm?$AAs?$AA?9?$AAw?$AAi?$AAn?$AA?9?$AAc?$AAo?$AAr?$AAe@ 0000000180015ed0     libucrt:winapi_thunks.obj
 0002:00001f20       ??_C@_1FK@FPHCKFIE@?$AAa?$AAp?$AAi?$AA?9?$AAm?$AAs?$AA?9?$AAw?$AAi?$AAn?$AA?9?$AAc?$AAo?$AAr?$AAe@ 0000000180015f20     libucrt:winapi_thunks.obj
 0002:00001f80       ??_C@_1EM@DILCGIIO@?$AAa?$AAp?$AAi?$AA?9?$AAm?$AAs?$AA?9?$AAw?$AAi?$AAn?$AA?9?$AAc?$AAo?$AAr?$AAe@ 0000000180015f80     libucrt:winapi_thunks.obj
 0002:00001fd0       ??_C@_1DM@LNCGDDPN@?$AAa?$AAp?$AAi?$AA?9?$AAm?$AAs?$AA?9?$AAw?$AAi?$AAn?$AA?9?$AAc?$AAo?$AAr?$AAe@ 0000000180015fd0     libucrt:winapi_thunks.obj
 0002:00002010       ??_C@_1DK@LPPGFMPP@?$AAa?$AAp?$AAi?$AA?9?$AAm?$AAs?$AA?9?$AAw?$AAi?$AAn?$AA?9?$AAc?$AAo?$AAr?$AAe@ 0000000180016010     libucrt:winapi_thunks.obj
 0002:00002050       ??_C@_1DO@FPAPJEMD@?$AAa?$AAp?$AAi?$AA?9?$AAm?$AAs?$AA?9?$AAw?$AAi?$AAn?$AA?9?$AAc?$AAo?$AAr?$AAe@ 0000000180016050     libucrt:winapi_thunks.obj
 0002:00002090       ??_C@_1DK@NDHNAHIO@?$AAa?$AAp?$AAi?$AA?9?$AAm?$AAs?$AA?9?$AAw?$AAi?$AAn?$AA?9?$AAc?$AAo?$AAr?$AAe@ 0000000180016090     libucrt:winapi_thunks.obj
 0002:000020d0       ??_C@_1DM@KGHDGBCM@?$AAa?$AAp?$AAi?$AA?9?$AAm?$AAs?$AA?9?$AAw?$AAi?$AAn?$AA?9?$AAc?$AAo?$AAr?$AAe@ 00000001800160d0     libucrt:winapi_thunks.obj
 0002:00002110       ??_C@_1EO@IJIOEFOH@?$AAa?$AAp?$AAi?$AA?9?$AAm?$AAs?$AA?9?$AAw?$AAi?$AAn?$AA?9?$AAr?$AAt?$AAc?$AAo@ 0000000180016110     libucrt:winapi_thunks.obj
 0002:00002160       ??_C@_1FG@HHGEKANL@?$AAa?$AAp?$AAi?$AA?9?$AAm?$AAs?$AA?9?$AAw?$AAi?$AAn?$AA?9?$AAs?$AAe?$AAc?$AAu@ 0000000180016160     libucrt:winapi_thunks.obj
 0002:000021c0       ??_C@_1EG@DBIOJECG@?$AAe?$AAx?$AAt?$AA?9?$AAm?$AAs?$AA?9?$AAw?$AAi?$AAn?$AA?9?$AAn?$AAt?$AAu?$AAs@ 00000001800161c0     libucrt:winapi_thunks.obj
 0002:00002210       ??_C@_1EO@FIHMJCLF@?$AAe?$AAx?$AAt?$AA?9?$AAm?$AAs?$AA?9?$AAw?$AAi?$AAn?$AA?9?$AAn?$AAt?$AAu?$AAs@ 0000000180016210     libucrt:winapi_thunks.obj
 0002:00002260       ??_C@_1BC@DNHGCMLG@?$AAa?$AAd?$AAv?$AAa?$AAp?$AAi?$AA3?$AA2@ 0000000180016260     libucrt:winapi_thunks.obj
 0002:00002278       ??_C@_1BC@GDMECMAK@?$AAk?$AAe?$AAr?$AAn?$AAe?$AAl?$AA3?$AA2@ 0000000180016278     libucrt:winapi_thunks.obj
 0002:00002290       ??_C@_1M@OAIMIKLP@?$AAn?$AAt?$AAd?$AAl?$AAl@ 0000000180016290     libucrt:winapi_thunks.obj
 0002:000022a0       ??_C@_1EG@DPGNFKGC@?$AAa?$AAp?$AAi?$AA?9?$AAm?$AAs?$AA?9?$AAw?$AAi?$AAn?$AA?9?$AAa?$AAp?$AAp?$AAm@ 00000001800162a0     libucrt:winapi_thunks.obj
 0002:000022e8       ??_C@_1O@BCCLBEOE@?$AAu?$AAs?$AAe?$AAr?$AA3?$AA2@ 00000001800162e8     libucrt:winapi_thunks.obj
 0002:000022f8       ??_C@_1BA@PFFKHIOG@?$AAa?$AAp?$AAi?$AA?9?$AAm?$AAs?$AA?9@ 00000001800162f8     libucrt:winapi_thunks.obj
 0002:00002308       ??_C@_1BA@IAIFMGEF@?$AAe?$AAx?$AAt?$AA?9?$AAm?$AAs?$AA?9@ 0000000180016308     libucrt:winapi_thunks.obj
 0002:00002320       ??_C@_0BA@FHFNEAED@AreFileApisANSI@ 0000000180016320     libucrt:winapi_thunks.obj
 0002:00002338       ??_C@_08KNHFBNJ@FlsAlloc@  0000000180016338     libucrt:winapi_thunks.obj
 0002:00002350       ??_C@_07PEJMOBNF@FlsFree@  0000000180016350     libucrt:winapi_thunks.obj
 0002:00002360       ??_C@_0M@GDNOONDI@FlsGetValue@ 0000000180016360     libucrt:winapi_thunks.obj
 0002:00002378       ??_C@_0M@JCPCPOEF@FlsSetValue@ 0000000180016378     libucrt:winapi_thunks.obj
 0002:00002390       ??_C@_0BM@HCFOFFN@InitializeCriticalSectionEx@ 0000000180016390     libucrt:winapi_thunks.obj
 0002:000023b8       ??_C@_0O@KKBNKAPF@LCMapStringEx@ 00000001800163b8     libucrt:winapi_thunks.obj
 0002:000023d0       ??_C@_0BB@HBDEELFH@LocaleNameToLCID@ 00000001800163d0     libucrt:winapi_thunks.obj
 0002:000023e8       ??_C@_0CF@OJOFEIGO@AppPolicyGetProcessTerminationM@ 00000001800163e8     libucrt:winapi_thunks.obj
 0002:00002410       __newctype                 0000000180016410     libucrt:ctype.obj
 0002:00002710       __newclmap                 0000000180016710     libucrt:ctype.obj
 0002:00002890       __newcumap                 0000000180016890     libucrt:ctype.obj
 0002:00002a10       ??_C@_15PJPFLCCM@?$AAu?$AAk@ 0000000180016a10     libucrt:get_qualified_locale.obj
 0002:00003860       ??_C@_15EMKDOKLE@?$AAa?$AAr@ 0000000180017860     libucrt:lcidtoname_downlevel.obj
 0002:00003868       ??_C@_15KNPADPLH@?$AAb?$AAg@ 0000000180017868     libucrt:lcidtoname_downlevel.obj
 0002:00003870       ??_C@_15EDMHLDMO@?$AAc?$AAa@ 0000000180017870     libucrt:lcidtoname_downlevel.obj
 0002:00003878       ??_C@_1O@BPEAJADD@?$AAz?$AAh?$AA?9?$AAC?$AAH?$AAS@ 0000000180017878     libucrt:lcidtoname_downlevel.obj
 0002:00003888       ??_C@_15LJNHCMNK@?$AAc?$AAs@ 0000000180017888     libucrt:lcidtoname_downlevel.obj
 0002:00003890       ??_C@_15FOMCIDHG@?$AAd?$AAa@ 0000000180017890     libucrt:lcidtoname_downlevel.obj
 0002:00003898       ??_C@_15NBKABECB@?$AAd?$AAe@ 0000000180017898     libucrt:lcidtoname_downlevel.obj
 0002:000038a0       ??_C@_15GHPEIIAO@?$AAe?$AAl@ 00000001800178a0     libucrt:lcidtoname_downlevel.obj
 0002:000038a8       ??_C@_15MNPNEAIF@?$AAe?$AAn@ 00000001800178a8     libucrt:lcidtoname_downlevel.obj
 0002:000038b0       ??_C@_15GPIOMPMH@?$AAe?$AAs@ 00000001800178b0     libucrt:lcidtoname_downlevel.obj
 0002:000038b8       ??_C@_15NGLOAKJC@?$AAf?$AAi@ 00000001800178b8     libucrt:lcidtoname_downlevel.obj
 0002:000038c0       ??_C@_15FBKGNKAM@?$AAf?$AAr@ 00000001800178c0     libucrt:lcidtoname_downlevel.obj
 0002:000038c8       ??_C@_15KGGCNEFK@?$AAh?$AAe@ 00000001800178c8     libucrt:lcidtoname_downlevel.obj
 0002:000038d0       ??_C@_15PGHLIDMF@?$AAh?$AAu@ 00000001800178d0     libucrt:lcidtoname_downlevel.obj
 0002:000038d8       ??_C@_15BIEMAPLM@?$AAi?$AAs@ 00000001800178d8     libucrt:lcidtoname_downlevel.obj
 0002:000038e0       ??_C@_15IFJLDHAF@?$AAi?$AAt@ 00000001800178e0     libucrt:lcidtoname_downlevel.obj
 0002:000038e8       ??_C@_15GEMIOCAG@?$AAj?$AAa@ 00000001800178e8     libucrt:lcidtoname_downlevel.obj
 0002:000038f0       ??_C@_15EPELEGJA@?$AAk?$AAo@ 00000001800178f0     libucrt:lcidtoname_downlevel.obj
 0002:000038f8       ??_C@_15NDDHIMN@?$AAn?$AAl@ 00000001800178f8     libucrt:lcidtoname_downlevel.obj
 0002:00003900       ??_C@_15BPIGNHCD@?$AAn?$AAo@ 0000000180017900     libucrt:lcidtoname_downlevel.obj
 0002:00003908       ??_C@_15DEOPBLCG@?$AAp?$AAl@ 0000000180017908     libucrt:lcidtoname_downlevel.obj
 0002:00003910       ??_C@_15KBECGEFG@?$AAp?$AAt@ 0000000180017910     libucrt:lcidtoname_downlevel.obj
 0002:00003918       ??_C@_15GLJCBFMD@?$AAr?$AAo@ 0000000180017918     libucrt:lcidtoname_downlevel.obj
 0002:00003920       ??_C@_15FEDGKCDI@?$AAr?$AAu@ 0000000180017920     libucrt:lcidtoname_downlevel.obj
 0002:00003928       ??_C@_15GLKMLLHM@?$AAh?$AAr@ 0000000180017928     libucrt:lcidtoname_downlevel.obj
 0002:00003930       ??_C@_15CPKMFBDB@?$AAs?$AAk@ 0000000180017930     libucrt:lcidtoname_downlevel.obj
 0002:00003938       ??_C@_15BAAIOGMK@?$AAs?$AAq@ 0000000180017938     libucrt:lcidtoname_downlevel.obj
 0002:00003940       ??_C@_15INNPNOHD@?$AAs?$AAv@ 0000000180017940     libucrt:lcidtoname_downlevel.obj
 0002:00003948       ??_C@_15CABMMOGH@?$AAt?$AAh@ 0000000180017948     libucrt:lcidtoname_downlevel.obj
 0002:00003950       ??_C@_15BPLIHJJM@?$AAt?$AAr@ 0000000180017950     libucrt:lcidtoname_downlevel.obj
 0002:00003958       ??_C@_15NEOEKKDJ@?$AAu?$AAr@ 0000000180017958     libucrt:lcidtoname_downlevel.obj
 0002:00003960       ??_C@_15NFICGAJK@?$AAi?$AAd@ 0000000180017960     libucrt:lcidtoname_downlevel.obj
 0002:00003968       ??_C@_15HPJPHDM@?$AAb?$AAe@ 0000000180017968     libucrt:lcidtoname_downlevel.obj
 0002:00003970       ??_C@_15LCHLGJII@?$AAs?$AAl@ 0000000180017970     libucrt:lcidtoname_downlevel.obj
 0002:00003978       ??_C@_15PCFJPHHO@?$AAe?$AAt@ 0000000180017978     libucrt:lcidtoname_downlevel.obj
 0002:00003980       ??_C@_15HPFPGODN@?$AAl?$AAv@ 0000000180017980     libucrt:lcidtoname_downlevel.obj
 0002:00003988       ??_C@_15NFFGKGLG@?$AAl?$AAt@ 0000000180017988     libucrt:lcidtoname_downlevel.obj
 0002:00003990       ??_C@_15BDAKCCHN@?$AAf?$AAa@ 0000000180017990     libucrt:lcidtoname_downlevel.obj
 0002:00003998       ??_C@_15NFGIAIAJ@?$AAv?$AAi@ 0000000180017998     libucrt:lcidtoname_downlevel.obj
 0002:000039a0       ??_C@_15LMKNDMHN@?$AAh?$AAy@ 00000001800179a0     libucrt:lcidtoname_downlevel.obj
 0002:000039a8       ??_C@_15IJBHMCFL@?$AAa?$AAz@ 00000001800179a8     libucrt:lcidtoname_downlevel.obj
 0002:000039b0       ??_C@_15EKOFJABL@?$AAe?$AAu@ 00000001800179b0     libucrt:lcidtoname_downlevel.obj
 0002:000039b8       ??_C@_15BGHADCNK@?$AAm?$AAk@ 00000001800179b8     libucrt:lcidtoname_downlevel.obj
 0002:000039c0       ??_C@_15JDNICKHM@?$AAa?$AAf@ 00000001800179c0     libucrt:lcidtoname_downlevel.obj
 0002:000039c8       ??_C@_15KPJEDBKD@?$AAk?$AAa@ 00000001800179c8     libucrt:lcidtoname_downlevel.obj
 0002:000039d0       ??_C@_15PDNFFFEO@?$AAf?$AAo@ 00000001800179d0     libucrt:lcidtoname_downlevel.obj
 0002:000039d8       ??_C@_15OMLEGLOC@?$AAh?$AAi@ 00000001800179d8     libucrt:lcidtoname_downlevel.obj
 0002:000039e0       ??_C@_15IDNNENKK@?$AAm?$AAs@ 00000001800179e0     libucrt:lcidtoname_downlevel.obj
 0002:000039e8       ??_C@_15MACJNBMH@?$AAk?$AAk@ 00000001800179e8     libucrt:lcidtoname_downlevel.obj
 0002:000039f0       ??_C@_15DKDJEOND@?$AAk?$AAy@ 00000001800179f0     libucrt:lcidtoname_downlevel.obj
 0002:000039f8       ??_C@_15DFGDLJBG@?$AAs?$AAw@ 00000001800179f8     libucrt:lcidtoname_downlevel.obj
 0002:00003a00       ??_C@_15BBFAICNG@?$AAu?$AAz@ 0000000180017a00     libucrt:lcidtoname_downlevel.obj
 0002:00003a08       ??_C@_15DKNDCGEA@?$AAt?$AAt@ 0000000180017a08     libucrt:lcidtoname_downlevel.obj
 0002:00003a10       ??_C@_15MGIFMDPL@?$AAp?$AAa@ 0000000180017a10     libucrt:lcidtoname_downlevel.obj
 0002:00003a18       ??_C@_15HCNDBBA@?$AAg?$AAu@ 0000000180017a18     libucrt:lcidtoname_downlevel.obj
 0002:00003a20       ??_C@_15FNBEIBON@?$AAt?$AAa@ 0000000180017a20     libucrt:lcidtoname_downlevel.obj
 0002:00003a28       ??_C@_15NCHGBGLK@?$AAt?$AAe@ 0000000180017a28     libucrt:lcidtoname_downlevel.obj
 0002:00003a30       ??_C@_15PHPHCBPF@?$AAk?$AAn@ 0000000180017a30     libucrt:lcidtoname_downlevel.obj
 0002:00003a38       ??_C@_15DLGBCKMP@?$AAm?$AAr@ 0000000180017a38     libucrt:lcidtoname_downlevel.obj
 0002:00003a40       ??_C@_15EABBLBFF@?$AAs?$AAa@ 0000000180017a40     libucrt:lcidtoname_downlevel.obj
 0002:00003a48       ??_C@_15CBKOMCOI@?$AAm?$AAn@ 0000000180017a48     libucrt:lcidtoname_downlevel.obj
 0002:00003a50       ??_C@_15CKDMCJAF@?$AAg?$AAl@ 0000000180017a50     libucrt:lcidtoname_downlevel.obj
 0002:00003a58       ??_C@_17CNJFBPG@?$AAk?$AAo?$AAk@ 0000000180017a58     libucrt:lcidtoname_downlevel.obj
 0002:00003a60       ??_C@_17FFBJICPL@?$AAs?$AAy?$AAr@ 0000000180017a60     libucrt:lcidtoname_downlevel.obj
 0002:00003a68       ??_C@_17KPNDCPAF@?$AAd?$AAi?$AAv@ 0000000180017a68     libucrt:lcidtoname_downlevel.obj
 0002:00003a70       ??_C@_1M@OKAHONE@?$AAa?$AAr?$AA?9?$AAS?$AAA@ 0000000180017a70     libucrt:lcidtoname_downlevel.obj
 0002:00003a80       ??_C@_1M@FFFIGIGK@?$AAb?$AAg?$AA?9?$AAB?$AAG@ 0000000180017a80     libucrt:lcidtoname_downlevel.obj
 0002:00003a90       ??_C@_1M@BJNKEDC@?$AAc?$AAa?$AA?9?$AAE?$AAS@ 0000000180017a90     libucrt:lcidtoname_downlevel.obj
 0002:00003aa0       ??_C@_1M@IJJHFJHA@?$AAc?$AAs?$AA?9?$AAC?$AAZ@ 0000000180017aa0     libucrt:lcidtoname_downlevel.obj
 0002:00003ab0       ??_C@_1M@CLPEOBGI@?$AAd?$AAa?$AA?9?$AAD?$AAK@ 0000000180017ab0     libucrt:lcidtoname_downlevel.obj
 0002:00003ac0       ??_C@_1M@MCMADGCB@?$AAd?$AAe?$AA?9?$AAD?$AAE@ 0000000180017ac0     libucrt:lcidtoname_downlevel.obj
 0002:00003ad0       ??_C@_1M@OOCKEMAM@?$AAe?$AAl?$AA?9?$AAG?$AAR@ 0000000180017ad0     libucrt:lcidtoname_downlevel.obj
 0002:00003ae0       ??_C@_1M@DDNJFGID@?$AAf?$AAi?$AA?9?$AAF?$AAI@ 0000000180017ae0     libucrt:lcidtoname_downlevel.obj
 0002:00003af0       ??_C@_1M@GLIPPMAC@?$AAf?$AAr?$AA?9?$AAF?$AAR@ 0000000180017af0     libucrt:lcidtoname_downlevel.obj
 0002:00003b00       ??_C@_1M@GFMCHPE@?$AAh?$AAe?$AA?9?$AAI?$AAL@ 0000000180017b00     libucrt:lcidtoname_downlevel.obj
 0002:00003b10       ??_C@_1M@MHLPGNKM@?$AAh?$AAu?$AA?9?$AAH?$AAU@ 0000000180017b10     libucrt:lcidtoname_downlevel.obj
 0002:00003b20       ??_C@_1M@LPDDNNPN@?$AAi?$AAs?$AA?9?$AAI?$AAS@ 0000000180017b20     libucrt:lcidtoname_downlevel.obj
 0002:00003b30       ??_C@_1M@MADIPODN@?$AAi?$AAt?$AA?9?$AAI?$AAT@ 0000000180017b30     libucrt:lcidtoname_downlevel.obj
 0002:00003b40       ??_C@_1M@IHBJJGG@?$AAn?$AAl?$AA?9?$AAN?$AAL@ 0000000180017b40     libucrt:lcidtoname_downlevel.obj
 0002:00003b50       ??_C@_1M@EANAGDL@?$AAn?$AAb?$AA?9?$AAN?$AAO@ 0000000180017b50     libucrt:lcidtoname_downlevel.obj
 0002:00003b60       ??_C@_1M@NEIEMEGP@?$AAp?$AAl?$AA?9?$AAP?$AAL@ 0000000180017b60     libucrt:lcidtoname_downlevel.obj
 0002:00003b70       ??_C@_1M@BOCFIGEP@?$AAp?$AAt?$AA?9?$AAB?$AAR@ 0000000180017b70     libucrt:lcidtoname_downlevel.obj
 0002:00003b80       ??_C@_1M@IMPFOPBG@?$AAr?$AAo?$AA?9?$AAR?$AAO@ 0000000180017b80     libucrt:lcidtoname_downlevel.obj
 0002:00003b90       ??_C@_1M@IDNNEJMM@?$AAr?$AAu?$AA?9?$AAR?$AAU@ 0000000180017b90     libucrt:lcidtoname_downlevel.obj
 0002:00003ba0       ??_C@_1M@LILEEOGM@?$AAh?$AAr?$AA?9?$AAH?$AAR@ 0000000180017ba0     libucrt:lcidtoname_downlevel.obj
 0002:00003bb0       ??_C@_1M@FKIFEHPB@?$AAs?$AAk?$AA?9?$AAS?$AAK@ 0000000180017bb0     libucrt:lcidtoname_downlevel.obj
 0002:00003bc0       ??_C@_1M@LJMAMNPJ@?$AAs?$AAq?$AA?9?$AAA?$AAL@ 0000000180017bc0     libucrt:lcidtoname_downlevel.obj
 0002:00003bd0       ??_C@_1M@GIAKDKJK@?$AAs?$AAv?$AA?9?$AAS?$AAE@ 0000000180017bd0     libucrt:lcidtoname_downlevel.obj
 0002:00003be0       ??_C@_1M@MKJKIKCL@?$AAt?$AAh?$AA?9?$AAT?$AAH@ 0000000180017be0     libucrt:lcidtoname_downlevel.obj
 0002:00003bf0       ??_C@_1M@MFLCCMPB@?$AAt?$AAr?$AA?9?$AAT?$AAR@ 0000000180017bf0     libucrt:lcidtoname_downlevel.obj
 0002:00003c00       ??_C@_1M@OIJHDKJN@?$AAu?$AAr?$AA?9?$AAP?$AAK@ 0000000180017c00     libucrt:lcidtoname_downlevel.obj
 0002:00003c10       ??_C@_1M@LHIPCIEK@?$AAi?$AAd?$AA?9?$AAI?$AAD@ 0000000180017c10     libucrt:lcidtoname_downlevel.obj
 0002:00003c20       ??_C@_1M@MFMOBGI@?$AAu?$AAk?$AA?9?$AAU?$AAA@ 0000000180017c20     libucrt:lcidtoname_downlevel.obj
 0002:00003c30       ??_C@_1M@OBGLJIPL@?$AAb?$AAe?$AA?9?$AAB?$AAY@ 0000000180017c30     libucrt:lcidtoname_downlevel.obj
 0002:00003c40       ??_C@_1M@BCFAJEAD@?$AAs?$AAl?$AA?9?$AAS?$AAI@ 0000000180017c40     libucrt:lcidtoname_downlevel.obj
 0002:00003c50       ??_C@_1M@FKFFEDDN@?$AAe?$AAt?$AA?9?$AAE?$AAE@ 0000000180017c50     libucrt:lcidtoname_downlevel.obj
 0002:00003c60       ??_C@_1M@KGKKAACI@?$AAl?$AAv?$AA?9?$AAL?$AAV@ 0000000180017c60     libucrt:lcidtoname_downlevel.obj
 0002:00003c70       ??_C@_1M@IFGBIJO@?$AAl?$AAt?$AA?9?$AAL?$AAT@ 0000000180017c70     libucrt:lcidtoname_downlevel.obj
 0002:00003c80       ??_C@_1M@FGEAHEDM@?$AAf?$AAa?$AA?9?$AAI?$AAR@ 0000000180017c80     libucrt:lcidtoname_downlevel.obj
 0002:00003c90       ??_C@_1M@KBMAIBFN@?$AAv?$AAi?$AA?9?$AAV?$AAN@ 0000000180017c90     libucrt:lcidtoname_downlevel.obj
 0002:00003ca0       ??_C@_1M@GPCBKDJK@?$AAh?$AAy?$AA?9?$AAA?$AAM@ 0000000180017ca0     libucrt:lcidtoname_downlevel.obj
 0002:00003cb0       ??_C@_1BG@BECMDDJB@?$AAa?$AAz?$AA?9?$AAA?$AAZ?$AA?9?$AAL?$AAa?$AAt?$AAn@ 0000000180017cb0     libucrt:lcidtoname_downlevel.obj
 0002:00003cc8       ??_C@_1M@MAOFCAEA@?$AAe?$AAu?$AA?9?$AAE?$AAS@ 0000000180017cc8     libucrt:lcidtoname_downlevel.obj
 0002:00003cd8       ??_C@_1M@IGHABKPI@?$AAm?$AAk?$AA?9?$AAM?$AAK@ 0000000180017cd8     libucrt:lcidtoname_downlevel.obj
 0002:00003ce8       ??_C@_1M@IAIGNEJG@?$AAt?$AAn?$AA?9?$AAZ?$AAA@ 0000000180017ce8     libucrt:lcidtoname_downlevel.obj
 0002:00003cf8       ??_C@_1M@IIJCOJFA@?$AAx?$AAh?$AA?9?$AAZ?$AAA@ 0000000180017cf8     libucrt:lcidtoname_downlevel.obj
 0002:00003d08       ??_C@_1M@LGPJHNJH@?$AAz?$AAu?$AA?9?$AAZ?$AAA@ 0000000180017d08     libucrt:lcidtoname_downlevel.obj
 0002:00003d18       ??_C@_1M@HOKAOIO@?$AAa?$AAf?$AA?9?$AAZ?$AAA@ 0000000180017d18     libucrt:lcidtoname_downlevel.obj
 0002:00003d28       ??_C@_1M@DPCLHLIE@?$AAk?$AAa?$AA?9?$AAG?$AAE@ 0000000180017d28     libucrt:lcidtoname_downlevel.obj
 0002:00003d38       ??_C@_1M@BLKMHJBI@?$AAf?$AAo?$AA?9?$AAF?$AAO@ 0000000180017d38     libucrt:lcidtoname_downlevel.obj
 0002:00003d48       ??_C@_1M@LGGJAPPB@?$AAh?$AAi?$AA?9?$AAI?$AAN@ 0000000180017d48     libucrt:lcidtoname_downlevel.obj
 0002:00003d58       ??_C@_1M@FIKPIHFE@?$AAm?$AAt?$AA?9?$AAM?$AAT@ 0000000180017d58     libucrt:lcidtoname_downlevel.obj
 0002:00003d68       ??_C@_1M@HEGGPBFA@?$AAs?$AAe?$AA?9?$AAN?$AAO@ 0000000180017d68     libucrt:lcidtoname_downlevel.obj
 0002:00003d78       ??_C@_1M@EIBJEEPA@?$AAm?$AAs?$AA?9?$AAM?$AAY@ 0000000180017d78     libucrt:lcidtoname_downlevel.obj
 0002:00003d88       ??_C@_1M@FHLBGMPP@?$AAk?$AAk?$AA?9?$AAK?$AAZ@ 0000000180017d88     libucrt:lcidtoname_downlevel.obj
 0002:00003d98       ??_C@_1M@NGJJLCGI@?$AAk?$AAy?$AA?9?$AAK?$AAG@ 0000000180017d98     libucrt:lcidtoname_downlevel.obj
 0002:00003da8       ??_C@_1M@GIENNBFC@?$AAs?$AAw?$AA?9?$AAK?$AAE@ 0000000180017da8     libucrt:lcidtoname_downlevel.obj
 0002:00003db8       ??_C@_1BG@NDGMJIMJ@?$AAu?$AAz?$AA?9?$AAU?$AAZ?$AA?9?$AAL?$AAa?$AAt?$AAn@ 0000000180017db8     libucrt:lcidtoname_downlevel.obj
 0002:00003dd0       ??_C@_1M@IDCCIHBC@?$AAt?$AAt?$AA?9?$AAR?$AAU@ 0000000180017dd0     libucrt:lcidtoname_downlevel.obj
 0002:00003de0       ??_C@_1M@LOICPMOJ@?$AAb?$AAn?$AA?9?$AAI?$AAN@ 0000000180017de0     libucrt:lcidtoname_downlevel.obj
 0002:00003df0       ??_C@_1M@KPKKNEAH@?$AAp?$AAa?$AA?9?$AAI?$AAN@ 0000000180017df0     libucrt:lcidtoname_downlevel.obj
 0002:00003e00       ??_C@_1M@PJGPPBOG@?$AAg?$AAu?$AA?9?$AAI?$AAN@ 0000000180017e00     libucrt:lcidtoname_downlevel.obj
 0002:00003e10       ??_C@_1M@KMKMOPHI@?$AAt?$AAa?$AA?9?$AAI?$AAN@ 0000000180017e10     libucrt:lcidtoname_downlevel.obj
 0002:00003e20       ??_C@_1M@KFEHEPAC@?$AAt?$AAe?$AA?9?$AAI?$AAN@ 0000000180017e20     libucrt:lcidtoname_downlevel.obj
 0002:00003e30       ??_C@_1M@CDCLMGHI@?$AAk?$AAn?$AA?9?$AAI?$AAN@ 0000000180017e30     libucrt:lcidtoname_downlevel.obj
 0002:00003e40       ??_C@_1M@MIODLDKF@?$AAm?$AAl?$AA?9?$AAI?$AAN@ 0000000180017e40     libucrt:lcidtoname_downlevel.obj
 0002:00003e50       ??_C@_1M@PBIEACPO@?$AAm?$AAr?$AA?9?$AAI?$AAN@ 0000000180017e50     libucrt:lcidtoname_downlevel.obj
 0002:00003e60       ??_C@_1M@NIDEAGPH@?$AAs?$AAa?$AA?9?$AAI?$AAN@ 0000000180017e60     libucrt:lcidtoname_downlevel.obj
 0002:00003e70       ??_C@_1M@FHIHCBIO@?$AAm?$AAn?$AA?9?$AAM?$AAN@ 0000000180017e70     libucrt:lcidtoname_downlevel.obj
 0002:00003e80       ??_C@_1M@JAIJPENP@?$AAc?$AAy?$AA?9?$AAG?$AAB@ 0000000180017e80     libucrt:lcidtoname_downlevel.obj
 0002:00003e90       ??_C@_1M@PHGFBEPN@?$AAg?$AAl?$AA?9?$AAE?$AAS@ 0000000180017e90     libucrt:lcidtoname_downlevel.obj
 0002:00003ea0       ??_C@_1O@KPIPDNCP@?$AAk?$AAo?$AAk?$AA?9?$AAI?$AAN@ 0000000180017ea0     libucrt:lcidtoname_downlevel.obj
 0002:00003eb0       ??_C@_1O@KNHJLDJA@?$AAs?$AAy?$AAr?$AA?9?$AAS?$AAY@ 0000000180017eb0     libucrt:lcidtoname_downlevel.obj
 0002:00003ec0       ??_C@_1O@MKEKBLAH@?$AAd?$AAi?$AAv?$AA?9?$AAM?$AAV@ 0000000180017ec0     libucrt:lcidtoname_downlevel.obj
 0002:00003ed0       ??_C@_1O@OHDCKDDF@?$AAq?$AAu?$AAz?$AA?9?$AAB?$AAO@ 0000000180017ed0     libucrt:lcidtoname_downlevel.obj
 0002:00003ee0       ??_C@_1M@LEPJNLFD@?$AAn?$AAs?$AA?9?$AAZ?$AAA@ 0000000180017ee0     libucrt:lcidtoname_downlevel.obj
 0002:00003ef0       ??_C@_1M@OMLEIIJB@?$AAm?$AAi?$AA?9?$AAN?$AAZ@ 0000000180017ef0     libucrt:lcidtoname_downlevel.obj
 0002:00003f00       ??_C@_1M@PMPEAILG@?$AAa?$AAr?$AA?9?$AAI?$AAQ@ 0000000180017f00     libucrt:lcidtoname_downlevel.obj
 0002:00003f10       ??_C@_1M@CNKPNOEE@?$AAd?$AAe?$AA?9?$AAC?$AAH@ 0000000180017f10     libucrt:lcidtoname_downlevel.obj
 0002:00003f20       ??_C@_1M@LKMGMLKO@?$AAe?$AAn?$AA?9?$AAG?$AAB@ 0000000180017f20     libucrt:lcidtoname_downlevel.obj
 0002:00003f30       ??_C@_1M@PGKJFFGL@?$AAe?$AAs?$AA?9?$AAM?$AAX@ 0000000180017f30     libucrt:lcidtoname_downlevel.obj
 0002:00003f40       ??_C@_1M@DNNANBDC@?$AAf?$AAr?$AA?9?$AAB?$AAE@ 0000000180017f40     libucrt:lcidtoname_downlevel.obj
 0002:00003f50       ??_C@_1M@HLGMDFHM@?$AAi?$AAt?$AA?9?$AAC?$AAH@ 0000000180017f50     libucrt:lcidtoname_downlevel.obj
 0002:00003f60       ??_C@_1M@CLLBGJH@?$AAn?$AAl?$AA?9?$AAB?$AAE@ 0000000180017f60     libucrt:lcidtoname_downlevel.obj
 0002:00003f70       ??_C@_1M@BODBOGLF@?$AAn?$AAn?$AA?9?$AAN?$AAO@ 0000000180017f70     libucrt:lcidtoname_downlevel.obj
 0002:00003f80       ??_C@_1M@HFFAHKAD@?$AAp?$AAt?$AA?9?$AAP?$AAT@ 0000000180017f80     libucrt:lcidtoname_downlevel.obj
 0002:00003f90       ??_C@_1BG@LNOAKHIE@?$AAs?$AAr?$AA?9?$AAS?$AAP?$AA?9?$AAL?$AAa?$AAt?$AAn@ 0000000180017f90     libucrt:lcidtoname_downlevel.obj
 0002:00003fa8       ??_C@_1M@HBMHBGAK@?$AAs?$AAv?$AA?9?$AAF?$AAI@ 0000000180017fa8     libucrt:lcidtoname_downlevel.obj
 0002:00003fb8       ??_C@_1BG@DGCJGJBE@?$AAa?$AAz?$AA?9?$AAA?$AAZ?$AA?9?$AAC?$AAy?$AAr?$AAl@ 0000000180017fb8     libucrt:lcidtoname_downlevel.obj
 0002:00003fd0       ??_C@_1M@KEJDAAHB@?$AAs?$AAe?$AA?9?$AAS?$AAE@ 0000000180017fd0     libucrt:lcidtoname_downlevel.obj
 0002:00003fe0       ??_C@_1M@HEIBJJAD@?$AAm?$AAs?$AA?9?$AAB?$AAN@ 0000000180017fe0     libucrt:lcidtoname_downlevel.obj
 0002:00003ff0       ??_C@_1BG@PBGJMCEM@?$AAu?$AAz?$AA?9?$AAU?$AAZ?$AA?9?$AAC?$AAy?$AAr?$AAl@ 0000000180017ff0     libucrt:lcidtoname_downlevel.obj
 0002:00004008       ??_C@_1O@LAOBCMDF@?$AAq?$AAu?$AAz?$AA?9?$AAE?$AAC@ 0000000180018008     libucrt:lcidtoname_downlevel.obj
 0002:00004018       ??_C@_1M@POEEMAIO@?$AAa?$AAr?$AA?9?$AAE?$AAG@ 0000000180018018     libucrt:lcidtoname_downlevel.obj
 0002:00004028       ??_C@_1M@EFAKDEDL@?$AAz?$AAh?$AA?9?$AAH?$AAK@ 0000000180018028     libucrt:lcidtoname_downlevel.obj
 0002:00004038       ??_C@_1M@HKKIJHGI@?$AAd?$AAe?$AA?9?$AAA?$AAT@ 0000000180018038     libucrt:lcidtoname_downlevel.obj
 0002:00004048       ??_C@_1M@KBFBEHJF@?$AAe?$AAn?$AA?9?$AAA?$AAU@ 0000000180018048     libucrt:lcidtoname_downlevel.obj
 0002:00004058       ??_C@_1M@MNPLFAAH@?$AAe?$AAs?$AA?9?$AAE?$AAS@ 0000000180018058     libucrt:lcidtoname_downlevel.obj
 0002:00004068       ??_C@_1M@HJOOJFMA@?$AAf?$AAr?$AA?9?$AAC?$AAA@ 0000000180018068     libucrt:lcidtoname_downlevel.obj
 0002:00004078       ??_C@_1BG@JPOFPNAB@?$AAs?$AAr?$AA?9?$AAS?$AAP?$AA?9?$AAC?$AAy?$AAr?$AAl@ 0000000180018078     libucrt:lcidtoname_downlevel.obj
 0002:00004090       ??_C@_1M@LNFOCMOB@?$AAs?$AAe?$AA?9?$AAF?$AAI@ 0000000180018090     libucrt:lcidtoname_downlevel.obj
 0002:000040a0       ??_C@_1O@MGJBOAMB@?$AAq?$AAu?$AAz?$AA?9?$AAP?$AAE@ 00000001800180a0     libucrt:lcidtoname_downlevel.obj
 0002:000040b0       ??_C@_1M@GJINLBOK@?$AAa?$AAr?$AA?9?$AAL?$AAY@ 00000001800180b0     libucrt:lcidtoname_downlevel.obj
 0002:000040c0       ??_C@_1M@GGMNHJNL@?$AAz?$AAh?$AA?9?$AAS?$AAG@ 00000001800180c0     libucrt:lcidtoname_downlevel.obj
 0002:000040d0       ??_C@_1M@HOIKODND@?$AAd?$AAe?$AA?9?$AAL?$AAU@ 00000001800180d0     libucrt:lcidtoname_downlevel.obj
 0002:000040e0       ??_C@_1M@DDOCCGFG@?$AAe?$AAn?$AA?9?$AAC?$AAA@ 00000001800180e0     libucrt:lcidtoname_downlevel.obj
 0002:000040f0       ??_C@_1M@BNOEMJLF@?$AAe?$AAs?$AA?9?$AAG?$AAT@ 00000001800180f0     libucrt:lcidtoname_downlevel.obj
 0002:00004100       ??_C@_1M@EOGNKEK@?$AAf?$AAr?$AA?9?$AAC?$AAH@ 0000000180018100     libucrt:lcidtoname_downlevel.obj
 0002:00004110       ??_C@_1M@FLIDJFHL@?$AAh?$AAr?$AA?9?$AAB?$AAA@ 0000000180018110     libucrt:lcidtoname_downlevel.obj
 0002:00004120       ??_C@_1O@FMCELNAJ@?$AAs?$AAm?$AAj?$AA?9?$AAN?$AAO@ 0000000180018120     libucrt:lcidtoname_downlevel.obj
 0002:00004130       ??_C@_1M@JHGLJMGJ@?$AAa?$AAr?$AA?9?$AAD?$AAZ@ 0000000180018130     libucrt:lcidtoname_downlevel.obj
 0002:00004140       ??_C@_1M@JKKFDCNP@?$AAz?$AAh?$AA?9?$AAM?$AAO@ 0000000180018140     libucrt:lcidtoname_downlevel.obj
 0002:00004150       ??_C@_1M@GEEFALPE@?$AAd?$AAe?$AA?9?$AAL?$AAI@ 0000000180018150     libucrt:lcidtoname_downlevel.obj
 0002:00004160       ??_C@_1M@IGEOFBG@?$AAe?$AAn?$AA?9?$AAN?$AAZ@ 0000000180018160     libucrt:lcidtoname_downlevel.obj
 0002:00004170       ??_C@_1M@KDBONEHP@?$AAe?$AAs?$AA?9?$AAC?$AAR@ 0000000180018170     libucrt:lcidtoname_downlevel.obj
 0002:00004180       ??_C@_1M@FHMDOHNN@?$AAf?$AAr?$AA?9?$AAL?$AAU@ 0000000180018180     libucrt:lcidtoname_downlevel.obj
 0002:00004190       ??_C@_1BG@NFKKMAFG@?$AAb?$AAs?$AA?9?$AAB?$AAA?$AA?9?$AAL?$AAa?$AAt?$AAn@ 0000000180018190     libucrt:lcidtoname_downlevel.obj
 0002:000041a8       ??_C@_1O@IMNBEMCI@?$AAs?$AAm?$AAj?$AA?9?$AAS?$AAE@ 00000001800181a8     libucrt:lcidtoname_downlevel.obj
 0002:000041b8       ??_C@_1M@DHHMBNDP@?$AAa?$AAr?$AA?9?$AAM?$AAA@ 00000001800181b8     libucrt:lcidtoname_downlevel.obj
 0002:000041c8       ??_C@_1M@BNBLJCGH@?$AAe?$AAn?$AA?9?$AAI?$AAE@ 00000001800181c8     libucrt:lcidtoname_downlevel.obj
 0002:000041d8       ??_C@_1M@GEPAFMDL@?$AAe?$AAs?$AA?9?$AAP?$AAA@ 00000001800181d8     libucrt:lcidtoname_downlevel.obj
 0002:000041e8       ??_C@_1M@OJONDMDL@?$AAf?$AAr?$AA?9?$AAM?$AAC@ 00000001800181e8     libucrt:lcidtoname_downlevel.obj
 0002:000041f8       ??_C@_1BG@OBCNFJB@?$AAs?$AAr?$AA?9?$AAB?$AAA?$AA?9?$AAL?$AAa?$AAt?$AAn@ 00000001800181f8     libucrt:lcidtoname_downlevel.obj
 0002:00004210       ??_C@_1O@KEMEEGPO@?$AAs?$AAm?$AAa?$AA?9?$AAN?$AAO@ 0000000180018210     libucrt:lcidtoname_downlevel.obj
 0002:00004220       ??_C@_1M@ELMGFODK@?$AAa?$AAr?$AA?9?$AAT?$AAN@ 0000000180018220     libucrt:lcidtoname_downlevel.obj
 0002:00004230       ??_C@_1M@BHDLHFAF@?$AAe?$AAn?$AA?9?$AAZ?$AAA@ 0000000180018230     libucrt:lcidtoname_downlevel.obj
 0002:00004240       ??_C@_1M@BMGIGLIF@?$AAe?$AAs?$AA?9?$AAD?$AAO@ 0000000180018240     libucrt:lcidtoname_downlevel.obj
 0002:00004250       ??_C@_1BG@CMBHIPBE@?$AAs?$AAr?$AA?9?$AAB?$AAA?$AA?9?$AAC?$AAy?$AAr?$AAl@ 0000000180018250     libucrt:lcidtoname_downlevel.obj
 0002:00004268       ??_C@_1O@HEDBLHNP@?$AAs?$AAm?$AAa?$AA?9?$AAS?$AAE@ 0000000180018268     libucrt:lcidtoname_downlevel.obj
 0002:00004278       ??_C@_1M@DAGCADIM@?$AAa?$AAr?$AA?9?$AAO?$AAM@ 0000000180018278     libucrt:lcidtoname_downlevel.obj
 0002:00004288       ??_C@_1M@FODLMICG@?$AAe?$AAn?$AA?9?$AAJ?$AAM@ 0000000180018288     libucrt:lcidtoname_downlevel.obj
 0002:00004298       ??_C@_1M@DNMLCIHB@?$AAe?$AAs?$AA?9?$AAV?$AAE@ 0000000180018298     libucrt:lcidtoname_downlevel.obj
 0002:000042a8       ??_C@_1O@EOKHMKJK@?$AAs?$AAm?$AAs?$AA?9?$AAF?$AAI@ 00000001800182a8     libucrt:lcidtoname_downlevel.obj
 0002:000042b8       ??_C@_1M@CAFJMKOF@?$AAa?$AAr?$AA?9?$AAY?$AAE@ 00000001800182b8     libucrt:lcidtoname_downlevel.obj
 0002:000042c8       ??_C@_1M@CBFHIJLI@?$AAe?$AAn?$AA?9?$AAC?$AAB@ 00000001800182c8     libucrt:lcidtoname_downlevel.obj
 0002:000042d8       ??_C@_1M@BGNFLDN@?$AAe?$AAs?$AA?9?$AAC?$AAO@ 00000001800182d8     libucrt:lcidtoname_downlevel.obj
 0002:000042e8       ??_C@_1O@JMPHMAMC@?$AAs?$AAm?$AAn?$AA?9?$AAF?$AAI@ 00000001800182e8     libucrt:lcidtoname_downlevel.obj
 0002:000042f8       ??_C@_1M@JLANABKE@?$AAa?$AAr?$AA?9?$AAS?$AAY@ 00000001800182f8     libucrt:lcidtoname_downlevel.obj
 0002:00004308       ??_C@_1M@HPKGCFGN@?$AAe?$AAn?$AA?9?$AAB?$AAZ@ 0000000180018308     libucrt:lcidtoname_downlevel.obj
 0002:00004318       ??_C@_1M@OLJCMLGM@?$AAe?$AAs?$AA?9?$AAP?$AAE@ 0000000180018318     libucrt:lcidtoname_downlevel.obj
 0002:00004328       ??_C@_1M@MKKGFKLE@?$AAa?$AAr?$AA?9?$AAJ?$AAO@ 0000000180018328     libucrt:lcidtoname_downlevel.obj
 0002:00004338       ??_C@_1M@EKPGLDNI@?$AAe?$AAn?$AA?9?$AAT?$AAT@ 0000000180018338     libucrt:lcidtoname_downlevel.obj
 0002:00004348       ??_C@_1M@OONGHFHE@?$AAe?$AAs?$AA?9?$AAA?$AAR@ 0000000180018348     libucrt:lcidtoname_downlevel.obj
 0002:00004358       ??_C@_1M@OOJFGBHE@?$AAa?$AAr?$AA?9?$AAL?$AAB@ 0000000180018358     libucrt:lcidtoname_downlevel.obj
 0002:00004368       ??_C@_1M@GCEJHNEG@?$AAe?$AAn?$AA?9?$AAZ?$AAW@ 0000000180018368     libucrt:lcidtoname_downlevel.obj
 0002:00004378       ??_C@_1M@JNOCAHJI@?$AAe?$AAs?$AA?9?$AAE?$AAC@ 0000000180018378     libucrt:lcidtoname_downlevel.obj
 0002:00004388       ??_C@_1M@JEFHPGGB@?$AAa?$AAr?$AA?9?$AAK?$AAW@ 0000000180018388     libucrt:lcidtoname_downlevel.obj
 0002:00004398       ??_C@_1M@MLKIBJOJ@?$AAe?$AAn?$AA?9?$AAP?$AAH@ 0000000180018398     libucrt:lcidtoname_downlevel.obj
 0002:000043a8       ??_C@_1M@BDNIPEND@?$AAe?$AAs?$AA?9?$AAC?$AAL@ 00000001800183a8     libucrt:lcidtoname_downlevel.obj
 0002:000043b8       ??_C@_1M@MPNMEKBD@?$AAa?$AAr?$AA?9?$AAA?$AAE@ 00000001800183b8     libucrt:lcidtoname_downlevel.obj
 0002:000043c8       ??_C@_1M@KBJALCPI@?$AAe?$AAs?$AA?9?$AAU?$AAY@ 00000001800183c8     libucrt:lcidtoname_downlevel.obj
 0002:000043d8       ??_C@_1M@LLCCOAGA@?$AAa?$AAr?$AA?9?$AAB?$AAH@ 00000001800183d8     libucrt:lcidtoname_downlevel.obj
 0002:000043e8       ??_C@_1M@PBFNCDEL@?$AAe?$AAs?$AA?9?$AAP?$AAY@ 00000001800183e8     libucrt:lcidtoname_downlevel.obj
 0002:000043f8       ??_C@_1M@EDGINPNP@?$AAa?$AAr?$AA?9?$AAQ?$AAA@ 00000001800183f8     libucrt:lcidtoname_downlevel.obj
 0002:00004408       ??_C@_1M@MKDBIIJI@?$AAe?$AAs?$AA?9?$AAB?$AAO@ 0000000180018408     libucrt:lcidtoname_downlevel.obj
 0002:00004418       ??_C@_1M@CPKKEBLD@?$AAe?$AAs?$AA?9?$AAS?$AAV@ 0000000180018418     libucrt:lcidtoname_downlevel.obj
 0002:00004428       ??_C@_1M@NDBGMMJL@?$AAe?$AAs?$AA?9?$AAH?$AAN@ 0000000180018428     libucrt:lcidtoname_downlevel.obj
 0002:00004438       ??_C@_1M@JIJIBHDP@?$AAe?$AAs?$AA?9?$AAN?$AAI@ 0000000180018438     libucrt:lcidtoname_downlevel.obj
 0002:00004448       ??_C@_1M@CGFMKEEK@?$AAe?$AAs?$AA?9?$AAP?$AAR@ 0000000180018448     libucrt:lcidtoname_downlevel.obj
 0002:00004458       ??_C@_1O@ICJHKIIK@?$AAz?$AAh?$AA?9?$AAC?$AAH?$AAT@ 0000000180018458     libucrt:lcidtoname_downlevel.obj
 0002:00004468       ??_C@_15CLNEJCE@?$AAs?$AAr@ 0000000180018468     libucrt:lcidtoname_downlevel.obj
 0002:000052b0       ??_C@_1M@KAHEKEIG@?$AAa?$AAf?$AA?9?$AAz?$AAa@ 00000001800192b0     libucrt:lcidtoname_downlevel.obj
 0002:000052c0       ??_C@_1M@GIECOABL@?$AAa?$AAr?$AA?9?$AAa?$AAe@ 00000001800192c0     libucrt:lcidtoname_downlevel.obj
 0002:000052d0       ??_C@_1M@BMLMEKGI@?$AAa?$AAr?$AA?9?$AAb?$AAh@ 00000001800192d0     libucrt:lcidtoname_downlevel.obj
 0002:000052e0       ??_C@_1M@DAPFDGGB@?$AAa?$AAr?$AA?9?$AAd?$AAz@ 00000001800192e0     libucrt:lcidtoname_downlevel.obj
 0002:000052f0       ??_C@_1M@FJNKGKIG@?$AAa?$AAr?$AA?9?$AAe?$AAg@ 00000001800192f0     libucrt:lcidtoname_downlevel.obj
 0002:00005300       ??_C@_1M@FLGKKCLO@?$AAa?$AAr?$AA?9?$AAi?$AAq@ 0000000180019300     libucrt:lcidtoname_downlevel.obj
 0002:00005310       ??_C@_1M@GNDIPALM@?$AAa?$AAr?$AA?9?$AAj?$AAo@ 0000000180019310     libucrt:lcidtoname_downlevel.obj
 0002:00005320       ??_C@_1M@DDMJFMGJ@?$AAa?$AAr?$AA?9?$AAk?$AAw@ 0000000180019320     libucrt:lcidtoname_downlevel.obj
 0002:00005330       ??_C@_1M@EJALMLHM@?$AAa?$AAr?$AA?9?$AAl?$AAb@ 0000000180019330     libucrt:lcidtoname_downlevel.obj
 0002:00005340       ??_C@_1M@MOBDBLOC@?$AAa?$AAr?$AA?9?$AAl?$AAy@ 0000000180019340     libucrt:lcidtoname_downlevel.obj
 0002:00005350       ??_C@_1M@JAOCLHDH@?$AAa?$AAr?$AA?9?$AAm?$AAa@ 0000000180019350     libucrt:lcidtoname_downlevel.obj
 0002:00005360       ??_C@_1M@JHPMKJIE@?$AAa?$AAr?$AA?9?$AAo?$AAm@ 0000000180019360     libucrt:lcidtoname_downlevel.obj
 0002:00005370       ??_C@_1M@OEPGHFNH@?$AAa?$AAr?$AA?9?$AAq?$AAa@ 0000000180019370     libucrt:lcidtoname_downlevel.obj
 0002:00005380       ??_C@_1M@KJDONENM@?$AAa?$AAr?$AA?9?$AAs?$AAa@ 0000000180019380     libucrt:lcidtoname_downlevel.obj
 0002:00005390       ??_C@_1M@DMJDKLKM@?$AAa?$AAr?$AA?9?$AAs?$AAy@ 0000000180019390     libucrt:lcidtoname_downlevel.obj
 0002:000053a0       ??_C@_1M@OMFIPEDC@?$AAa?$AAr?$AA?9?$AAt?$AAn@ 00000001800193a0     libucrt:lcidtoname_downlevel.obj
 0002:000053b0       ??_C@_1M@IHMHGAON@?$AAa?$AAr?$AA?9?$AAy?$AAe@ 00000001800193b0     libucrt:lcidtoname_downlevel.obj
 0002:000053c0       ??_C@_1BG@KDCPGJGB@?$AAa?$AAz?$AA?9?$AAa?$AAz?$AA?9?$AAc?$AAy?$AAr?$AAl@ 00000001800193c0     libucrt:lcidtoname_downlevel.obj
 0002:000053d8       ??_C@_1BG@IBCKDDOE@?$AAa?$AAz?$AA?9?$AAa?$AAz?$AA?9?$AAl?$AAa?$AAt?$AAn@ 00000001800193d8     libucrt:lcidtoname_downlevel.obj
 0002:000053f0       ??_C@_1M@EGPFDCPD@?$AAb?$AAe?$AA?9?$AAb?$AAy@ 00000001800193f0     libucrt:lcidtoname_downlevel.obj
 0002:00005400       ??_C@_1M@PCMGMCGC@?$AAb?$AAg?$AA?9?$AAb?$AAg@ 0000000180019400     libucrt:lcidtoname_downlevel.obj
 0002:00005410       ??_C@_1M@BJBMFGOB@?$AAb?$AAn?$AA?9?$AAi?$AAn@ 0000000180019410     libucrt:lcidtoname_downlevel.obj
 0002:00005420       ??_C@_1BG@EAKMMACD@?$AAb?$AAs?$AA?9?$AAb?$AAa?$AA?9?$AAl?$AAa?$AAt?$AAn@ 0000000180019420     libucrt:lcidtoname_downlevel.obj
 0002:00005438       ??_C@_1M@KGADAODK@?$AAc?$AAa?$AA?9?$AAe?$AAs@ 0000000180019438     libucrt:lcidtoname_downlevel.obj
 0002:00005448       ??_C@_1M@COAJPDHI@?$AAc?$AAs?$AA?9?$AAc?$AAz@ 0000000180019448     libucrt:lcidtoname_downlevel.obj
 0002:00005458       ??_C@_1M@DHBHFONH@?$AAc?$AAy?$AA?9?$AAg?$AAb@ 0000000180019458     libucrt:lcidtoname_downlevel.obj
 0002:00005468       ??_C@_1M@IMGKELGA@?$AAd?$AAa?$AA?9?$AAd?$AAk@ 0000000180019468     libucrt:lcidtoname_downlevel.obj
 0002:00005478       ??_C@_1M@NNDGDNGA@?$AAd?$AAe?$AA?9?$AAa?$AAt@ 0000000180019478     libucrt:lcidtoname_downlevel.obj
 0002:00005488       ??_C@_1M@IKDBHEEM@?$AAd?$AAe?$AA?9?$AAc?$AAh@ 0000000180019488     libucrt:lcidtoname_downlevel.obj
 0002:00005498       ??_C@_1M@GFFOJMCJ@?$AAd?$AAe?$AA?9?$AAd?$AAe@ 0000000180019498     libucrt:lcidtoname_downlevel.obj
 0002:000054a8       ??_C@_1M@MDNLKBPM@?$AAd?$AAe?$AA?9?$AAl?$AAi@ 00000001800194a8     libucrt:lcidtoname_downlevel.obj
 0002:000054b8       ??_C@_1M@NJBEEJNL@?$AAd?$AAe?$AA?9?$AAl?$AAu@ 00000001800194b8     libucrt:lcidtoname_downlevel.obj
 0002:000054c8       ??_C@_1O@GNNELBAP@?$AAd?$AAi?$AAv?$AA?9?$AAm?$AAv@ 00000001800194c8     libucrt:lcidtoname_downlevel.obj
 0002:000054d8       ??_C@_1M@EJLEOGAE@?$AAe?$AAl?$AA?9?$AAg?$AAr@ 00000001800194d8     libucrt:lcidtoname_downlevel.obj
 0002:000054e8       ??_C@_1M@GMPONJN@?$AAe?$AAn?$AA?9?$AAa?$AAu@ 00000001800194e8     libucrt:lcidtoname_downlevel.obj
 0002:000054f8       ??_C@_1M@NIDIIPGF@?$AAe?$AAn?$AA?9?$AAb?$AAz@ 00000001800194f8     libucrt:lcidtoname_downlevel.obj
 0002:00005508       ??_C@_1M@JEHMIMFO@?$AAe?$AAn?$AA?9?$AAc?$AAa@ 0000000180019508     libucrt:lcidtoname_downlevel.obj
 0002:00005518       ??_C@_1M@IGMJCDLA@?$AAe?$AAn?$AA?9?$AAc?$AAb@ 0000000180019518     libucrt:lcidtoname_downlevel.obj
 0002:00005528       ??_C@_1M@BNFIGBKG@?$AAe?$AAn?$AA?9?$AAg?$AAb@ 0000000180019528     libucrt:lcidtoname_downlevel.obj
 0002:00005538       ??_C@_1M@LKIFDIGP@?$AAe?$AAn?$AA?9?$AAi?$AAe@ 0000000180019538     libucrt:lcidtoname_downlevel.obj
 0002:00005548       ??_C@_1M@PJKFGCCO@?$AAe?$AAn?$AA?9?$AAj?$AAm@ 0000000180019548     libucrt:lcidtoname_downlevel.obj
 0002:00005558       ??_C@_1M@KPPKEPBO@?$AAe?$AAn?$AA?9?$AAn?$AAz@ 0000000180019558     libucrt:lcidtoname_downlevel.obj
 0002:00005568       ??_C@_1M@GMDGLDOB@?$AAe?$AAn?$AA?9?$AAp?$AAh@ 0000000180019568     libucrt:lcidtoname_downlevel.obj
 0002:00005578       ??_C@_1M@ONGIBJNA@?$AAe?$AAn?$AA?9?$AAt?$AAt@ 0000000180019578     libucrt:lcidtoname_downlevel.obj
 0002:00005588       ??_C@_1M@LLODPCMM@?$AAe?$AAn?$AA?9?$AAu?$AAs@ 0000000180019588     libucrt:lcidtoname_downlevel.obj
 0002:00005598       ??_C@_1M@LAKFNPAN@?$AAe?$AAn?$AA?9?$AAz?$AAa@ 0000000180019598     libucrt:lcidtoname_downlevel.obj
 0002:000055a8       ??_C@_1M@MFNHNHEO@?$AAe?$AAn?$AA?9?$AAz?$AAw@ 00000001800195a8     libucrt:lcidtoname_downlevel.obj
 0002:000055b8       ??_C@_1M@EJEINPHM@?$AAe?$AAs?$AA?9?$AAa?$AAr@ 00000001800195b8     libucrt:lcidtoname_downlevel.obj
 0002:000055c8       ??_C@_1M@GNKPCCJA@?$AAe?$AAs?$AA?9?$AAb?$AAo@ 00000001800195c8     libucrt:lcidtoname_downlevel.obj
 0002:000055d8       ??_C@_1M@LEEGFONL@?$AAe?$AAs?$AA?9?$AAc?$AAl@ 00000001800195d8     libucrt:lcidtoname_downlevel.obj
 0002:000055e8       ??_C@_1M@KGPDPBDF@?$AAe?$AAs?$AA?9?$AAc?$AAo@ 00000001800195e8     libucrt:lcidtoname_downlevel.obj
 0002:000055f8       ??_C@_1M@EIAHOHH@?$AAe?$AAs?$AA?9?$AAc?$AAr@ 00000001800195f8     libucrt:lcidtoname_downlevel.obj
 0002:00005608       ??_C@_1M@LLPGMBIN@?$AAe?$AAs?$AA?9?$AAd?$AAo@ 0000000180019608     libucrt:lcidtoname_downlevel.obj
 0002:00005618       ??_C@_1M@DKHMKNJA@?$AAe?$AAs?$AA?9?$AAe?$AAc@ 0000000180019618     libucrt:lcidtoname_downlevel.obj
 0002:00005628       ??_C@_1M@GKGFPKAP@?$AAe?$AAs?$AA?9?$AAe?$AAs@ 0000000180019628     libucrt:lcidtoname_downlevel.obj
 0002:00005638       ??_C@_1M@LKHKGDLN@?$AAe?$AAs?$AA?9?$AAg?$AAt@ 0000000180019638     libucrt:lcidtoname_downlevel.obj
 0002:00005648       ??_C@_1M@HEIIGGJD@?$AAe?$AAs?$AA?9?$AAh?$AAn@ 0000000180019648     libucrt:lcidtoname_downlevel.obj
 0002:00005658       ??_C@_1M@FBDHPPGD@?$AAe?$AAs?$AA?9?$AAm?$AAx@ 0000000180019658     libucrt:lcidtoname_downlevel.obj
 0002:00005668       ??_C@_1M@DPAGLNDH@?$AAe?$AAs?$AA?9?$AAn?$AAi@ 0000000180019668     libucrt:lcidtoname_downlevel.obj
 0002:00005678       ??_C@_1M@MDGOPGDD@?$AAe?$AAs?$AA?9?$AAp?$AAa@ 0000000180019678     libucrt:lcidtoname_downlevel.obj
 0002:00005688       ??_C@_1M@EMAMGBGE@?$AAe?$AAs?$AA?9?$AAp?$AAe@ 0000000180019688     libucrt:lcidtoname_downlevel.obj
 0002:00005698       ??_C@_1M@IBMCAOEC@?$AAe?$AAs?$AA?9?$AAp?$AAr@ 0000000180019698     libucrt:lcidtoname_downlevel.obj
 0002:000056a8       ??_C@_1M@FGMDIJED@?$AAe?$AAs?$AA?9?$AAp?$AAy@ 00000001800196a8     libucrt:lcidtoname_downlevel.obj
 0002:000056b8       ??_C@_1M@IIDEOLLL@?$AAe?$AAs?$AA?9?$AAs?$AAv@ 00000001800196b8     libucrt:lcidtoname_downlevel.obj
 0002:000056c8       ??_C@_1M@GAOBIPA@?$AAe?$AAs?$AA?9?$AAu?$AAy@ 00000001800196c8     libucrt:lcidtoname_downlevel.obj
 0002:000056d8       ??_C@_1M@JKFFICHJ@?$AAe?$AAs?$AA?9?$AAv?$AAe@ 00000001800196d8     libucrt:lcidtoname_downlevel.obj
 0002:000056e8       ??_C@_1M@PNMLOJDF@?$AAe?$AAt?$AA?9?$AAe?$AAe@ 00000001800196e8     libucrt:lcidtoname_downlevel.obj
 0002:000056f8       ??_C@_1M@GHHLIKEI@?$AAe?$AAu?$AA?9?$AAe?$AAs@ 00000001800196f8     libucrt:lcidtoname_downlevel.obj
 0002:00005708       ??_C@_1M@PBNONODE@?$AAf?$AAa?$AA?9?$AAi?$AAr@ 0000000180019708     libucrt:lcidtoname_downlevel.obj
 0002:00005718       ??_C@_1M@JEEHPMIL@?$AAf?$AAi?$AA?9?$AAf?$AAi@ 0000000180019718     libucrt:lcidtoname_downlevel.obj
 0002:00005728       ??_C@_1M@LMDCNDBA@?$AAf?$AAo?$AA?9?$AAf?$AAo@ 0000000180019728     libucrt:lcidtoname_downlevel.obj
 0002:00005738       ??_C@_1M@JKEOHLDK@?$AAf?$AAr?$AA?9?$AAb?$AAe@ 0000000180019738     libucrt:lcidtoname_downlevel.obj
 0002:00005748       ??_C@_1M@NOHADPMI@?$AAf?$AAr?$AA?9?$AAc?$AAa@ 0000000180019748     libucrt:lcidtoname_downlevel.obj
 0002:00005758       ??_C@_1M@KDHIHAEC@?$AAf?$AAr?$AA?9?$AAc?$AAh@ 0000000180019758     libucrt:lcidtoname_downlevel.obj
 0002:00005768       ??_C@_1M@MMBBFGAK@?$AAf?$AAr?$AA?9?$AAf?$AAr@ 0000000180019768     libucrt:lcidtoname_downlevel.obj
 0002:00005778       ??_C@_1M@PAFNENNF@?$AAf?$AAr?$AA?9?$AAl?$AAu@ 0000000180019778     libucrt:lcidtoname_downlevel.obj
 0002:00005788       ??_C@_1M@EOHDJGDD@?$AAf?$AAr?$AA?9?$AAm?$AAc@ 0000000180019788     libucrt:lcidtoname_downlevel.obj
 0002:00005798       ??_C@_1M@FAPLLOPF@?$AAg?$AAl?$AA?9?$AAe?$AAs@ 0000000180019798     libucrt:lcidtoname_downlevel.obj
 0002:000057a8       ??_C@_1M@FOPBFLOO@?$AAg?$AAu?$AA?9?$AAi?$AAn@ 00000001800197a8     libucrt:lcidtoname_downlevel.obj
 0002:000057b8       ??_C@_1M@KBMCINPM@?$AAh?$AAe?$AA?9?$AAi?$AAl@ 00000001800197b8     libucrt:lcidtoname_downlevel.obj
 0002:000057c8       ??_C@_1M@BBPHKFPJ@?$AAh?$AAi?$AA?9?$AAi?$AAn@ 00000001800197c8     libucrt:lcidtoname_downlevel.obj
 0002:000057d8       ??_C@_1M@PMBNDPHD@?$AAh?$AAr?$AA?9?$AAb?$AAa@ 00000001800197d8     libucrt:lcidtoname_downlevel.obj
 0002:000057e8       ??_C@_1M@BPCKOEGE@?$AAh?$AAr?$AA?9?$AAh?$AAr@ 00000001800197e8     libucrt:lcidtoname_downlevel.obj
 0002:000057f8       ??_C@_1M@GACBMHKE@?$AAh?$AAu?$AA?9?$AAh?$AAu@ 00000001800197f8     libucrt:lcidtoname_downlevel.obj
 0002:00005808       ??_C@_1M@MILPAJJC@?$AAh?$AAy?$AA?9?$AAa?$AAm@ 0000000180019808     libucrt:lcidtoname_downlevel.obj
 0002:00005818       ??_C@_1M@BABBICEC@?$AAi?$AAd?$AA?9?$AAi?$AAd@ 0000000180019818     libucrt:lcidtoname_downlevel.obj
 0002:00005828       ??_C@_1M@BIKNHHPF@?$AAi?$AAs?$AA?9?$AAi?$AAs@ 0000000180019828     libucrt:lcidtoname_downlevel.obj
 0002:00005838       ??_C@_1M@NMPCJPHE@?$AAi?$AAt?$AA?9?$AAc?$AAh@ 0000000180019838     libucrt:lcidtoname_downlevel.obj
 0002:00005848       ??_C@_1M@GHKGFEDF@?$AAi?$AAt?$AA?9?$AAi?$AAt@ 0000000180019848     libucrt:lcidtoname_downlevel.obj
 0002:00005858       ??_C@_1M@NIEJCJJA@?$AAj?$AAa?$AA?9?$AAj?$AAp@ 0000000180019858     libucrt:lcidtoname_downlevel.obj
 0002:00005868       ??_C@_1M@JILFNBIM@?$AAk?$AAa?$AA?9?$AAg?$AAe@ 0000000180019868     libucrt:lcidtoname_downlevel.obj
 0002:00005878       ??_C@_1M@PACPMGPH@?$AAk?$AAk?$AA?9?$AAk?$AAz@ 0000000180019878     libucrt:lcidtoname_downlevel.obj
 0002:00005888       ??_C@_1M@IELFGMHA@?$AAk?$AAn?$AA?9?$AAi?$AAn@ 0000000180019888     libucrt:lcidtoname_downlevel.obj
 0002:00005898       ??_C@_1O@IBBJHCH@?$AAk?$AAo?$AAk?$AA?9?$AAi?$AAn@ 0000000180019898     libucrt:lcidtoname_downlevel.obj
 0002:000058a8       ??_C@_1M@DMHAEOGC@?$AAk?$AAo?$AA?9?$AAk?$AAr@ 00000001800198a8     libucrt:lcidtoname_downlevel.obj
 0002:000058b8       ??_C@_1M@HBAHBIGA@?$AAk?$AAy?$AA?9?$AAk?$AAg@ 00000001800198b8     libucrt:lcidtoname_downlevel.obj
 0002:000058c8       ??_C@_1M@KPMILCJG@?$AAl?$AAt?$AA?9?$AAl?$AAt@ 00000001800198c8     libucrt:lcidtoname_downlevel.obj
 0002:000058d8       ??_C@_1M@BDEKKCA@?$AAl?$AAv?$AA?9?$AAl?$AAv@ 00000001800198d8     libucrt:lcidtoname_downlevel.obj
 0002:000058e8       ??_C@_1M@ELCKCCJJ@?$AAm?$AAi?$AA?9?$AAn?$AAz@ 00000001800198e8     libucrt:lcidtoname_downlevel.obj
 0002:000058f8       ??_C@_1M@CBOOLAPA@?$AAm?$AAk?$AA?9?$AAm?$AAk@ 00000001800198f8     libucrt:lcidtoname_downlevel.obj
 0002:00005908       ??_C@_1M@GPHNBJKN@?$AAm?$AAl?$AA?9?$AAi?$AAn@ 0000000180019908     libucrt:lcidtoname_downlevel.obj
 0002:00005918       ??_C@_1M@PABJILIG@?$AAm?$AAn?$AA?9?$AAm?$AAn@ 0000000180019918     libucrt:lcidtoname_downlevel.obj
 0002:00005928       ??_C@_1M@FGBKKIPG@?$AAm?$AAr?$AA?9?$AAi?$AAn@ 0000000180019928     libucrt:lcidtoname_downlevel.obj
 0002:00005938       ??_C@_1M@NDBPDDAL@?$AAm?$AAs?$AA?9?$AAb?$AAn@ 0000000180019938     libucrt:lcidtoname_downlevel.obj
 0002:00005948       ??_C@_1M@OPIHOOPI@?$AAm?$AAs?$AA?9?$AAm?$AAy@ 0000000180019948     libucrt:lcidtoname_downlevel.obj
 0002:00005958       ??_C@_1M@PPDBCNFM@?$AAm?$AAt?$AA?9?$AAm?$AAt@ 0000000180019958     libucrt:lcidtoname_downlevel.obj
 0002:00005968       ??_C@_1M@KDJDKMDD@?$AAn?$AAb?$AA?9?$AAn?$AAo@ 0000000180019968     libucrt:lcidtoname_downlevel.obj
 0002:00005978       ??_C@_1M@KFCFLMJP@?$AAn?$AAl?$AA?9?$AAb?$AAe@ 0000000180019978     libucrt:lcidtoname_downlevel.obj
 0002:00005988       ??_C@_1M@KPOPDDGO@?$AAn?$AAl?$AA?9?$AAn?$AAl@ 0000000180019988     libucrt:lcidtoname_downlevel.obj
 0002:00005998       ??_C@_1M@LJKPEMLN@?$AAn?$AAn?$AA?9?$AAn?$AAo@ 0000000180019998     libucrt:lcidtoname_downlevel.obj
 0002:000059a8       ??_C@_1M@BDGHHBFL@?$AAn?$AAs?$AA?9?$AAz?$AAa@ 00000001800199a8     libucrt:lcidtoname_downlevel.obj
 0002:000059b8       ??_C@_1M@IDEHOAP@?$AAp?$AAa?$AA?9?$AAi?$AAn@ 00000001800199b8     libucrt:lcidtoname_downlevel.obj
 0002:000059c8       ??_C@_1M@HDBKGOGH@?$AAp?$AAl?$AA?9?$AAp?$AAl@ 00000001800199c8     libucrt:lcidtoname_downlevel.obj
 0002:000059d8       ??_C@_1M@LJLLCMEH@?$AAp?$AAt?$AA?9?$AAb?$AAr@ 00000001800199d8     libucrt:lcidtoname_downlevel.obj
 0002:000059e8       ??_C@_1M@NCMONAAL@?$AAp?$AAt?$AA?9?$AAp?$AAt@ 00000001800199e8     libucrt:lcidtoname_downlevel.obj
 0002:000059f8       ??_C@_1O@EAKMAJDN@?$AAq?$AAu?$AAz?$AA?9?$AAb?$AAo@ 00000001800199f8     libucrt:lcidtoname_downlevel.obj
 0002:00005a08       ??_C@_1O@BHHPIGDN@?$AAq?$AAu?$AAz?$AA?9?$AAe?$AAc@ 0000000180019a08     libucrt:lcidtoname_downlevel.obj
 0002:00005a18       ??_C@_1O@GBAPEKMJ@?$AAq?$AAu?$AAz?$AA?9?$AAp?$AAe@ 0000000180019a18     libucrt:lcidtoname_downlevel.obj
 0002:00005a28       ??_C@_1M@CLGLEFBO@?$AAr?$AAo?$AA?9?$AAr?$AAo@ 0000000180019a28     libucrt:lcidtoname_downlevel.obj
 0002:00005a38       ??_C@_1M@CEEDODME@?$AAr?$AAu?$AA?9?$AAr?$AAu@ 0000000180019a38     libucrt:lcidtoname_downlevel.obj
 0002:00005a48       ??_C@_1M@HPKKKMPP@?$AAs?$AAa?$AA?9?$AAi?$AAn@ 0000000180019a48     libucrt:lcidtoname_downlevel.obj
 0002:00005a58       ??_C@_1M@BKMAIGOJ@?$AAs?$AAe?$AA?9?$AAf?$AAi@ 0000000180019a58     libucrt:lcidtoname_downlevel.obj
 0002:00005a68       ??_C@_1M@NDPIFLFI@?$AAs?$AAe?$AA?9?$AAn?$AAo@ 0000000180019a68     libucrt:lcidtoname_downlevel.obj
 0002:00005a78       ??_C@_1M@DANKKHJ@?$AAs?$AAe?$AA?9?$AAs?$AAe@ 0000000180019a78     libucrt:lcidtoname_downlevel.obj
 0002:00005a88       ??_C@_1M@PNBLONPJ@?$AAs?$AAk?$AA?9?$AAs?$AAk@ 0000000180019a88     libucrt:lcidtoname_downlevel.obj
 0002:00005a98       ??_C@_1M@LFMODOAL@?$AAs?$AAl?$AA?9?$AAs?$AAi@ 0000000180019a98     libucrt:lcidtoname_downlevel.obj
 0002:00005aa8       ??_C@_1O@DFKOMPG@?$AAs?$AAm?$AAa?$AA?9?$AAn?$AAo@ 0000000180019aa8     libucrt:lcidtoname_downlevel.obj
 0002:00005ab8       ??_C@_1O@NDKPBNNH@?$AAs?$AAm?$AAa?$AA?9?$AAs?$AAe@ 0000000180019ab8     libucrt:lcidtoname_downlevel.obj
 0002:00005ac8       ??_C@_1O@PLLKBHAB@?$AAs?$AAm?$AAj?$AA?9?$AAn?$AAo@ 0000000180019ac8     libucrt:lcidtoname_downlevel.obj
 0002:00005ad8       ??_C@_1O@CLEPOGCA@?$AAs?$AAm?$AAj?$AA?9?$AAs?$AAe@ 0000000180019ad8     libucrt:lcidtoname_downlevel.obj
 0002:00005ae8       ??_C@_1O@DLGJGKMK@?$AAs?$AAm?$AAn?$AA?9?$AAf?$AAi@ 0000000180019ae8     libucrt:lcidtoname_downlevel.obj
 0002:00005af8       ??_C@_1O@OJDJGAJC@?$AAs?$AAm?$AAs?$AA?9?$AAf?$AAi@ 0000000180019af8     libucrt:lcidtoname_downlevel.obj
 0002:00005b08       ??_C@_1M@BOFOGHPB@?$AAs?$AAq?$AA?9?$AAa?$AAl@ 0000000180019b08     libucrt:lcidtoname_downlevel.obj
 0002:00005b18       ??_C@_1BG@LJBBIPGB@?$AAs?$AAr?$AA?9?$AAb?$AAa?$AA?9?$AAc?$AAy?$AAr?$AAl@ 0000000180019b18     libucrt:lcidtoname_downlevel.obj
 0002:00005b30       ??_C@_1BG@JLBENFOE@?$AAs?$AAr?$AA?9?$AAb?$AAa?$AA?9?$AAl?$AAa?$AAt?$AAn@ 0000000180019b30     libucrt:lcidtoname_downlevel.obj
 0002:00005b48       ??_C@_1BG@KODPNHE@?$AAs?$AAr?$AA?9?$AAs?$AAp?$AA?9?$AAc?$AAy?$AAr?$AAl@ 0000000180019b48     libucrt:lcidtoname_downlevel.obj
 0002:00005b60       ??_C@_1BG@CIOGKHPB@?$AAs?$AAr?$AA?9?$AAs?$AAp?$AA?9?$AAl?$AAa?$AAt?$AAn@ 0000000180019b60     libucrt:lcidtoname_downlevel.obj
 0002:00005b78       ??_C@_1M@NGFJLMAC@?$AAs?$AAv?$AA?9?$AAf?$AAi@ 0000000180019b78     libucrt:lcidtoname_downlevel.obj
 0002:00005b88       ??_C@_1M@MPJEJAJC@?$AAs?$AAv?$AA?9?$AAs?$AAe@ 0000000180019b88     libucrt:lcidtoname_downlevel.obj
 0002:00005b98       ??_C@_1M@MPNDHLFK@?$AAs?$AAw?$AA?9?$AAk?$AAe@ 0000000180019b98     libucrt:lcidtoname_downlevel.obj
 0002:00005ba8       ??_C@_1O@KOHBJJI@?$AAs?$AAy?$AAr?$AA?9?$AAs?$AAy@ 0000000180019ba8     libucrt:lcidtoname_downlevel.obj
 0002:00005bb8       ??_C@_1M@LDCEFHA@?$AAt?$AAa?$AA?9?$AAi?$AAn@ 0000000180019bb8     libucrt:lcidtoname_downlevel.obj
 0002:00005bc8       ??_C@_1M@CNJOFAK@?$AAt?$AAe?$AA?9?$AAi?$AAn@ 0000000180019bc8     libucrt:lcidtoname_downlevel.obj
 0002:00005bd8       ??_C@_1M@GNAECACD@?$AAt?$AAh?$AA?9?$AAt?$AAh@ 0000000180019bd8     libucrt:lcidtoname_downlevel.obj
 0002:00005be8       ??_C@_1M@CHBIHOJO@?$AAt?$AAn?$AA?9?$AAz?$AAa@ 0000000180019be8     libucrt:lcidtoname_downlevel.obj
 0002:00005bf8       ??_C@_1M@GCCMIGPJ@?$AAt?$AAr?$AA?9?$AAt?$AAr@ 0000000180019bf8     libucrt:lcidtoname_downlevel.obj
 0002:00005c08       ??_C@_1M@CELMCNBK@?$AAt?$AAt?$AA?9?$AAr?$AAu@ 0000000180019c08     libucrt:lcidtoname_downlevel.obj
 0002:00005c18       ??_C@_1M@KLMCELGA@?$AAu?$AAk?$AA?9?$AAu?$AAa@ 0000000180019c18     libucrt:lcidtoname_downlevel.obj
 0002:00005c28       ??_C@_1M@EPAJJAJF@?$AAu?$AAr?$AA?9?$AAp?$AAk@ 0000000180019c28     libucrt:lcidtoname_downlevel.obj
 0002:00005c38       ??_C@_1BG@GEGPMCDJ@?$AAu?$AAz?$AA?9?$AAu?$AAz?$AA?9?$AAc?$AAy?$AAr?$AAl@ 0000000180019c38     libucrt:lcidtoname_downlevel.obj
 0002:00005c50       ??_C@_1BG@EGGKJILM@?$AAu?$AAz?$AA?9?$AAu?$AAz?$AA?9?$AAl?$AAa?$AAt?$AAn@ 0000000180019c50     libucrt:lcidtoname_downlevel.obj
 0002:00005c68       ??_C@_1M@GFOCLFF@?$AAv?$AAi?$AA?9?$AAv?$AAn@ 0000000180019c68     libucrt:lcidtoname_downlevel.obj
 0002:00005c78       ??_C@_1M@CPAMEDFI@?$AAx?$AAh?$AA?9?$AAz?$AAa@ 0000000180019c78     libucrt:lcidtoname_downlevel.obj
 0002:00005c88       ??_C@_1O@EBKIFIGN@?$AAz?$AAh?$AA?9?$AAc?$AAh?$AAs@ 0000000180019c88     libucrt:lcidtoname_downlevel.obj
 0002:00005c98       ??_C@_1O@NMHPGANE@?$AAz?$AAh?$AA?9?$AAc?$AAh?$AAt@ 0000000180019c98     libucrt:lcidtoname_downlevel.obj
 0002:00005ca8       ??_C@_1M@LPINJOMC@?$AAz?$AAh?$AA?9?$AAc?$AAn@ 0000000180019ca8     libucrt:lcidtoname_downlevel.obj
 0002:00005cb8       ??_C@_1M@OCJEJODD@?$AAz?$AAh?$AA?9?$AAh?$AAk@ 0000000180019cb8     libucrt:lcidtoname_downlevel.obj
 0002:00005cc8       ??_C@_1M@DNDLJINH@?$AAz?$AAh?$AA?9?$AAm?$AAo@ 0000000180019cc8     libucrt:lcidtoname_downlevel.obj
 0002:00005cd8       ??_C@_1M@MBFDNDND@?$AAz?$AAh?$AA?9?$AAs?$AAg@ 0000000180019cd8     libucrt:lcidtoname_downlevel.obj
 0002:00005ce8       ??_C@_1M@IMEPLEPE@?$AAz?$AAh?$AA?9?$AAt?$AAw@ 0000000180019ce8     libucrt:lcidtoname_downlevel.obj
 0002:00005cf8       ??_C@_1M@BBGHNHJP@?$AAz?$AAu?$AA?9?$AAz?$AAa@ 0000000180019cf8     libucrt:lcidtoname_downlevel.obj
 0002:00005d08       ??_C@_1BA@BALFACEM@?$AAC?$AAO?$AAN?$AAO?$AAU?$AAT?$AA$@ 0000000180019d08     libucrt:initcon.obj
 0002:00005d18       ??_C@_15EFLNJKHH@?$AA?$CF?$AAu@ 0000000180019d18     FARCmds.obj
 0002:00005d20       ??_C@_11LOCGONAA@@         0000000180019d20     FARCmds.obj
 0002:00005d28       ??_C@_1BM@IEHCKIMD@?$AAS?$AAh?$AAo?$AAw?$AAC?$AAm?$AAd?$AAO?$AAu?$AAt?$AAp?$AAu?$AAt@ 0000000180019d28     FARCmds.obj
 0002:00005d48       ??_C@_1BE@EKEFMMPP@?$AAC?$AAa?$AAt?$AAc?$AAh?$AAM?$AAo?$AAd?$AAe@ 0000000180019d48     FARCmds.obj
 0002:00005d60       ??_C@_1BM@BMDAMABJ@?$AAV?$AAi?$AAe?$AAw?$AAZ?$AAe?$AAr?$AAo?$AAF?$AAi?$AAl?$AAe?$AAs@ 0000000180019d60     FARCmds.obj
 0002:00005d80       ??_C@_1BK@LOJIPNKK@?$AAE?$AAd?$AAi?$AAt?$AAN?$AAe?$AAw?$AAF?$AAi?$AAl?$AAe?$AAs@ 0000000180019d80     FARCmds.obj
 0002:00005da0       ??_C@_1BI@BKNCFIOG@?$AAM?$AAa?$AAx?$AAD?$AAa?$AAt?$AAa?$AAS?$AAi?$AAz?$AAe@ 0000000180019da0     FARCmds.obj
 0002:00005db8       ??_C@_1BE@KBOCGMKN@?$AAS?$AAe?$AAp?$AAa?$AAr?$AAa?$AAt?$AAo?$AAr@ 0000000180019db8     FARCmds.obj
 0002:00005dd0       ??_C@_1BA@LGNBLCFH@?$AAF?$AAA?$AAR?$AAC?$AAm?$AAd?$AAs@ 0000000180019dd0     FARCmds.obj
 0002:00005de0       ??_C@_1EI@IHKPBHMH@?$AAF?$AAA?$AAR?$AA?5?$AAC?$AAo?$AAm?$AAm?$AAa?$AAn?$AAd?$AAs?$AA?5?$AAP?$AAl@ 0000000180019de0     FARCmds.obj
 0002:00005e28       ??_C@_1DE@BGKMIKPD@?$AAE?$AAu?$AAg?$AAe?$AAn?$AAe?$AA?5?$AAR?$AAo?$AAs?$AAh?$AAa?$AAl?$AA?5?$AA?$CG@ 0000000180019e28     FARCmds.obj
 0002:00005e5c       ??_C@_13HOIJIPNN@?$AA?5@   0000000180019e5c     FARCmds.obj
 0002:00005e60       ??_C@_1GC@PBJAIBOO@?$AAv?$AAi?$AAe?$AAw?$AA?3?$AAe?$AAd?$AAi?$AAt?$AA?3?$AAg?$AAo?$AAt?$AAo?$AA?3@ 0000000180019e60     FARCmds.obj
 0002:00005ec8       ??_C@_1O@BJPKKLLM@?$AAC?$AAo?$AAn?$AAf?$AAi?$AAg@ 0000000180019ec8     FARCmds.obj
 0002:00005ed8       MainGuid                   0000000180019ed8     FARCmds.obj
 0002:00005ef0       ??_7PluginCheckBoxBinding@@6B@ 0000000180019ef0     FARCmds.obj
 0002:00005f08       ??_7PluginUIntEditFieldBinding@@6B@ 0000000180019f08     FARCmds.obj
 0002:00005f18       DialogGuid                 0000000180019f18     FARCmds.obj
 0002:00005f30       ??_7PluginRadioButtonBinding@@6B@ 0000000180019f30     FARCmds.obj
 0002:00005f40       ConfigMenuGuid             0000000180019f40     FARCmds.obj
 0002:00005f50       ??_C@_1BE@EKCMLKPN@?$AA?$CF?$AAC?$AAO?$AAM?$AAS?$AAP?$AAE?$AAC?$AA?$CF@ 0000000180019f50     Mix.obj
 0002:00005f64       ??_C@_15BNIPFGCG@?$AA$?$AA?$CK@ 0000000180019f64     Mix.obj
 0002:00005f70       ??_C@_0BC@KFCLBIA@?$AB?$BE?$AC?$AA?$AA?$AA?$AA?$AA?$MA?$AA?$AA?$AA?$AA?$AA?$AAF?$JL@ 0000000180019f70     Mix.obj
 0002:00005f88       ??_C@_19BKJMDJK@?$AA?2?$AA?2?$AA?4?$AA?2@ 0000000180019f88     OpenCmd.obj
 0002:00005f98       ??_C@_1CE@JKDBMIKG@?$AA?2?$AA?2?$AA?4?$AA?2?$AAP?$AAh?$AAy?$AAs?$AAi?$AAc?$AAa?$AAl?$AAD?$AAr?$AAi@ 0000000180019f98     OpenCmd.obj
 0002:00005fc0       ??_C@_1BE@BNONMOPA@?$AA?2?$AA?2?$AA?4?$AA?2?$AAc?$AAd?$AAr?$AAo?$AAm@ 0000000180019fc0     OpenCmd.obj
 0002:00005fd4       ??_C@_13FPGAJAPJ@?$AA?2@   0000000180019fd4     OpenCmd.obj
 0002:00005fd8       ??_C@_1BA@EIPEFBMB@?$AA?$CF?$AAl?$AAu?$AA?1?$AA?$CF?$AAl?$AAu@ 0000000180019fd8     OpenCmd.obj
 0002:00005fe8       ??_C@_17IJMNDCL@?$AA?$CF?$AAl?$AAu@ 0000000180019fe8     OpenCmd.obj
 0002:00005ff0       ??_C@_1BM@MDBPDFDA@?$AA?$CF?$AAC?$AAO?$AAM?$AAS?$AAP?$AAE?$AAC?$AA?$CF?$AA?5?$AA?1?$AAc?$AA?5@ 0000000180019ff0     OpenCmd.obj
 0002:0000600c       ??_C@_13NEIAEHFG@?$AA?$CC@ 000000018001a00c     OpenCmd.obj
 0002:00006010       ??_C@_1BA@IBNPAI@?$AAF?$AAA?$AAR?$AAH?$AAO?$AAM?$AAE@ 000000018001a010     OpenCmd.obj
 0002:00006020       ??_C@_19IJOJOJIB@?$AAP?$AAA?$AAT?$AAH@ 000000018001a020     OpenCmd.obj
 0002:00006030       ??_C@_1BA@HAHEJCII@?$AAP?$AAA?$AAT?$AAH?$AAE?$AAX?$AAT@ 000000018001a030     OpenCmd.obj
 0002:00006040       ??_C@_13PJJBFPED@?$AA?$DL@ 000000018001a040     OpenCmd.obj
 0002:00006050       ??_C@_1GK@PPEHOOAL@?$AAS?$AAO?$AAF?$AAT?$AAW?$AAA?$AAR?$AAE?$AA?2?$AAM?$AAi?$AAc?$AAr?$AAo?$AAs@ 000000018001a050     OpenCmd.obj
 0002:000060c0       ??_C@_19JMGCACDF@?$AA?1?$AAM?$AAS?$AAG@ 000000018001a0c0     OpenCmd.obj
 0002:000060cc       ??_C@_15MDAMMGLB@?$AA?1?$AAN@ 000000018001a0cc     OpenCmd.obj
 0002:000060d4       ??_C@_15GBHPEJPD@?$AA?1?$AAS@ 000000018001a0d4     OpenCmd.obj
 0002:000060e0       ??_C@_17KKFGGCGH@?$AAR?$AAU?$AAN@ 000000018001a0e0     OpenCmd.obj
 0002:000060e8       ??_C@_17NMIMIGP@?$AAR?$AAu?$AAn@ 000000018001a0e8     OpenCmd.obj
 0002:000060f0       ??_C@_19JHOCBEIE@?$AAV?$AAI?$AAE?$AAW@ 000000018001a0f0     OpenCmd.obj
 0002:00006100       ??_C@_19MJAKNMNK@?$AAV?$AAi?$AAe?$AAw@ 000000018001a100     OpenCmd.obj
 0002:00006110       ??_C@_19PEJAKIIO@?$AAC?$AAL?$AAI?$AAP@ 000000018001a110     OpenCmd.obj
 0002:00006120       ??_C@_19KKHIGANA@?$AAC?$AAl?$AAi?$AAp@ 000000018001a120     OpenCmd.obj
 0002:00006130       ??_C@_1BA@NBLHMMII@?$AAW?$AAH?$AAE?$AAR?$AAE?$AAI?$AAS@ 000000018001a130     OpenCmd.obj
 0002:00006140       ??_C@_1BA@BCPLKBBA@?$AAW?$AAh?$AAe?$AAr?$AAe?$AAI?$AAs@ 000000018001a140     OpenCmd.obj
 0002:00006150       ??_C@_19KFAJFECL@?$AAE?$AAD?$AAI?$AAT@ 000000018001a150     OpenCmd.obj
 0002:00006160       ??_C@_19PLOBJMHF@?$AAE?$AAd?$AAi?$AAt@ 000000018001a160     OpenCmd.obj
 0002:00006170       ??_C@_19MEMGFJJL@?$AAG?$AAO?$AAT?$AAO@ 000000018001a170     OpenCmd.obj
 0002:00006180       ??_C@_19JKCOJBMF@?$AAG?$AAo?$AAt?$AAo@ 000000018001a180     OpenCmd.obj
 0002:00006190       ??_C@_19NHGGBNEB@?$AAL?$AAI?$AAN?$AAK@ 000000018001a190     OpenCmd.obj
 0002:000061a0       ??_C@_19IJIONFBP@?$AAL?$AAi?$AAn?$AAk@ 000000018001a1a0     OpenCmd.obj
 0002:000061b0       ??_C@_19LIDMLGEF@?$AAL?$AAO?$AAA?$AAD@ 000000018001a1b0     OpenCmd.obj
 0002:000061c0       ??_C@_19OGNEHOBL@?$AAL?$AAo?$AAa?$AAd@ 000000018001a1c0     OpenCmd.obj
 0002:000061d0       ??_C@_1O@PAPHGGOK@?$AAU?$AAN?$AAL?$AAO?$AAA?$AAD@ 000000018001a1d0     OpenCmd.obj
 0002:000061e0       ??_C@_1O@PJHDHGJM@?$AAU?$AAn?$AAl?$AAo?$AAa?$AAd@ 000000018001a1e0     OpenCmd.obj
 0002:000061f0       ??_C@_1BC@ENICKDH@?$AAC?$AAo?$AAn?$AAt?$AAe?$AAn?$AAt?$AAs@ 000000018001a1f0     OpenCmd.obj
 0002:000062f0       _load_config_used          000000018001a2f0     LIBCMT:loadcfg.obj
 0002:00006480       ??_R4type_info@@6B@        000000018001a480     LIBCMT:std_type_info_static.obj
 0002:000064a8       ??_R3type_info@@8          000000018001a4a8     LIBCMT:std_type_info_static.obj
 0002:000064c0       ??_R2type_info@@8          000000018001a4c0     LIBCMT:std_type_info_static.obj
 0002:000064d0       ??_R1A@?0A@EA@type_info@@8 000000018001a4d0     LIBCMT:std_type_info_static.obj
 0002:000064f8       ??_R4exception@std@@6B@    000000018001a4f8     LIBCMT:throw_bad_alloc.obj
 0002:00006520       ??_R3exception@std@@8      000000018001a520     LIBCMT:throw_bad_alloc.obj
 0002:00006538       ??_R2exception@std@@8      000000018001a538     LIBCMT:throw_bad_alloc.obj
 0002:00006548       ??_R1A@?0A@EA@exception@std@@8 000000018001a548     LIBCMT:throw_bad_alloc.obj
 0002:00006570       ??_R4bad_alloc@std@@6B@    000000018001a570     LIBCMT:throw_bad_alloc.obj
 0002:00006598       ??_R3bad_alloc@std@@8      000000018001a598     LIBCMT:throw_bad_alloc.obj
 0002:000065b0       ??_R2bad_alloc@std@@8      000000018001a5b0     LIBCMT:throw_bad_alloc.obj
 0002:000065c8       ??_R1A@?0A@EA@bad_alloc@std@@8 000000018001a5c8     LIBCMT:throw_bad_alloc.obj
 0002:000065f0       ??_R4bad_array_new_length@std@@6B@ 000000018001a5f0     LIBCMT:throw_bad_alloc.obj
 0002:00006618       ??_R3bad_array_new_length@std@@8 000000018001a618     LIBCMT:throw_bad_alloc.obj
 0002:00006630       ??_R2bad_array_new_length@std@@8 000000018001a630     LIBCMT:throw_bad_alloc.obj
 0002:00006650       ??_R1A@?0A@EA@bad_array_new_length@std@@8 000000018001a650     LIBCMT:throw_bad_alloc.obj
 0002:00006678       ??_R4bad_exception@std@@6B@ 000000018001a678     libvcruntime:frame.obj
 0002:000066a0       ??_R3bad_exception@std@@8  000000018001a6a0     libvcruntime:frame.obj
 0002:000066b8       ??_R2bad_exception@std@@8  000000018001a6b8     libvcruntime:frame.obj
 0002:000066d0       ??_R1A@?0A@EA@bad_exception@std@@8 000000018001a6d0     libvcruntime:frame.obj
 0002:000066f8       ??_R3DialogAPIBinding@@8   000000018001a6f8     FARCmds.obj
 0002:00006710       ??_R1A@?0A@EA@PluginCheckBoxBinding@@8 000000018001a710     FARCmds.obj
 0002:00006738       ??_R2PluginRadioButtonBinding@@8 000000018001a738     FARCmds.obj
 0002:00006750       ??_R3PluginRadioButtonBinding@@8 000000018001a750     FARCmds.obj
 0002:00006768       ??_R4PluginUIntEditFieldBinding@@6B@ 000000018001a768     FARCmds.obj
 0002:00006790       ??_R4PluginRadioButtonBinding@@6B@ 000000018001a790     FARCmds.obj
 0002:000067b8       ??_R3PluginCheckBoxBinding@@8 000000018001a7b8     FARCmds.obj
 0002:000067d0       ??_R1A@?0A@EA@PluginUIntEditFieldBinding@@8 000000018001a7d0     FARCmds.obj
 0002:000067f8       ??_R2DialogAPIBinding@@8   000000018001a7f8     FARCmds.obj
 0002:00006808       ??_R4PluginCheckBoxBinding@@6B@ 000000018001a808     FARCmds.obj
 0002:00006830       ??_R1A@?0A@EA@PluginRadioButtonBinding@@8 000000018001a830     FARCmds.obj
 0002:00006858       ??_R3PluginUIntEditFieldBinding@@8 000000018001a858     FARCmds.obj
 0002:00006870       ??_R2PluginCheckBoxBinding@@8 000000018001a870     FARCmds.obj
 0002:00006888       ??_R2PluginUIntEditFieldBinding@@8 000000018001a888     FARCmds.obj
 0002:000068a0       ??_R1A@?0A@EA@DialogAPIBinding@@8 000000018001a8a0     FARCmds.obj
 0002:00006bc0       __rtc_iaa                  000000018001abc0     LIBCMT:initsect.obj
 0002:00006bc8       __rtc_izz                  000000018001abc8     LIBCMT:initsect.obj
 0002:00006bd0       __rtc_taa                  000000018001abd0     LIBCMT:initsect.obj
 0002:00006bd8       __rtc_tzz                  000000018001abd8     LIBCMT:initsect.obj
 0002:000078c0       _TI2?AVbad_alloc@std@@     000000018001b8c0     LIBCMT:throw_bad_alloc.obj
 0002:000078e0       _CTA2?AVbad_alloc@std@@    000000018001b8e0     LIBCMT:throw_bad_alloc.obj
 0002:000078f8       _CT??_R0?AVbad_alloc@std@@@8??0bad_alloc@std@@QEAA@AEBV01@@Z24 000000018001b8f8     LIBCMT:throw_bad_alloc.obj
 0002:00007920       _CT??_R0?AVexception@std@@@8??0exception@std@@QEAA@AEBV01@@Z24 000000018001b920     LIBCMT:throw_bad_alloc.obj
 0002:00007948       _TI3?AVbad_array_new_length@std@@ 000000018001b948     LIBCMT:throw_bad_alloc.obj
 0002:00007968       _CTA3?AVbad_array_new_length@std@@ 000000018001b968     LIBCMT:throw_bad_alloc.obj
 0002:00007988       _CT??_R0?AVbad_array_new_length@std@@@8??0bad_array_new_length@std@@QEAA@AEBV01@@Z24 000000018001b988     LIBCMT:throw_bad_alloc.obj
 0002:000079b0       _TI2?AVbad_exception@std@@ 000000018001b9b0     libvcruntime:frame.obj
 0002:000079d0       _CTA2?AVbad_exception@std@@ 000000018001b9d0     libvcruntime:frame.obj
 0002:000079e8       _CT??_R0?AVbad_exception@std@@@8??0bad_exception@std@@QEAA@AEBV01@@Z24 000000018001b9e8     libvcruntime:frame.obj
 0002:00007ab8       __IMPORT_DESCRIPTOR_KERNEL32 000000018001bab8     kernel32:KERNEL32.dll
 0002:00007acc       __IMPORT_DESCRIPTOR_ADVAPI32 000000018001bacc     advapi32:ADVAPI32.dll
 0002:00007ae0       __IMPORT_DESCRIPTOR_USER32 000000018001bae0     user32:USER32.dll
 0002:00007af4       __IMPORT_DESCRIPTOR_ole32  000000018001baf4     ole32:ole32.dll
 0002:00007b08       __IMPORT_DESCRIPTOR_RPCRT4 000000018001bb08     rpcrt4:RPCRT4.dll
 0002:00007b1c       __NULL_IMPORT_DESCRIPTOR   000000018001bb1c     kernel32:KERNEL32.dll
 0003:00000000       __security_cookie          000000018001d000     LIBCMT:gs_cookie.obj
 0003:00000008       __security_cookie_complement 000000018001d008     LIBCMT:gs_cookie.obj
 0003:00000010       __scrt_native_dllmain_reason 000000018001d010     LIBCMT:utility.obj
 0003:00000018       __abort_behavior           000000018001d018     libucrt:abort.obj
 0003:00000030       __acrt_initial_locale_data 000000018001d030     libucrt:nlsdata.obj
 0003:00000188       __acrt_initial_locale_pointers 000000018001d188     libucrt:nlsdata.obj
 0003:00000198       __acrt_wide_c_locale_string 000000018001d198     libucrt:nlsdata.obj
 0003:000001a0       __acrt_initial_multibyte_data 000000018001d1a0     libucrt:mbctype.obj
 0003:000006e0       _iob                       000000018001d6e0     libucrt:_file.obj
 0003:000007e8       __globallocalestatus       000000018001d7e8     libucrt:glstatus.obj
 0003:000007f0       __acrt_lconv_c             000000018001d7f0     libucrt:localeconv.obj
 0003:00000888       __acrt_lconv_static_decimal 000000018001d888     libucrt:localeconv.obj
 0003:0000088c       __acrt_lconv_static_W_decimal 000000018001d88c     libucrt:localeconv.obj
 0003:00000890       _lookuptrailbytes          000000018001d890     libucrt:read.obj
 0003:00000998       _fltused                   000000018001d998     LIBCMT:fltused.obj
 0003:00000ae8       ??_R0?AVbad_alloc@std@@@8  000000018001dae8     LIBCMT:throw_bad_alloc.obj
 0003:00000b10       ??_R0?AVexception@std@@@8  000000018001db10     LIBCMT:throw_bad_alloc.obj
 0003:00000b38       ??_R0?AVbad_array_new_length@std@@@8 000000018001db38     LIBCMT:throw_bad_alloc.obj
 0003:00000b68       ??_R0?AVbad_exception@std@@@8 000000018001db68     libvcruntime:frame.obj
 0003:00000b90       ??_R0?AVtype_info@@@8      000000018001db90     LIBCMT:std_type_info_static.obj
 0003:00000bb0       ??_R0?AVPluginUIntEditFieldBinding@@@8 000000018001dbb0     FARCmds.obj
 0003:00000be8       ??_R0?AVPluginRadioButtonBinding@@@8 000000018001dbe8     FARCmds.obj
 0003:00000c18       ??_R0?AVDialogAPIBinding@@@8 000000018001dc18     FARCmds.obj
 0003:00000c40       ??_R0?AVPluginCheckBoxBinding@@@8 000000018001dc40     FARCmds.obj
 0003:000010b0       ?__type_info_root_node@@3U__type_info_node@@A 000000018001e0b0     LIBCMT:tncleanup.obj
 0003:000010c0       ?_OptionsStorage@?1??__local_stdio_printf_options@@9@4_KA 000000018001e0c0     LIBCMT:default_local_stdio_options.obj
 0003:000010c8       ?_OptionsStorage@?1??__local_stdio_scanf_options@@9@4_KA 000000018001e0c8     LIBCMT:default_local_stdio_options.obj
 0003:000010d0       __scrt_current_native_startup_state 000000018001e0d0     LIBCMT:utility.obj
 0003:000010d8       __scrt_native_startup_lock 000000018001e0d8     LIBCMT:utility.obj
 0003:00001118       __castguard_check_failure_os_handled_fptr 000000018001e118     LIBCMT:guard_support.obj
 0003:00001120       ?__WinRTOutOfMemoryExceptionCallback@@3P6APEAXXZEA 000000018001e120     libvcruntime:ehhelpers.obj
 0003:000011b0       __pPurecall                000000018001e1b0     libvcruntime:purevirt_data.obj
 0003:000011e0       ?pArgList@UnDecorator@@0PEAVReplicator@@EA 000000018001e1e0     libvcruntime:undname.obj
 0003:000011e8       ?pZNameList@UnDecorator@@0PEAVReplicator@@EA 000000018001e1e8     libvcruntime:undname.obj
 0003:000011f0       ?pTemplateArgList@UnDecorator@@0PEAVReplicator@@EA 000000018001e1f0     libvcruntime:undname.obj
 0003:000011f8       ?gName@UnDecorator@@0PEBDEB 000000018001e1f8     libvcruntime:undname.obj
 0003:00001200       ?name@UnDecorator@@0PEBDEB 000000018001e200     libvcruntime:undname.obj
 0003:00001208       ?disableFlags@UnDecorator@@0KA 000000018001e208     libvcruntime:undname.obj
 0003:0000120c       ?fExplicitTemplateParams@UnDecorator@@0_NA 000000018001e20c     libvcruntime:undname.obj
 0003:0000120d       ?fGetTemplateArgumentList@UnDecorator@@0_NA 000000018001e20d     libvcruntime:undname.obj
 0003:00001210       ?m_pGetParameter@UnDecorator@@0P6APEADJ@ZEA 000000018001e210     libvcruntime:undname.obj
 0003:00001218       ?m_CHPENameOffset@UnDecorator@@0KA 000000018001e218     libvcruntime:undname.obj
 0003:0000121c       ?m_recursionLevel@UnDecorator@@0KA 000000018001e21c     libvcruntime:undname.obj
 0003:00001268       ?c_exit_complete@?1???R<lambda_6e4b09c48022b2350581041d5f6b0c4c>@@QEBA@XZ@4_NA 000000018001e268     libucrt:exit.obj
 0003:00001378       _environ_table             000000018001e378     libucrt:environment_initialization.obj
 0003:00001380       _wenviron_table            000000018001e380     libucrt:environment_initialization.obj
 0003:00001388       __dcrt_initial_wide_environment 000000018001e388     libucrt:environment_initialization.obj
 0003:00001390       __dcrt_initial_narrow_environment 000000018001e390     libucrt:environment_initialization.obj
 0003:00001398       __acrt_atexit_table        000000018001e398     libucrt:onexit.obj
 0003:000013b0       __acrt_at_quick_exit_table 000000018001e3b0     libucrt:onexit.obj
 0003:000013d0       __acrt_locale_changed_data 000000018001e3d0     libucrt:wsetlocale.obj
 0003:000013d8       __acrt_current_locale_data 000000018001e3d8     libucrt:nlsdata.obj
 0003:00001618       _mbctype                   000000018001e618     libucrt:mbctype.obj
 0003:00001620       _mbcasemap                 000000018001e620     libucrt:mbctype.obj
 0003:00001628       __acrt_current_multibyte_data 000000018001e628     libucrt:mbctype.obj
 0003:00001638       _pgmptr                    000000018001e638     libucrt:argv_data.obj
 0003:00001640       __argc                     000000018001e640     libucrt:argv_data.obj
 0003:00001648       __argv                     000000018001e648     libucrt:argv_data.obj
 0003:00001650       __wargv                    000000018001e650     libucrt:argv_data.obj
 0003:00001658       _acmdln                    000000018001e658     libucrt:argv_data.obj
 0003:00001660       _wcmdln                    000000018001e660     libucrt:argv_data.obj
 0003:00001820       __acrt_heap                000000018001e820     libucrt:heap_handle.obj
 0003:00001830       __pioinfo                  000000018001e830     libucrt:ioinit.obj
 0003:00001c30       _nhandle                   000000018001ec30     libucrt:ioinit.obj
 0003:00001c60       _nstream                   000000018001ec60     libucrt:_file.obj
 0003:00001c68       __piob                     000000018001ec68     libucrt:_file.obj
 0003:00001c70       __acrt_stdout_buffer       000000018001ec70     libucrt:_sftbuf.obj
 0003:00001c78       __acrt_stderr_buffer       000000018001ec78     libucrt:_sftbuf.obj
 0003:00001c8c       __acrt_lconv_static_null   000000018001ec8c     libucrt:localeconv.obj
 0003:00001c90       __acrt_lconv_static_W_null 000000018001ec90     libucrt:localeconv.obj
 0003:00001ca0       ?Opt@@3UOptions@@A         000000018001eca0     FARCmds.obj
 0003:00001cc0       ?PsInfo@@3UPluginStartupInfo@@A 000000018001ecc0     FARCmds.obj
 0003:00001de0       ?FSF@@3UFarStandardFunctions@@A 000000018001ede0     FARCmds.obj
 0003:00005d68       __scrt_ucrt_dll_is_in_use  0000000180022d68     <common>
 0003:00005d70       __dyn_tls_init_callback    0000000180022d70     <common>

 entry point at        0001:00006618

 Static symbols

 0000:fffda000       .debug$S                   0000000180000000     FarCmds.exp
 0000:fffda000       .debug$S                   0000000180000000     advapi32:ADVAPI32.dll
 0000:fffda000       .debug$S                   0000000180000000     advapi32:ADVAPI32.dll
 0000:fffda000       .debug$S                   0000000180000000     advapi32:ADVAPI32.dll
 0000:fffda000       .debug$S                   0000000180000000     advapi32:ADVAPI32.dll
 0000:fffda000       .debug$S                   0000000180000000     kernel32:KERNEL32.dll
 0000:fffda000       .debug$S                   0000000180000000     kernel32:KERNEL32.dll
 0000:fffda000       .debug$S                   0000000180000000     kernel32:KERNEL32.dll
 0000:fffda000       .debug$S                   0000000180000000     kernel32:KERNEL32.dll
 0000:fffda000       .debug$S                   0000000180000000     kernel32:KERNEL32.dll
 0000:fffda000       .debug$S                   0000000180000000     kernel32:KERNEL32.dll
 0000:fffda000       .debug$S                   0000000180000000     kernel32:KERNEL32.dll
 0000:fffda000       .debug$S                   0000000180000000     kernel32:KERNEL32.dll
 0000:fffda000       .debug$S                   0000000180000000     kernel32:KERNEL32.dll
 0000:fffda000       .debug$S                   0000000180000000     kernel32:KERNEL32.dll
 0000:fffda000       .debug$S                   0000000180000000     kernel32:KERNEL32.dll
 0000:fffda000       .debug$S                   0000000180000000     kernel32:KERNEL32.dll
 0000:fffda000       .debug$S                   0000000180000000     kernel32:KERNEL32.dll
 0000:fffda000       .debug$S                   0000000180000000     kernel32:KERNEL32.dll
 0000:fffda000       .debug$S                   0000000180000000     kernel32:KERNEL32.dll
 0000:fffda000       .debug$S                   0000000180000000     kernel32:KERNEL32.dll
 0000:fffda000       .debug$S                   0000000180000000     kernel32:KERNEL32.dll
 0000:fffda000       .debug$S                   0000000180000000     kernel32:KERNEL32.dll
 0000:fffda000       .debug$S                   0000000180000000     kernel32:KERNEL32.dll
 0000:fffda000       .debug$S                   0000000180000000     kernel32:KERNEL32.dll
 0000:fffda000       .debug$S                   0000000180000000     kernel32:KERNEL32.dll
 0000:fffda000       .debug$S                   0000000180000000     kernel32:KERNEL32.dll
 0000:fffda000       .debug$S                   0000000180000000     kernel32:KERNEL32.dll
 0000:fffda000       .debug$S                   0000000180000000     kernel32:KERNEL32.dll
 0000:fffda000       .debug$S                   0000000180000000     kernel32:KERNEL32.dll
 0000:fffda000       .debug$S                   0000000180000000     kernel32:KERNEL32.dll
 0000:fffda000       .debug$S                   0000000180000000     kernel32:KERNEL32.dll
 0000:fffda000       .debug$S                   0000000180000000     kernel32:KERNEL32.dll
 0000:fffda000       .debug$S                   0000000180000000     kernel32:KERNEL32.dll
 0000:fffda000       .debug$S                   0000000180000000     kernel32:KERNEL32.dll
 0000:fffda000       .debug$S                   0000000180000000     kernel32:KERNEL32.dll
 0000:fffda000       .debug$S                   0000000180000000     kernel32:KERNEL32.dll
 0000:fffda000       .debug$S                   0000000180000000     kernel32:KERNEL32.dll
 0000:fffda000       .debug$S                   0000000180000000     kernel32:KERNEL32.dll
 0000:fffda000       .debug$S                   0000000180000000     kernel32:KERNEL32.dll
 0000:fffda000       .debug$S                   0000000180000000     kernel32:KERNEL32.dll
 0000:fffda000       .debug$S                   0000000180000000     kernel32:KERNEL32.dll
 0000:fffda000       .debug$S                   0000000180000000     kernel32:KERNEL32.dll
 0000:fffda000       .debug$S                   0000000180000000     kernel32:KERNEL32.dll
 0000:fffda000       .debug$S                   0000000180000000     kernel32:KERNEL32.dll
 0000:fffda000       .debug$S                   0000000180000000     kernel32:KERNEL32.dll
 0000:fffda000       .debug$S                   0000000180000000     kernel32:KERNEL32.dll
 0000:fffda000       .debug$S                   0000000180000000     kernel32:KERNEL32.dll
 0000:fffda000       .debug$S                   0000000180000000     kernel32:KERNEL32.dll
 0000:fffda000       .debug$S                   0000000180000000     kernel32:KERNEL32.dll
 0000:fffda000       .debug$S                   0000000180000000     kernel32:KERNEL32.dll
 0000:fffda000       .debug$S                   0000000180000000     kernel32:KERNEL32.dll
 0000:fffda000       .debug$S                   0000000180000000     kernel32:KERNEL32.dll
 0000:fffda000       .debug$S                   0000000180000000     kernel32:KERNEL32.dll
 0000:fffda000       .debug$S                   0000000180000000     kernel32:KERNEL32.dll
 0000:fffda000       .debug$S                   0000000180000000     kernel32:KERNEL32.dll
 0000:fffda000       .debug$S                   0000000180000000     kernel32:KERNEL32.dll
 0000:fffda000       .debug$S                   0000000180000000     kernel32:KERNEL32.dll
 0000:fffda000       .debug$S                   0000000180000000     kernel32:KERNEL32.dll
 0000:fffda000       .debug$S                   0000000180000000     kernel32:KERNEL32.dll
 0000:fffda000       .debug$S                   0000000180000000     kernel32:KERNEL32.dll
 0000:fffda000       .debug$S                   0000000180000000     kernel32:KERNEL32.dll
 0000:fffda000       .debug$S                   0000000180000000     kernel32:KERNEL32.dll
 0000:fffda000       .debug$S                   0000000180000000     kernel32:KERNEL32.dll
 0000:fffda000       .debug$S                   0000000180000000     kernel32:KERNEL32.dll
 0000:fffda000       .debug$S                   0000000180000000     kernel32:KERNEL32.dll
 0000:fffda000       .debug$S                   0000000180000000     kernel32:KERNEL32.dll
 0000:fffda000       .debug$S                   0000000180000000     kernel32:KERNEL32.dll
 0000:fffda000       .debug$S                   0000000180000000     kernel32:KERNEL32.dll
 0000:fffda000       .debug$S                   0000000180000000     kernel32:KERNEL32.dll
 0000:fffda000       .debug$S                   0000000180000000     kernel32:KERNEL32.dll
 0000:fffda000       .debug$S                   0000000180000000     kernel32:KERNEL32.dll
 0000:fffda000       .debug$S                   0000000180000000     kernel32:KERNEL32.dll
 0000:fffda000       .debug$S                   0000000180000000     kernel32:KERNEL32.dll
 0000:fffda000       .debug$S                   0000000180000000     kernel32:KERNEL32.dll
 0000:fffda000       .debug$S                   0000000180000000     kernel32:KERNEL32.dll
 0000:fffda000       .debug$S                   0000000180000000     kernel32:KERNEL32.dll
 0000:fffda000       .debug$S                   0000000180000000     kernel32:KERNEL32.dll
 0000:fffda000       .debug$S                   0000000180000000     kernel32:KERNEL32.dll
 0000:fffda000       .debug$S                   0000000180000000     kernel32:KERNEL32.dll
 0000:fffda000       .debug$S                   0000000180000000     kernel32:KERNEL32.dll
 0000:fffda000       .debug$S                   0000000180000000     kernel32:KERNEL32.dll
 0000:fffda000       .debug$S                   0000000180000000     kernel32:KERNEL32.dll
 0000:fffda000       .debug$S                   0000000180000000     kernel32:KERNEL32.dll
 0000:fffda000       .debug$S                   0000000180000000     kernel32:KERNEL32.dll
 0000:fffda000       .debug$S                   0000000180000000     kernel32:KERNEL32.dll
 0000:fffda000       .debug$S                   0000000180000000     kernel32:KERNEL32.dll
 0000:fffda000       .debug$S                   0000000180000000     kernel32:KERNEL32.dll
 0000:fffda000       .debug$S                   0000000180000000     kernel32:KERNEL32.dll
 0000:fffda000       .debug$S                   0000000180000000     kernel32:KERNEL32.dll
 0000:fffda000       .debug$S                   0000000180000000     kernel32:KERNEL32.dll
 0000:fffda000       .debug$S                   0000000180000000     kernel32:KERNEL32.dll
 0000:fffda000       .debug$S                   0000000180000000     kernel32:KERNEL32.dll
 0000:fffda000       .debug$S                   0000000180000000     kernel32:KERNEL32.dll
 0000:fffda000       .debug$S                   0000000180000000     kernel32:KERNEL32.dll
 0000:fffda000       .debug$S                   0000000180000000     kernel32:KERNEL32.dll
 0000:fffda000       .debug$S                   0000000180000000     kernel32:KERNEL32.dll
 0000:fffda000       .debug$S                   0000000180000000     kernel32:KERNEL32.dll
 0000:fffda000       .debug$S                   0000000180000000     kernel32:KERNEL32.dll
 0000:fffda000       .debug$S                   0000000180000000     kernel32:KERNEL32.dll
 0000:fffda000       .debug$S                   0000000180000000     kernel32:KERNEL32.dll
 0000:fffda000       .debug$S                   0000000180000000     kernel32:KERNEL32.dll
 0000:fffda000       .debug$S                   0000000180000000     kernel32:KERNEL32.dll
 0000:fffda000       .debug$S                   0000000180000000     kernel32:KERNEL32.dll
 0000:fffda000       .debug$S                   0000000180000000     kernel32:KERNEL32.dll
 0000:fffda000       .debug$S                   0000000180000000     kernel32:KERNEL32.dll
 0000:fffda000       .debug$S                   0000000180000000     kernel32:KERNEL32.dll
 0000:fffda000       .debug$S                   0000000180000000     kernel32:KERNEL32.dll
 0000:fffda000       .debug$S                   0000000180000000     kernel32:KERNEL32.dll
 0000:fffda000       .debug$S                   0000000180000000     kernel32:KERNEL32.dll
 0000:fffda000       .debug$S                   0000000180000000     kernel32:KERNEL32.dll
 0000:fffda000       .debug$S                   0000000180000000     kernel32:KERNEL32.dll
 0000:fffda000       .debug$S                   0000000180000000     kernel32:KERNEL32.dll
 0000:fffda000       .debug$S                   0000000180000000     kernel32:KERNEL32.dll
 0000:fffda000       .debug$S                   0000000180000000     kernel32:KERNEL32.dll
 0000:fffda000       .debug$S                   0000000180000000     ole32:ole32.dll
 0000:fffda000       .debug$S                   0000000180000000     ole32:ole32.dll
 0000:fffda000       .debug$S                   0000000180000000     ole32:ole32.dll
 0000:fffda000       .debug$S                   0000000180000000     rpcrt4:RPCRT4.dll
 0000:fffda000       .debug$S                   0000000180000000     user32:USER32.dll
 0000:fffda000       .debug$S                   0000000180000000     user32:USER32.dll
 0001:00000570       Table                      0000000180001570     libvcruntime:memset.obj
 0001:00000dc0       $LN42                      0000000180001dc0     FARCmds.obj
 0001:00000dc1       $LN43                      0000000180001dc1     FARCmds.obj
 0001:00000dc2       $LN44                      0000000180001dc2     FARCmds.obj
 0001:00000dc3       $LN45                      0000000180001dc3     FARCmds.obj
 0001:00000dc4       $LN46                      0000000180001dc4     FARCmds.obj
 0001:00000dc5       $LN47                      0000000180001dc5     FARCmds.obj
 0001:00000dc6       $LN48                      0000000180001dc6     FARCmds.obj
 0001:00000dc7       $LN49                      0000000180001dc7     FARCmds.obj
 0001:00000dc8       $LN50                      0000000180001dc8     FARCmds.obj
 0001:00000dc9       $LN51                      0000000180001dc9     FARCmds.obj
 0001:00000dca       $LN52                      0000000180001dca     FARCmds.obj
 0001:00000dcb       $LN53                      0000000180001dcb     FARCmds.obj
 0001:00000f8c       $LN50                      0000000180001f8c     FARCmds.obj
 0001:00000f8d       $LN51                      0000000180001f8d     FARCmds.obj
 0001:00000f8e       $LN52                      0000000180001f8e     FARCmds.obj
 0001:00000f8f       $LN53                      0000000180001f8f     FARCmds.obj
 0001:00000f90       $LN54                      0000000180001f90     FARCmds.obj
 0001:00000f91       $LN55                      0000000180001f91     FARCmds.obj
 0001:00000f92       $LN56                      0000000180001f92     FARCmds.obj
 0001:00000f93       $LN57                      0000000180001f93     FARCmds.obj
 0001:00000f94       $LN58                      0000000180001f94     FARCmds.obj
 0001:00000f95       $LN59                      0000000180001f95     FARCmds.obj
 0001:00000f96       $LN60                      0000000180001f96     FARCmds.obj
 0001:00000f97       $LN61                      0000000180001f97     FARCmds.obj
 0001:000012b8       $LN18                      00000001800022b8     FARCmds.obj
 0001:00001470       $LN48                      0000000180002470     FARCmds.obj
 0001:00001471       $LN49                      0000000180002471     FARCmds.obj
 0001:00001472       $LN50                      0000000180002472     FARCmds.obj
 0001:00001473       $LN51                      0000000180002473     FARCmds.obj
 0001:00001474       $LN52                      0000000180002474     FARCmds.obj
 0001:00001475       $LN53                      0000000180002475     FARCmds.obj
 0001:00001476       $LN54                      0000000180002476     FARCmds.obj
 0001:00001477       $LN55                      0000000180002477     FARCmds.obj
 0001:00001478       $LN56                      0000000180002478     FARCmds.obj
 0001:00001479       $LN57                      0000000180002479     FARCmds.obj
 0001:0000147a       $LN58                      000000018000247a     FARCmds.obj
 0001:0000147b       $LN59                      000000018000247b     FARCmds.obj
 0001:00002378       $LN238                     0000000180003378     FARCmds.obj
 0001:0000237c       $LN239                     000000018000337c     FARCmds.obj
 0001:00002380       $LN240                     0000000180003380     FARCmds.obj
 0001:00002384       $LN241                     0000000180003384     FARCmds.obj
 0001:00002388       $LN242                     0000000180003388     FARCmds.obj
 0001:0000238c       $LN243                     000000018000338c     FARCmds.obj
 0001:00002390       $LN244                     0000000180003390     FARCmds.obj
 0001:00002394       $LN245                     0000000180003394     FARCmds.obj
 0001:00002398       $LN246                     0000000180003398     FARCmds.obj
 0001:0000239c       $LN247                     000000018000339c     FARCmds.obj
 0001:000023a0       $LN248                     00000001800033a0     FARCmds.obj
 0001:000023a4       $LN249                     00000001800033a4     FARCmds.obj
 0001:000023a8       $LN252                     00000001800033a8     FARCmds.obj
 0001:000023ac       $LN253                     00000001800033ac     FARCmds.obj
 0001:000023b0       $LN254                     00000001800033b0     FARCmds.obj
 0001:000023b4       $LN255                     00000001800033b4     FARCmds.obj
 0001:000023b8       $LN256                     00000001800033b8     FARCmds.obj
 0001:000023bc       $LN257                     00000001800033bc     FARCmds.obj
 0001:000023c0       $LN258                     00000001800033c0     FARCmds.obj
 0001:000023c4       $LN259                     00000001800033c4     FARCmds.obj
 0001:000023c8       $LN260                     00000001800033c8     FARCmds.obj
 0001:000023cc       $LN261                     00000001800033cc     FARCmds.obj
 0001:000023d0       $LN262                     00000001800033d0     FARCmds.obj
 0001:000023d4       $LN263                     00000001800033d4     FARCmds.obj
 0001:000023d8       $LN266                     00000001800033d8     FARCmds.obj
 0001:000023dc       $LN267                     00000001800033dc     FARCmds.obj
 0001:000023e0       $LN268                     00000001800033e0     FARCmds.obj
 0001:000023e4       $LN269                     00000001800033e4     FARCmds.obj
 0001:000023e8       $LN270                     00000001800033e8     FARCmds.obj
 0001:000023ec       $LN271                     00000001800033ec     FARCmds.obj
 0001:000023f0       $LN272                     00000001800033f0     FARCmds.obj
 0001:000023f4       $LN273                     00000001800033f4     FARCmds.obj
 0001:000023f8       $LN274                     00000001800033f8     FARCmds.obj
 0001:000023fc       $LN275                     00000001800033fc     FARCmds.obj
 0001:00002400       $LN276                     0000000180003400     FARCmds.obj
 0001:00002404       $LN277                     0000000180003404     FARCmds.obj
 0001:00002568       ?GetAlias@@YAPEA_WPEB_W0@Z 0000000180003568 f   Mix.obj
 0001:00003260       ?getCurrDir@@YAPEA_W_N@Z   0000000180004260 f   OpenCmd.obj
 0001:00003320       ?killTemp@@YAXPEA_W@Z      0000000180004320 f   OpenCmd.obj
 0001:00003388       ?createFile@@YAPEAXPEA_WH@Z 0000000180004388 f   OpenCmd.obj
 0001:00003460       ?createFileStream@@YAXPEB_WPEAXPEAUTShowOutputStreamData@@1@Z 0000000180004460 f   OpenCmd.obj
 0001:000034d0       ?validForView@@YA_NPEB_W_N1@Z 00000001800044d0 f   OpenCmd.obj
 0001:00003808       ?showPartOfOutput@@YAKPEAUTShowOutputStreamData@@_N@Z 0000000180004808 f   OpenCmd.obj
 0001:000039e8       ?ThreadWhatUpdateScreen@@YAKPEAX@Z 00000001800049e8 f   OpenCmd.obj
 0001:00003bc8       ?MakeExecuteString@@YAPEB_WPEB_W@Z 0000000180004bc8 f   OpenCmd.obj
 0001:00003fa0       ?loadFile@@YAPEA_WPEB_WKHAEA_KAEA_N@Z 0000000180004fa0 f   OpenCmd.obj
 0001:000041e8       ?__getContent@@YAPEA_WHPEA_W@Z 00000001800051e8 f   OpenCmd.obj
 0001:00004960       $LN61                      0000000180005960     OpenCmd.obj
 0001:00006184       $LN335                     0000000180007184     OpenCmd.obj
 0001:00006188       $LN336                     0000000180007188     OpenCmd.obj
 0001:0000618c       $LN337                     000000018000718c     OpenCmd.obj
 0001:00006190       $LN338                     0000000180007190     OpenCmd.obj
 0001:00006194       $LN339                     0000000180007194     OpenCmd.obj
 0001:00006198       $LN342                     0000000180007198     OpenCmd.obj
 0001:0000619c       $LN343                     000000018000719c     OpenCmd.obj
 0001:000061a0       $LN344                     00000001800071a0     OpenCmd.obj
 0001:000061a4       $LN345                     00000001800071a4     OpenCmd.obj
 0001:000061a8       $LN346                     00000001800071a8     OpenCmd.obj
 0001:000061ac       $LN347                     00000001800071ac     OpenCmd.obj
 0001:000061b0       $LN348                     00000001800071b0     OpenCmd.obj
 0001:000061b4       $LN349                     00000001800071b4     OpenCmd.obj
 0001:000061b8       $LN350                     00000001800071b8     OpenCmd.obj
 0001:00006250       ?dllmain_crt_dispatch@@YAHQEAUHINSTANCE__@@KQEAX@Z 0000000180007250 f   LIBCMT:dll_dllmain.obj
 0001:000062b0       ?dllmain_crt_process_attach@@YAHQEAUHINSTANCE__@@QEAX@Z 00000001800072b0 f   LIBCMT:dll_dllmain.obj
 0001:000063e0       ?dllmain_crt_process_detach@@YAH_N@Z 00000001800073e0 f   LIBCMT:dll_dllmain.obj
 0001:00006480       ?dllmain_dispatch@@YAHQEAUHINSTANCE__@@KQEAX@Z 0000000180007480 f   LIBCMT:dll_dllmain.obj
 0001:000065b8       ?dllmain_raw@@YAHQEAUHINSTANCE__@@KQEAX@Z 00000001800075b8 f   LIBCMT:dll_dllmain.obj
 0001:00006960       $LN9                       0000000180007960     LIBCMT:gs_support.obj
 0001:00006968       $LN10                      0000000180007968     LIBCMT:gs_support.obj
 0001:00006970       initialize_environment     0000000180007970 f   libucrt:initialization.obj
 0001:00006970       initialize_global_state_isolation 0000000180007970 f   libucrt:initialization.obj
 0001:00006970       report_memory_leaks        0000000180007970 f   libucrt:initialization.obj
 0001:00006970       uninitialize_c             0000000180007970 f   libucrt:initialization.obj
 0001:00006970       uninitialize_global_state_isolation 0000000180007970 f   libucrt:initialization.obj
 0001:00007408       $LN6                       0000000180008408     libvcruntime:risctrnsctrl.obj
 0001:00007670       $LN28                      0000000180008670     libvcruntime:ehhelpers.obj
 0001:00007674       $LN29                      0000000180008674     libvcruntime:ehhelpers.obj
 0001:00007778       $LN13                      0000000180008778     libvcruntime:ehhelpers.obj
 0001:0000777c       $LN14                      000000018000877c     libvcruntime:ehhelpers.obj
 0001:00007780       $LN15                      0000000180008780     libvcruntime:ehhelpers.obj
 0001:00007d38       $LN54                      0000000180008d38     libvcruntime:riscchandler.obj
 0001:00007ed0       $LN6                       0000000180008ed0     libvcruntime:throw.obj
 0001:00007ed8       $LN7                       0000000180008ed8     libvcruntime:throw.obj
 0001:00007ee0       $LN8                       0000000180008ee0     libvcruntime:throw.obj
 0001:000083d0       ??$BuildCatchObjectHelperInternal@V__FrameHandler3@@@@YAHPEAUEHExceptionRecord@@PEAXPEBU_s_HandlerType@@PEBU_s_CatchableType@@@Z 00000001800093d0 f   libvcruntime:frame.obj
 0001:000085b8       ??$BuildCatchObjectInternal@V__FrameHandler3@@@@YAXPEAUEHExceptionRecord@@PEAXPEBU_s_HandlerType@@PEBU_s_CatchableType@@@Z 00000001800095b8 f   libvcruntime:frame.obj
 0001:00008698       ??$CatchIt@V__FrameHandler3@@@@YAXPEAUEHExceptionRecord@@PEA_KPEAU_CONTEXT@@PEAU_xDISPATCHER_CONTEXT@@PEBU_s_FuncInfo@@PEBU_s_HandlerType@@PEBU_s_CatchableType@@PEBU_s_TryBlockMapEntry@@H1EE@Z 0000000180009698 f   libvcruntime:frame.obj
 0001:00008768       ??$FindHandler@V__FrameHandler3@@@@YAXPEAUEHExceptionRecord@@PEA_KPEAU_CONTEXT@@PEAU_xDISPATCHER_CONTEXT@@PEBU_s_FuncInfo@@EH1@Z 0000000180009768 f   libvcruntime:frame.obj
 0001:00008c98       $LN128                     0000000180009c98     libvcruntime:frame.obj
 0001:00008c9c       $LN129                     0000000180009c9c     libvcruntime:frame.obj
 0001:00008ca0       $LN130                     0000000180009ca0     libvcruntime:frame.obj
 0001:00008ca8       ??$FindHandlerForForeignException@V__FrameHandler3@@@@YAXPEAUEHExceptionRecord@@PEA_KPEAU_CONTEXT@@PEAU_xDISPATCHER_CONTEXT@@PEBU_s_FuncInfo@@HH1@Z 0000000180009ca8 f   libvcruntime:frame.obj
 0001:00008ef8       $LN54                      0000000180009ef8     libvcruntime:frame.obj
 0001:00008efc       $LN55                      0000000180009efc     libvcruntime:frame.obj
 0001:00009288       $LN51                      000000018000a288     libvcruntime:frame.obj
 0001:00009290       $LN47                      000000018000a290     libvcruntime:frame.obj
 0001:00009294       $LN48                      000000018000a294     libvcruntime:frame.obj
 0001:00009298       $LN49                      000000018000a298     libvcruntime:frame.obj
 0001:0000929c       $LN50                      000000018000a29c     libvcruntime:frame.obj
 0001:000092a0       $LN52                      000000018000a2a0     libvcruntime:frame.obj
 0001:00009520       $LN29                      000000018000a520     libvcruntime:frame.obj
 0001:00009524       $LN30                      000000018000a524     libvcruntime:frame.obj
 0001:00009528       ?ExFilterRethrow@@YAHPEAU_EXCEPTION_POINTERS@@PEAUEHExceptionRecord@@PEAH@Z 000000018000a528 f   libvcruntime:frame.obj
 0001:000095e0       $LN12                      000000018000a5e0     libvcruntime:frame.obj
 0001:000095e4       $LN13                      000000018000a5e4     libvcruntime:frame.obj
 0001:00009870       ?IsInExceptionSpec@@YAEPEAUEHExceptionRecord@@PEBU_s_ESTypeList@@@Z 000000018000a870 f   libvcruntime:frame.obj
 0001:0000a0c8       ??$?RV<lambda_d80eeec6fff315bfe5c115232f3240e3>@@AEAV<lambda_6e4b09c48022b2350581041d5f6b0c4c>@@V<lambda_2358e3775559c9db80273638284d5e45>@@@?$__crt_seh_guarded_call@X@@QEAAX$$QEAV<lambda_d80eeec6fff315bfe5c115232f3240e3>@@AEAV<lambda_6e4b09c48022b2350581041d5f6b0c4c>@@$$QEAV<lambda_2358e3775559c9db80273638284d5e45>@@@Z 000000018000b0c8 f   libucrt:exit.obj
 0001:0000a108       ??R<lambda_6e4b09c48022b2350581041d5f6b0c4c>@@QEBA@XZ 000000018000b108 f   libucrt:exit.obj
 0001:0000a218       ?atexit_exception_filter@@YAHK@Z 000000018000b218 f   libucrt:exit.obj
 0001:0000a230       ?common_exit@@YAXHW4_crt_exit_cleanup_mode@@W4_crt_exit_return_mode@@@Z 000000018000b230 f   libucrt:exit.obj
 0001:0000a308       ?exit_or_terminate_process@@YAXI@Z 000000018000b308 f   libucrt:exit.obj
 0001:0000a378       ?try_cor_exit_process@@YAXI@Z 000000018000b378 f   libucrt:exit.obj
 0001:0000a450       ??$parse_command_line@D@@YAXPEADPEAPEAD0PEA_K2@Z 000000018000b450 f   libucrt:argv_parsing.obj
 0001:0000a8a8       ??$common_initialize_environment_nolock@D@@YAHXZ 000000018000b8a8 f   libucrt:environment_initialization.obj
 0001:0000a928       ??$create_environment@D@@YAQEAPEADQEAD@Z 000000018000b928 f   libucrt:environment_initialization.obj
 0001:0000aa50       ??$uninitialize_environment_internal@D@@YAXAEAPEAPEAD@Z 000000018000ba50 f   libucrt:environment_initialization.obj
 0001:0000aaa8       ??$uninitialize_environment_internal@_W@@YAXAEAPEAPEA_W@Z 000000018000baa8 f   libucrt:environment_initialization.obj
 0001:0000ab98       ??$?RV<lambda_7777bce6b2f8c936911f934f8298dc43>@@AEAV<lambda_f03950bc5685219e0bcd2087efbe011e>@@V<lambda_3883c3dff614d5e0c5f61bb1ac94921c>@@@?$__crt_seh_guarded_call@H@@QEAAH$$QEAV<lambda_7777bce6b2f8c936911f934f8298dc43>@@AEAV<lambda_f03950bc5685219e0bcd2087efbe011e>@@$$QEAV<lambda_3883c3dff614d5e0c5f61bb1ac94921c>@@@Z 000000018000bb98 f   libucrt:onexit.obj
 0001:0000abe0       ??R<lambda_f03950bc5685219e0bcd2087efbe011e>@@QEBAHXZ 000000018000bbe0 f   libucrt:onexit.obj
 0001:0000ada0       initialize_global_variables 000000018000bda0 f   libucrt:initialization.obj
 0001:0000adb8       initialize_c               000000018000bdb8 f   libucrt:initialization.obj
 0001:0000ade8       uninitialize_environment   000000018000bde8 f   libucrt:initialization.obj
 0001:0000ae00       initialize_pointers        000000018000be00 f   libucrt:initialization.obj
 0001:0000ae50       uninitialize_vcruntime     000000018000be50 f   libucrt:initialization.obj
 0001:0000ae70       uninitialize_allocated_memory 000000018000be70 f   libucrt:initialization.obj
 0001:0000aed0       uninitialize_allocated_io_buffers 000000018000bed0 f   libucrt:initialization.obj
 0001:0000b548       ??$?RV<lambda_0ae27a3a962d80f24befdcbee591983d>@@AEAV<lambda_8d0ee55de4b1038c4002e0adecdf1839>@@V<lambda_dc504788e8f1664fe9b84e20bfb512f2>@@@?$__crt_seh_guarded_call@X@@QEAAX$$QEAV<lambda_0ae27a3a962d80f24befdcbee591983d>@@AEAV<lambda_8d0ee55de4b1038c4002e0adecdf1839>@@$$QEAV<lambda_dc504788e8f1664fe9b84e20bfb512f2>@@@Z 000000018000c548 f   libucrt:per_thread_data.obj
 0001:0000b5a0       ??$?RV<lambda_2d41944a1d46af3157314b8a01080d33>@@AEAV<lambda_8f455de75cd7d7f24b4096f044d8b9e6>@@V<lambda_aa500f224e6afead328df44964fe2772>@@@?$__crt_seh_guarded_call@X@@QEAAX$$QEAV<lambda_2d41944a1d46af3157314b8a01080d33>@@AEAV<lambda_8f455de75cd7d7f24b4096f044d8b9e6>@@$$QEAV<lambda_aa500f224e6afead328df44964fe2772>@@@Z 000000018000c5a0 f   libucrt:per_thread_data.obj
 0001:0000b620       ??$?RV<lambda_aa87e3671a710a21b5dc78c0bdf72e11>@@AEAV<lambda_92619d2358a28f41a33ba319515a20b9>@@V<lambda_6992ecaafeb10aed2b74cb1fae11a551>@@@?$__crt_seh_guarded_call@X@@QEAAX$$QEAV<lambda_aa87e3671a710a21b5dc78c0bdf72e11>@@AEAV<lambda_92619d2358a28f41a33ba319515a20b9>@@$$QEAV<lambda_6992ecaafeb10aed2b74cb1fae11a551>@@@Z 000000018000c620 f   libucrt:per_thread_data.obj
 0001:0000b670       ??$?RV<lambda_f2e299630e499de9f9a165e60fcd3db5>@@AEAV<lambda_2ae9d31cdba2644fcbeaf08da7c24588>@@V<lambda_40d01ff24d0e7b3814fdbdcee8eab3c7>@@@?$__crt_seh_guarded_call@X@@QEAAX$$QEAV<lambda_f2e299630e499de9f9a165e60fcd3db5>@@AEAV<lambda_2ae9d31cdba2644fcbeaf08da7c24588>@@$$QEAV<lambda_40d01ff24d0e7b3814fdbdcee8eab3c7>@@@Z 000000018000c670 f   libucrt:per_thread_data.obj
 0001:0000b6e0       ?construct_ptd_array@@YAXQEAU__acrt_ptd@@@Z 000000018000c6e0 f   libucrt:per_thread_data.obj
 0001:0000b7a8       ?destroy_fls@@YAXPEAX@Z    000000018000c7a8 f   libucrt:per_thread_data.obj
 0001:0000b7d8       ?destroy_ptd_array@@YAXQEAU__acrt_ptd@@@Z 000000018000c7d8 f   libucrt:per_thread_data.obj
 0001:0000b8c8       ?replace_current_thread_locale_nolock@@YAXQEAU__acrt_ptd@@QEAU__crt_locale_data@@@Z 000000018000c8c8 f   libucrt:per_thread_data.obj
 0001:0000bd40       ??$?RV<lambda_410d79af7f07d98d83a3f525b3859a53>@@AEAV<lambda_3e16ef9562a7dcce91392c22ab16ea36>@@V<lambda_38119f0e861e05405d8a144b9b982f0a>@@@?$__crt_seh_guarded_call@X@@QEAAX$$QEAV<lambda_410d79af7f07d98d83a3f525b3859a53>@@AEAV<lambda_3e16ef9562a7dcce91392c22ab16ea36>@@$$QEAV<lambda_38119f0e861e05405d8a144b9b982f0a>@@@Z 000000018000cd40 f   libucrt:wsetlocale.obj
 0001:0000c038       ?<lambda_invoker_cdecl>@<lambda_a1ce4c8ae42411fd470c77163914f50e>@@CAHPEBX0@Z 000000018000d038 f   libucrt:argv_wildcards.obj
 0001:0000c380       ??$common_expand_argv_wildcards@D@@YAHQEAPEADQEAPEAPEAD@Z 000000018000d380 f   libucrt:argv_wildcards.obj
 0001:0000c5b8       ??$copy_and_add_argument_to_buffer@D@@YAHQEBD0_KAEAV?$argument_list@D@?A0x5f5c8891@@@Z 000000018000d5b8 f   libucrt:argv_wildcards.obj
 0001:0000c748       ??$expand_argument_wildcards@D@@YAHQEAD0AEAV?$argument_list@D@?A0x5f5c8891@@@Z 000000018000d748 f   libucrt:argv_wildcards.obj
 0001:0000cce8       ??$?RV<lambda_efdfa57d1f175319df784efa44bb7b81>@@AEAV<lambda_5f0a4c1567f8adc6734073e5d1e1b35c>@@V<lambda_2e8a7d3640ea6ccb4c2413664c2db6fd>@@@?$__crt_seh_guarded_call@X@@QEAAX$$QEAV<lambda_efdfa57d1f175319df784efa44bb7b81>@@AEAV<lambda_5f0a4c1567f8adc6734073e5d1e1b35c>@@$$QEAV<lambda_2e8a7d3640ea6ccb4c2413664c2db6fd>@@@Z 000000018000dce8 f   libucrt:mbctype.obj
 0001:0000ce40       ?CPtoLocaleName@@YAPEB_WH@Z 000000018000de40 f   libucrt:mbctype.obj
 0001:0000ce90       ?getSystemCP@@YAHH@Z       000000018000de90 f   libucrt:mbctype.obj
 0001:0000cf38       ?setSBCS@@YAXPEAU__crt_multibyte_data@@@Z 000000018000df38 f   libucrt:mbctype.obj
 0001:0000cfc0       ?setSBUpLow@@YAXPEAU__crt_multibyte_data@@@Z 000000018000dfc0 f   libucrt:mbctype.obj
 0001:0000d1d0       ?setmbcp_internal@@YAHH_NQEAU__acrt_ptd@@QEAPEAU__crt_multibyte_data@@@Z 000000018000e1d0 f   libucrt:mbctype.obj
 0001:0000d340       ?update_thread_multibyte_data_internal@@YAPEAU__crt_multibyte_data@@QEAU__acrt_ptd@@QEAPEAU1@@Z 000000018000e340 f   libucrt:mbctype.obj
 0001:0000d728       ?x_ismbbtype_l@@YAHPEAU__crt_locale_pointers@@IHH@Z 000000018000e728 f   libucrt:ismbbyte.obj
 0001:0000db18       ?try_get_function@@YAPEAXW4function_id@?A0x391cf84c@@QEBDQEBW4module_id@2@2@Z 000000018000eb18 f   libucrt:winapi_thunks.obj
 0001:0000e2c8       ?initialize_inherited_file_handles_nolock@@YAXXZ 000000018000f2c8 f   libucrt:ioinit.obj
 0001:0000e3c8       ?initialize_stdio_handles_nolock@@YAXXZ 000000018000f3c8 f   libucrt:ioinit.obj
 0001:0000e6c0       ??$?RV<lambda_450d765d439847d4c735a33c368b5fc0>@@AEAV<lambda_44731a7d0e6d81c3e6aa82d741081786>@@V<lambda_601a2a7da3b7a96e9554ac7215c4b07c>@@@?$__crt_seh_guarded_call@P6AXH@Z@@QEAAP6AXH@Z$$QEAV<lambda_450d765d439847d4c735a33c368b5fc0>@@AEAV<lambda_44731a7d0e6d81c3e6aa82d741081786>@@$$QEAV<lambda_601a2a7da3b7a96e9554ac7215c4b07c>@@@Z 000000018000f6c0 f   libucrt:signal.obj
 0001:0000e710       ?get_global_action_nolock@@YAPEAP6AXH@ZH@Z 000000018000f710 f   libucrt:signal.obj
 0001:0000ea40       ??$?RV<lambda_842d9ff0dc9ef11c61343bbaebe7f885>@@AEAV<lambda_c5860995281e5c4ce005b3de8f5874ee>@@V<lambda_d90129c13df834fdcbf8d2b88dafcf2d>@@@?$__crt_seh_guarded_call@X@@QEAAX$$QEAV<lambda_842d9ff0dc9ef11c61343bbaebe7f885>@@AEAV<lambda_c5860995281e5c4ce005b3de8f5874ee>@@$$QEAV<lambda_d90129c13df834fdcbf8d2b88dafcf2d>@@@Z 000000018000fa40 f   libucrt:fflush.obj
 0001:0000eb08       ??$?RV<lambda_886d6c58226a84441f68b9f2b8217b83>@@AEAV<lambda_ab61a845afdef5b7c387490eaf3616ee>@@V<lambda_f7f22ab5edc0698d5f6905b0d3f44752>@@@?$__crt_seh_guarded_call@X@@QEAAX$$QEAV<lambda_886d6c58226a84441f68b9f2b8217b83>@@AEAV<lambda_ab61a845afdef5b7c387490eaf3616ee>@@$$QEAV<lambda_f7f22ab5edc0698d5f6905b0d3f44752>@@@Z 000000018000fb08 f   libucrt:fflush.obj
 0001:0000ebf8       ?common_flush_all@@YAH_N@Z 000000018000fbf8 f   libucrt:fflush.obj
 0001:0000f7f8       ?free_crt_array_internal@@YAXQEAPEBX_K@Z 00000001800107f8 f   libucrt:inittime.obj
 0001:00010148       ?__acrt_LCMapStringA_stat@@YAHPEAU__crt_locale_pointers@@PEB_WKPEBDHPEADHHH@Z 0000000180011148 f   libucrt:lcmapstringa.obj
 0001:000104f8       ?initialize_multibyte@@YAHXZ 00000001800114f8 f   libucrt:multibyte_initializer.obj
 0001:000109f0       ??$?RV<lambda_a37b2b86f63e897a80ea819b0eb08c01>@@AEAV<lambda_38ce7e780aa69e748d6df282ebc68efe>@@V<lambda_99fb1378e971ab6e7edea83e3a7a83a2>@@@?$__crt_seh_guarded_call@H@@QEAAH$$QEAV<lambda_a37b2b86f63e897a80ea819b0eb08c01>@@AEAV<lambda_38ce7e780aa69e748d6df282ebc68efe>@@$$QEAV<lambda_99fb1378e971ab6e7edea83e3a7a83a2>@@@Z 00000001800119f0 f   libucrt:commit.obj
 0001:00010b48       ?write_double_translated_ansi_nolock@@YA?AUwrite_result@?A0x17268360@@HQEBDI@Z 0000000180011b48 f   libucrt:write.obj
 0001:00011028       ?write_text_ansi_nolock@@YA?AUwrite_result@?A0x17268360@@HQEBDI@Z 0000000180012028 f   libucrt:write.obj
 0001:00011178       ?write_text_utf16le_nolock@@YA?AUwrite_result@?A0x17268360@@HQEBDI@Z 0000000180012178 f   libucrt:write.obj
 0001:000112d0       ?write_text_utf8_nolock@@YA?AUwrite_result@?A0x17268360@@HQEBDI@Z 00000001800122d0 f   libucrt:write.obj
 0001:00011d40       ??$common_lseek_nolock@_J@@YA_JH_JH@Z 0000000180012d40 f   libucrt:lseek.obj
 0001:000122a8       ??$?RV<lambda_751a882b2c74d4b022dec766aa51a29a>@@AEAV<lambda_628dfdc04ba53c8bfc02c9951375f3f5>@@V<lambda_f6c7be5f7998530c34de24c7437d6b54>@@@?$__crt_seh_guarded_call@H@@QEAAH$$QEAV<lambda_751a882b2c74d4b022dec766aa51a29a>@@AEAV<lambda_628dfdc04ba53c8bfc02c9951375f3f5>@@$$QEAV<lambda_f6c7be5f7998530c34de24c7437d6b54>@@@Z 00000001800132a8 f   libucrt:close.obj
 0001:000126e4       ?dtor$0@?0??OpenFromCommandLine@@YAPEA_WPEB_W@Z@4HA 00000001800136e4 f   OpenCmd.obj
 0001:00012700       ?dtor$1@?0??OpenFromCommandLine@@YAPEA_WPEB_W@Z@4HA 0000000180013700 f   OpenCmd.obj
 0001:00012700       ?dtor$2@?0??OpenFromCommandLine@@YAPEA_WPEB_W@Z@4HA 0000000180013700 f   OpenCmd.obj
 0001:00012700       ?dtor$3@?0??OpenFromCommandLine@@YAPEA_WPEB_W@Z@4HA 0000000180013700 f   OpenCmd.obj
 0001:00012700       ?dtor$4@?0??OpenFromCommandLine@@YAPEA_WPEB_W@Z@4HA 0000000180013700 f   OpenCmd.obj
 0001:0001271c       ?fin$0@?0??dllmain_crt_process_attach@@YAHQEAUHINSTANCE__@@QEAX@Z@4HA 000000018001371c f   LIBCMT:dll_dllmain.obj
 0001:0001273c       ?fin$0@?0??dllmain_crt_process_detach@@YAH_N@Z@4HA 000000018001373c f   LIBCMT:dll_dllmain.obj
 0001:0001275c       ?fin$1@?0??dllmain_crt_process_detach@@YAH_N@Z@4HA 000000018001375c f   LIBCMT:dll_dllmain.obj
 0001:00012778       ?filt$0@?0??dllmain_dispatch@@YAHQEAUHINSTANCE__@@KQEAX@Z@4HA 0000000180013778 f   LIBCMT:dll_dllmain.obj
 0001:000127b4       __scrt_is_nonwritable_in_current_image$filt$0 00000001800137b4 f   LIBCMT:utility.obj
 0001:000127dc       $LN31                      00000001800137dc     LIBCMT:utility.obj
 0001:000127e0       ?filt$0@?0???$_CallSETranslator@V__FrameHandler3@@@@YAHPEAUEHExceptionRecord@@PEA_KPEAU_CONTEXT@@PEAU_xDISPATCHER_CONTEXT@@PEBU_s_FuncInfo@@K1H@Z@4HA 00000001800137e0 f   libvcruntime:risctrnsctrl.obj
 0001:00012870       __DestructExceptionObject$filt$0 0000000180013870 f   libvcruntime:ehhelpers.obj
 0001:00012968       $LN30                      0000000180013968     libvcruntime:ehhelpers.obj
 0001:0001296c       $LN31                      000000018001396c     libvcruntime:ehhelpers.obj
 0001:00012970       $LN32                      0000000180013970     libvcruntime:ehhelpers.obj
 0001:00012974       $LN33                      0000000180013974     libvcruntime:ehhelpers.obj
 0001:00012978       ?filt$0@?0??CxxCallCatchBlock@__FrameHandler3@@SAPEAXPEAU_EXCEPTION_RECORD@@@Z@4HA 0000000180013978 f   libvcruntime:frame.obj
 0001:000129a0       ?fin$1@?0??CxxCallCatchBlock@__FrameHandler3@@SAPEAXPEAU_EXCEPTION_RECORD@@@Z@4HA 00000001800139a0 f   libvcruntime:frame.obj
 0001:00012a38       $LN31                      0000000180013a38     libvcruntime:frame.obj
 0001:00012a3c       $LN32                      0000000180013a3c     libvcruntime:frame.obj
 0001:00012a40       ?filt$0@?0??FrameUnwindToState@__FrameHandler3@@SAXPEA_KPEAU_xDISPATCHER_CONTEXT@@PEBU_s_FuncInfo@@H@Z@4HA 0000000180013a40 f   libvcruntime:frame.obj
 0001:00012a5c       ?fin$1@?0??FrameUnwindToState@__FrameHandler3@@SAXPEA_KPEAU_xDISPATCHER_CONTEXT@@PEBU_s_FuncInfo@@H@Z@4HA 0000000180013a5c f   libvcruntime:frame.obj
 0001:00012a90       _query_new_handler$fin$0   0000000180013a90 f   libucrt:new_handler.obj
 0001:00012ab0       ?fin$0@?0???$?RV<lambda_0ae27a3a962d80f24befdcbee591983d>@@AEAV<lambda_8d0ee55de4b1038c4002e0adecdf1839>@@V<lambda_dc504788e8f1664fe9b84e20bfb512f2>@@@?$__crt_seh_guarded_call@X@@QEAAX$$QEAV<lambda_0ae27a3a962d80f24befdcbee591983d>@@AEAV<lambda_8d0ee55de4b1038c4002e0adecdf1839>@@$$QEAV<lambda_dc504788e8f1664fe9b84e20bfb512f2>@@@Z@4HA 0000000180013ab0 f   libucrt:per_thread_data.obj
 0001:00012ab0       ?fin$0@?0???$?RV<lambda_2d41944a1d46af3157314b8a01080d33>@@AEAV<lambda_8f455de75cd7d7f24b4096f044d8b9e6>@@V<lambda_aa500f224e6afead328df44964fe2772>@@@?$__crt_seh_guarded_call@X@@QEAAX$$QEAV<lambda_2d41944a1d46af3157314b8a01080d33>@@AEAV<lambda_8f455de75cd7d7f24b4096f044d8b9e6>@@$$QEAV<lambda_aa500f224e6afead328df44964fe2772>@@@Z@4HA 0000000180013ab0 f   libucrt:per_thread_data.obj
 0001:00012ab0       ?fin$0@?0???$?RV<lambda_aa87e3671a710a21b5dc78c0bdf72e11>@@AEAV<lambda_92619d2358a28f41a33ba319515a20b9>@@V<lambda_6992ecaafeb10aed2b74cb1fae11a551>@@@?$__crt_seh_guarded_call@X@@QEAAX$$QEAV<lambda_aa87e3671a710a21b5dc78c0bdf72e11>@@AEAV<lambda_92619d2358a28f41a33ba319515a20b9>@@$$QEAV<lambda_6992ecaafeb10aed2b74cb1fae11a551>@@@Z@4HA 0000000180013ab0 f   libucrt:per_thread_data.obj
 0001:00012ab0       ?fin$0@?0???$?RV<lambda_f2e299630e499de9f9a165e60fcd3db5>@@AEAV<lambda_2ae9d31cdba2644fcbeaf08da7c24588>@@V<lambda_40d01ff24d0e7b3814fdbdcee8eab3c7>@@@?$__crt_seh_guarded_call@X@@QEAAX$$QEAV<lambda_f2e299630e499de9f9a165e60fcd3db5>@@AEAV<lambda_2ae9d31cdba2644fcbeaf08da7c24588>@@$$QEAV<lambda_40d01ff24d0e7b3814fdbdcee8eab3c7>@@@Z@4HA 0000000180013ab0 f   libucrt:per_thread_data.obj
 0001:00012ab0       ?fin$0@?0???$?RV<lambda_efdfa57d1f175319df784efa44bb7b81>@@AEAV<lambda_5f0a4c1567f8adc6734073e5d1e1b35c>@@V<lambda_2e8a7d3640ea6ccb4c2413664c2db6fd>@@@?$__crt_seh_guarded_call@X@@QEAAX$$QEAV<lambda_efdfa57d1f175319df784efa44bb7b81>@@AEAV<lambda_5f0a4c1567f8adc6734073e5d1e1b35c>@@$$QEAV<lambda_2e8a7d3640ea6ccb4c2413664c2db6fd>@@@Z@4HA 0000000180013ab0 f   libucrt:mbctype.obj
 0001:00012ab0       ?fin$0@?0???$?RV<lambda_450d765d439847d4c735a33c368b5fc0>@@AEAV<lambda_44731a7d0e6d81c3e6aa82d741081786>@@V<lambda_601a2a7da3b7a96e9554ac7215c4b07c>@@@?$__crt_seh_guarded_call@P6AXH@Z@@QEAAP6AXH@Z$$QEAV<lambda_450d765d439847d4c735a33c368b5fc0>@@AEAV<lambda_44731a7d0e6d81c3e6aa82d741081786>@@$$QEAV<lambda_601a2a7da3b7a96e9554ac7215c4b07c>@@@Z@4HA 0000000180013ab0 f   libucrt:signal.obj
 0001:00012ab0       ?fin$0@?0???$?RV<lambda_d80eeec6fff315bfe5c115232f3240e3>@@AEAV<lambda_6e4b09c48022b2350581041d5f6b0c4c>@@V<lambda_2358e3775559c9db80273638284d5e45>@@@?$__crt_seh_guarded_call@X@@QEAAX$$QEAV<lambda_d80eeec6fff315bfe5c115232f3240e3>@@AEAV<lambda_6e4b09c48022b2350581041d5f6b0c4c>@@$$QEAV<lambda_2358e3775559c9db80273638284d5e45>@@@Z@4HA 0000000180013ab0 f   libucrt:exit.obj
 0001:00012ab0       ?fin$0@?0???$?RV<lambda_7777bce6b2f8c936911f934f8298dc43>@@AEAV<lambda_f03950bc5685219e0bcd2087efbe011e>@@V<lambda_3883c3dff614d5e0c5f61bb1ac94921c>@@@?$__crt_seh_guarded_call@H@@QEAAH$$QEAV<lambda_7777bce6b2f8c936911f934f8298dc43>@@AEAV<lambda_f03950bc5685219e0bcd2087efbe011e>@@$$QEAV<lambda_3883c3dff614d5e0c5f61bb1ac94921c>@@@Z@4HA 0000000180013ab0 f   libucrt:onexit.obj
 0001:00012ad4       ?filt$0@?0???R<lambda_6e4b09c48022b2350581041d5f6b0c4c>@@QEBA@XZ@4HA 0000000180013ad4 f   libucrt:exit.obj
 0001:00012af8       ?fin$0@?0???$?RV<lambda_410d79af7f07d98d83a3f525b3859a53>@@AEAV<lambda_3e16ef9562a7dcce91392c22ab16ea36>@@V<lambda_38119f0e861e05405d8a144b9b982f0a>@@@?$__crt_seh_guarded_call@X@@QEAAX$$QEAV<lambda_410d79af7f07d98d83a3f525b3859a53>@@AEAV<lambda_3e16ef9562a7dcce91392c22ab16ea36>@@$$QEAV<lambda_38119f0e861e05405d8a144b9b982f0a>@@@Z@4HA 0000000180013af8 f   libucrt:wsetlocale.obj
 0001:00012b1c       ?fin$0@?0??update_thread_multibyte_data_internal@@YAPEAU__crt_multibyte_data@@QEAU__acrt_ptd@@QEAPEAU1@@Z@4HA 0000000180013b1c f   libucrt:mbctype.obj
 0001:00012b3c       __acrt_initialize_lowio$fin$0 0000000180013b3c f   libucrt:ioinit.obj
 0001:00012b3c       __acrt_lowio_ensure_fh_exists$fin$0 0000000180013b3c f   libucrt:osfinfo.obj
 0001:00012b5c       raise$fin$0                0000000180013b5c f   libucrt:signal.obj
 0001:00012b84       ?fin$0@?0???$?RV<lambda_842d9ff0dc9ef11c61343bbaebe7f885>@@AEAV<lambda_c5860995281e5c4ce005b3de8f5874ee>@@V<lambda_d90129c13df834fdcbf8d2b88dafcf2d>@@@?$__crt_seh_guarded_call@X@@QEAAX$$QEAV<lambda_842d9ff0dc9ef11c61343bbaebe7f885>@@AEAV<lambda_c5860995281e5c4ce005b3de8f5874ee>@@$$QEAV<lambda_d90129c13df834fdcbf8d2b88dafcf2d>@@@Z@4HA 0000000180013b84 f   libucrt:fflush.obj
 0001:00012ba8       ?fin$0@?0???$?RV<lambda_886d6c58226a84441f68b9f2b8217b83>@@AEAV<lambda_ab61a845afdef5b7c387490eaf3616ee>@@V<lambda_f7f22ab5edc0698d5f6905b0d3f44752>@@@?$__crt_seh_guarded_call@X@@QEAAX$$QEAV<lambda_886d6c58226a84441f68b9f2b8217b83>@@AEAV<lambda_ab61a845afdef5b7c387490eaf3616ee>@@$$QEAV<lambda_f7f22ab5edc0698d5f6905b0d3f44752>@@@Z@4HA 0000000180013ba8 f   libucrt:fflush.obj
 0001:00012bcc       __acrt_update_thread_locale_data$fin$0 0000000180013bcc f   libucrt:locale_refcounting.obj
 0001:00012bec       ?fin$0@?0???$?RV<lambda_751a882b2c74d4b022dec766aa51a29a>@@AEAV<lambda_628dfdc04ba53c8bfc02c9951375f3f5>@@V<lambda_f6c7be5f7998530c34de24c7437d6b54>@@@?$__crt_seh_guarded_call@H@@QEAAH$$QEAV<lambda_751a882b2c74d4b022dec766aa51a29a>@@AEAV<lambda_628dfdc04ba53c8bfc02c9951375f3f5>@@$$QEAV<lambda_f6c7be5f7998530c34de24c7437d6b54>@@@Z@4HA 0000000180013bec f   libucrt:close.obj
 0001:00012bec       ?fin$0@?0???$?RV<lambda_a37b2b86f63e897a80ea819b0eb08c01>@@AEAV<lambda_38ce7e780aa69e748d6df282ebc68efe>@@V<lambda_99fb1378e971ab6e7edea83e3a7a83a2>@@@?$__crt_seh_guarded_call@H@@QEAAH$$QEAV<lambda_a37b2b86f63e897a80ea819b0eb08c01>@@AEAV<lambda_38ce7e780aa69e748d6df282ebc68efe>@@$$QEAV<lambda_99fb1378e971ab6e7edea83e3a7a83a2>@@@Z@4HA 0000000180013bec f   libucrt:commit.obj
 0001:00012c10       _write$fin$0               0000000180013c10 f   libucrt:write.obj
 0001:00012c30       _fcloseall$fin$0           0000000180013c30 f   libucrt:closeall.obj
 0001:00012c50       fclose$fin$0               0000000180013c50 f   libucrt:fclose.obj
 0001:00012c70       _IsNonwritableInCurrentImage$filt$0 0000000180013c70 f   LIBCMT:pesect.obj
 0002:00000418       GS_ExceptionPointers       0000000180014418     LIBCMT:gs_report.obj
 0002:000004b0       ?ExceptionTemplate@?1??UnwindNestedFrames@__FrameHandler3@@SAXPEA_KPEAUEHExceptionRecord@@PEAU_CONTEXT@@0PEAXPEBU_s_FuncInfo@@HHPEBU_s_HandlerType@@PEAU_xDISPATCHER_CONTEXT@@E@Z@4U_EXCEPTION_RECORD@@B 00000001800144b0     libvcruntime:risctrnsctrl.obj
 0002:00000580       ?tokenTable@@3QBUStringLiteral@@B 0000000180014580     libvcruntime:undname.obj
 0002:00000680       ?nameTable@@3QBUStringLiteral@@B 0000000180014680     libvcruntime:undname.obj
 0002:00000bb0       ?rttiTable@@3QBUStringLiteral@@B 0000000180014bb0     libvcruntime:undname.obj
 0002:00000c00       ?IndirectionName@@3QBUStringLiteral@@B 0000000180014c00     libvcruntime:undname.obj
 0002:00000c60       ?PrefixName@@3QBUStringLiteral@@B 0000000180014c60     libvcruntime:undname.obj
 0002:00001440       __acrt_initializers        0000000180015440     libucrt:initialization.obj
 0002:00001540       ?errtable@@3QBUerrentry@?A0x31fdb9ec@@B 0000000180015540     libucrt:errno.obj
 0002:00001d70       ?module_names@?A0x391cf84c@@3QBQEB_WB 0000000180015d70     libucrt:winapi_thunks.obj
 0002:00002318       ?candidate_modules@?1??try_get_AreFileApisANSI@@YAP6AHXZXZ@4QBW4module_id@?A0x391cf84c@@B 0000000180016318     libucrt:winapi_thunks.obj
 0002:00002330       ?candidate_modules@?1??try_get_FlsAlloc@@YAP6AKP6AXPEAX@Z@ZXZ@4QBW4module_id@?A0x391cf84c@@B 0000000180016330     libucrt:winapi_thunks.obj
 0002:00002348       ?candidate_modules@?1??try_get_FlsFree@@YAP6AHK@ZXZ@4QBW4module_id@?A0x391cf84c@@B 0000000180016348     libucrt:winapi_thunks.obj
 0002:00002358       ?candidate_modules@?1??try_get_FlsGetValue@@YAP6APEAXK@ZXZ@4QBW4module_id@?A0x391cf84c@@B 0000000180016358     libucrt:winapi_thunks.obj
 0002:00002370       ?candidate_modules@?1??try_get_FlsSetValue@@YAP6AHKPEAX@ZXZ@4QBW4module_id@?A0x391cf84c@@B 0000000180016370     libucrt:winapi_thunks.obj
 0002:00002388       ?candidate_modules@?1??try_get_InitializeCriticalSectionEx@@YAP6AHPEAU_RTL_CRITICAL_SECTION@@KK@ZXZ@4QBW4module_id@?A0x391cf84c@@B 0000000180016388     libucrt:winapi_thunks.obj
 0002:000023b0       ?candidate_modules@?1??try_get_LCMapStringEx@@YAP6AHPEB_WK0HPEA_WHPEAU_nlsversioninfo@@PEAX_J@ZXZ@4QBW4module_id@?A0x391cf84c@@B 00000001800163b0     libucrt:winapi_thunks.obj
 0002:000023c8       ?candidate_modules@?1??try_get_LocaleNameToLCID@@YAP6AKPEB_WK@ZXZ@4QBW4module_id@?A0x391cf84c@@B 00000001800163c8     libucrt:winapi_thunks.obj
 0002:000023e4       ?candidate_modules@?1??try_get_AppPolicyGetProcessTerminationMethod@@YAP6AJPEAXPEAW4AppPolicyProcessTerminationMethod@@@ZXZ@4QBW4module_id@?A0x391cf84c@@B 00000001800163e4     libucrt:winapi_thunks.obj
 0002:00002a20       ?LcidToLocaleNameTable@?A0x881e4c05@@3QBULcidToLocaleName@1@B 0000000180016a20     libucrt:lcidtoname_downlevel.obj
 0002:00004470       ?LocaleNameToIndexTable@?A0x881e4c05@@3QBULocaleNameIndex@1@B 0000000180018470     libucrt:lcidtoname_downlevel.obj
 0002:00006208       ?tmpPrefix@?1??MakeTempNames@@YA_NPEAPEA_W0@Z@4QB_WB 000000018001a208     OpenCmd.obj
 0002:00006210       $cppxdata$ConfigureW       000000018001a210     FARCmds.obj
 0002:00006240       $cppxdata$SetStartupInfoW  000000018001a240     FARCmds.obj
 0002:00006270       $cppxdata$?OpenFromCommandLine@@YAPEA_WPEB_W@Z 000000018001a270     OpenCmd.obj
 0002:00006be0       $unwind$?SaveValue@PluginCheckBoxBinding@@UEAAXPEBUFarDialogItem@@H@Z 000000018001abe0     FARCmds.obj
 0002:00006bf8       $unwind$?AddOKCancel@PluginDialogBuilder@@QEAAXHHH_N@Z 000000018001abf8     FARCmds.obj
 0002:00006c14       $unwind$SetStartupInfoW    000000018001ac14     FARCmds.obj
 0002:00006c30       $stateUnwindMap$ConfigureW 000000018001ac30     FARCmds.obj
 0002:00006c30       $stateUnwindMap$SetStartupInfoW 000000018001ac30     FARCmds.obj
 0002:00006c40       $ip2state$SetStartupInfoW  000000018001ac40     FARCmds.obj
 0002:00006c58       $unwind$OpenW              000000018001ac58     FARCmds.obj
 0002:00006c70       $unwind$ConfigureW         000000018001ac70     FARCmds.obj
 0002:00006ca0       $ip2state$ConfigureW       000000018001aca0     FARCmds.obj
 0002:00006cf0       $unwind$?GetInt@@YAHPEB_WPEA_W@Z 000000018001acf0     Mix.obj
 0002:00006d00       $unwind$?GetShellLinkPath@@YAPEA_WPEB_W@Z 000000018001ad00     Mix.obj
 0002:00006d18       $unwind$?getCurrDir@@YAPEA_W_N@Z 000000018001ad18     OpenCmd.obj
 0002:00006d2c       $unwind$?createFile@@YAPEAXPEA_WH@Z 000000018001ad2c     OpenCmd.obj
 0002:00006d40       $unwind$?ThreadWhatUpdateScreen@@YAKPEAX@Z 000000018001ad40     OpenCmd.obj
 0002:00006d5c       $unwind$?MakeExecuteString@@YAPEB_WPEB_W@Z 000000018001ad5c     OpenCmd.obj
 0002:00006d74       $unwind$?__getContent@@YAPEA_WHPEA_W@Z 000000018001ad74     OpenCmd.obj
 0002:00006d88       $unwind$?__proc_WhereIs@@YAPEA_WHPEA_W_N@Z 000000018001ad88     OpenCmd.obj
 0002:00006da4       $unwind$?__proc_Link@@YA_NHPEA_W@Z 000000018001ada4     OpenCmd.obj
 0002:00006dbc       $unwind$?OpenFromCommandLine@@YAPEA_WPEB_W@Z 000000018001adbc     OpenCmd.obj
 0002:00006de0       $stateUnwindMap$?OpenFromCommandLine@@YAPEA_WPEB_W@Z 000000018001ade0     OpenCmd.obj
 0002:00006e10       $ip2state$?OpenFromCommandLine@@YAPEA_WPEB_W@Z 000000018001ae10     OpenCmd.obj
 0002:00006e90       $unwind$?dtor$0@?0??OpenFromCommandLine@@YAPEA_WPEB_W@Z@4HA 000000018001ae90     OpenCmd.obj
 0002:00006e90       $unwind$?dtor$1@?0??OpenFromCommandLine@@YAPEA_WPEB_W@Z@4HA 000000018001ae90     OpenCmd.obj
 0002:00006e90       $unwind$?dtor$2@?0??OpenFromCommandLine@@YAPEA_WPEB_W@Z@4HA 000000018001ae90     OpenCmd.obj
 0002:00006e90       $unwind$?dtor$3@?0??OpenFromCommandLine@@YAPEA_WPEB_W@Z@4HA 000000018001ae90     OpenCmd.obj
 0002:00006e90       $unwind$?dtor$4@?0??OpenFromCommandLine@@YAPEA_WPEB_W@Z@4HA 000000018001ae90     OpenCmd.obj
 0002:00006e98       __security_check_cookie_xdata 000000018001ae98     LIBCMT:arm64secgs.obj
 0002:00006ea0       __security_check_cookie_xdata_prolog 000000018001aea0     LIBCMT:arm64secgs.obj
 0002:00006ea1       __security_check_cookie_xdata_epilog1 000000018001aea1     LIBCMT:arm64secgs.obj
 0002:00006ea4       __gsfailure_xdata          000000018001aea4     LIBCMT:arm64secgs.obj
 0002:00006ea4       __security_check_cookie_xdata_end 000000018001aea4     LIBCMT:arm64secgs.obj
 0002:00006ea8       __gsfailure_xdata_prolog   000000018001aea8     LIBCMT:arm64secgs.obj
 0002:00006eac       __gsfailure_xdata_end      000000018001aeac     LIBCMT:arm64secgs.obj
 0002:00006eac       $unwind$??2@YAPEAX_K@Z     000000018001aeac     LIBCMT:new_scalar.obj
 0002:00006ebc       $unwind$?dllmain_crt_process_attach@@YAHQEAUHINSTANCE__@@QEAX@Z 000000018001aebc     LIBCMT:dll_dllmain.obj
 0002:00006ef4       $unwind$?fin$0@?0??dllmain_crt_process_attach@@YAHQEAUHINSTANCE__@@QEAX@Z@4HA 000000018001aef4     LIBCMT:dll_dllmain.obj
 0002:00006ef4       $unwind$?fin$0@?0??dllmain_crt_process_detach@@YAH_N@Z@4HA 000000018001aef4     LIBCMT:dll_dllmain.obj
 0002:00006ef4       $unwind$_query_new_handler$fin$0 000000018001aef4     libucrt:new_handler.obj
 0002:00006ef4       $unwind$__acrt_update_thread_locale_data$fin$0 000000018001aef4     libucrt:locale_refcounting.obj
 0002:00006ef4       $unwind$__acrt_initialize_lowio$fin$0 000000018001aef4     libucrt:ioinit.obj
 0002:00006ef4       $unwind$__acrt_lowio_ensure_fh_exists$fin$0 000000018001aef4     libucrt:osfinfo.obj
 0002:00006ef4       $unwind$_write$fin$0       000000018001aef4     libucrt:write.obj
 0002:00006ef4       $unwind$?fin$0@?0??update_thread_multibyte_data_internal@@YAPEAU__crt_multibyte_data@@QEAU__acrt_ptd@@QEAPEAU1@@Z@4HA 000000018001aef4     libucrt:mbctype.obj
 0002:00006ef4       $unwind$_fcloseall$fin$0   000000018001aef4     libucrt:closeall.obj
 0002:00006ef4       $unwind$fclose$fin$0       000000018001aef4     libucrt:fclose.obj
 0002:00006f00       $unwind$?dllmain_crt_process_detach@@YAH_N@Z 000000018001af00     LIBCMT:dll_dllmain.obj
 0002:00006f58       $unwind$?fin$1@?0??dllmain_crt_process_detach@@YAH_N@Z@4HA 000000018001af58     LIBCMT:dll_dllmain.obj
 0002:00006f58       $unwind$?filt$0@?0??FrameUnwindToState@__FrameHandler3@@SAXPEA_KPEAU_xDISPATCHER_CONTEXT@@PEBU_s_FuncInfo@@H@Z@4HA 000000018001af58     libvcruntime:frame.obj
 0002:00006f64       $unwind$?dllmain_dispatch@@YAHQEAUHINSTANCE__@@KQEAX@Z 000000018001af64     LIBCMT:dll_dllmain.obj
 0002:00006f88       $unwind$?filt$0@?0??dllmain_dispatch@@YAHQEAUHINSTANCE__@@KQEAX@Z@4HA 000000018001af88     LIBCMT:dll_dllmain.obj
 0002:00006f94       $unwind$?__scrt_throw_std_bad_alloc@@YAXXZ 000000018001af94     LIBCMT:throw_bad_alloc.obj
 0002:00006f94       $unwind$?__scrt_throw_std_bad_array_new_length@@YAXXZ 000000018001af94     LIBCMT:throw_bad_alloc.obj
 0002:00006f9c       $unwind$__scrt_is_nonwritable_in_current_image 000000018001af9c     LIBCMT:utility.obj
 0002:00006fbc       $unwind$__scrt_is_nonwritable_in_current_image$filt$0 000000018001afbc     LIBCMT:utility.obj
 0002:00006fc8       $unwind$__scrt_acquire_startup_lock 000000018001afc8     LIBCMT:utility.obj
 0002:00006fd4       $unwind$__scrt_initialize_onexit_tables 000000018001afd4     LIBCMT:utility.obj
 0002:00006fe0       $unwind$?UnwindNestedFrames@__FrameHandler3@@SAXPEA_KPEAUEHExceptionRecord@@PEAU_CONTEXT@@0PEAXPEBU_s_FuncInfo@@HHPEBU_s_HandlerType@@PEAU_xDISPATCHER_CONTEXT@@E@Z 000000018001afe0     libvcruntime:risctrnsctrl.obj
 0002:00006ff4       $unwind$?GetRangeOfTrysToCheck@__FrameHandler3@@SA?AU?$pair@Viterator@TryBlockMap@__FrameHandler3@@V123@@std@@AEAVTryBlockMap@1@HPEAU_xDISPATCHER_CONTEXT@@PEBU_s_FuncInfo@@H@Z 000000018001aff4     libvcruntime:risctrnsctrl.obj
 0002:00007004       $unwind$_FindAndUnlinkFrame 000000018001b004     libvcruntime:risctrnsctrl.obj
 0002:00007010       $unwind$??$_CallSETranslator@V__FrameHandler3@@@@YAHPEAUEHExceptionRecord@@PEA_KPEAU_CONTEXT@@PEAU_xDISPATCHER_CONTEXT@@PEBU_s_FuncInfo@@K1H@Z 000000018001b010     libvcruntime:risctrnsctrl.obj
 0002:00007030       $unwind$?filt$0@?0???$_CallSETranslator@V__FrameHandler3@@@@YAHPEAUEHExceptionRecord@@PEA_KPEAU_CONTEXT@@PEAU_xDISPATCHER_CONTEXT@@PEBU_s_FuncInfo@@K1H@Z@4HA 000000018001b030     libvcruntime:risctrnsctrl.obj
 0002:0000703c       $unwind$_IsExceptionObjectToBeDestroyed 000000018001b03c     libvcruntime:ehhelpers.obj
 0002:0000704c       $unwind$__FrameUnwindFilter 000000018001b04c     libvcruntime:ehhelpers.obj
 0002:00007058       $unwind$__DestructExceptionObject 000000018001b058     libvcruntime:ehhelpers.obj
 0002:0000707c       $unwind$__DestructExceptionObject$filt$0 000000018001b07c     libvcruntime:ehhelpers.obj
 0002:00007088       $unwind$__vcrt_getptd      000000018001b088     libvcruntime:per_thread_data.obj
 0002:00007094       $unwind$?FrameUnwindToState@__FrameHandler3@@SAXPEA_KPEAU_xDISPATCHER_CONTEXT@@PEBU_s_FuncInfo@@H@Z 000000018001b094     libvcruntime:frame.obj
 0002:000070e0       $unwind$?fin$1@?0??FrameUnwindToState@__FrameHandler3@@SAXPEA_KPEAU_xDISPATCHER_CONTEXT@@PEBU_s_FuncInfo@@H@Z@4HA 000000018001b0e0     libvcruntime:frame.obj
 0002:000070ec       $unwind$?CxxCallCatchBlock@__FrameHandler3@@SAPEAXPEAU_EXCEPTION_RECORD@@@Z 000000018001b0ec     libvcruntime:frame.obj
 0002:00007128       $unwind$?filt$0@?0??CxxCallCatchBlock@__FrameHandler3@@SAPEAXPEAU_EXCEPTION_RECORD@@@Z@4HA 000000018001b128     libvcruntime:frame.obj
 0002:00007128       $unwind$raise$fin$0        000000018001b128     libucrt:signal.obj
 0002:00007134       $unwind$?fin$1@?0??CxxCallCatchBlock@__FrameHandler3@@SAPEAXPEAU_EXCEPTION_RECORD@@@Z@4HA 000000018001b134     libvcruntime:frame.obj
 0002:00007140       $unwind$?IsInExceptionSpec@@YAEPEAUEHExceptionRecord@@PEBU_s_ESTypeList@@@Z 000000018001b140     libvcruntime:frame.obj
 0002:00007154       $unwind$??$__InternalCxxFrameHandler@V__FrameHandler3@@@@YA?AW4_EXCEPTION_DISPOSITION@@PEAUEHExceptionRecord@@PEA_KPEAU_CONTEXT@@PEAU_xDISPATCHER_CONTEXT@@PEBU_s_FuncInfo@@H1E@Z 000000018001b154     libvcruntime:frame.obj
 0002:00007168       $unwind$??$BuildCatchObjectHelperInternal@V__FrameHandler3@@@@YAHPEAUEHExceptionRecord@@PEAXPEBU_s_HandlerType@@PEBU_s_CatchableType@@@Z 000000018001b168     libvcruntime:frame.obj
 0002:000071a0       $unwind$??$BuildCatchObjectInternal@V__FrameHandler3@@@@YAXPEAUEHExceptionRecord@@PEAXPEBU_s_HandlerType@@PEBU_s_CatchableType@@@Z 000000018001b1a0     libvcruntime:frame.obj
 0002:000071c8       $unwind$??$FindHandler@V__FrameHandler3@@@@YAXPEAUEHExceptionRecord@@PEA_KPEAU_CONTEXT@@PEAU_xDISPATCHER_CONTEXT@@PEBU_s_FuncInfo@@EH1@Z 000000018001b1c8     libvcruntime:frame.obj
 0002:000071e8       $unwind$??$FindHandlerForForeignException@V__FrameHandler3@@@@YAXPEAUEHExceptionRecord@@PEA_KPEAU_CONTEXT@@PEAU_xDISPATCHER_CONTEXT@@PEBU_s_FuncInfo@@HH1@Z 000000018001b1e8     libvcruntime:frame.obj
 0002:000071fc       _NLG_Notify_xdata          000000018001b1fc     libvcruntime:notify.obj
 0002:00007204       _NLG_Notify_xdata_prolog   000000018001b204     libvcruntime:notify.obj
 0002:00007206       _NLG_Notify_xdata_epilog1  000000018001b206     libvcruntime:notify.obj
 0002:00007208       _NLG_Notify_xdata_end      000000018001b208     libvcruntime:notify.obj
 0002:00007208       __NLG_Return2_xdata        000000018001b208     libvcruntime:notify.obj
 0002:0000720c       __NLG_Return2_xdata_prolog 000000018001b20c     libvcruntime:notify.obj
 0002:00007210       __C_ExecuteExceptionFilter_xdata 000000018001b210     libvcruntime:handler.obj
 0002:00007210       __NLG_Return2_xdata_end    000000018001b210     libvcruntime:notify.obj
 0002:00007218       __C_ExecuteExceptionFilter_xdata_prolog 000000018001b218     libvcruntime:handler.obj
 0002:00007225       __C_ExecuteExceptionFilter_xdata_epilog1 000000018001b225     libvcruntime:handler.obj
 0002:00007230       __C_ExecuteExceptionFilter_xdata_end 000000018001b230     libvcruntime:handler.obj
 0002:00007230       __C_ExecuteTerminationHandler_xdata 000000018001b230     libvcruntime:handler.obj
 0002:00007238       __C_ExecuteTerminationHandler_xdata_prolog 000000018001b238     libvcruntime:handler.obj
 0002:00007245       __C_ExecuteTerminationHandler_xdata_epilog1 000000018001b245     libvcruntime:handler.obj
 0002:00007250       __C_ExecuteTerminationHandler_xdata_end 000000018001b250     libvcruntime:handler.obj
 0002:00007250       _CallSettingFrame_xdata    000000018001b250     libvcruntime:handlers.obj
 0002:00007258       _CallSettingFrame_xdata_prolog 000000018001b258     libvcruntime:handlers.obj
 0002:00007265       _CallSettingFrame_xdata_epilog1 000000018001b265     libvcruntime:handlers.obj
 0002:00007274       _CallSettingFrame_xdata_end 000000018001b274     libvcruntime:handlers.obj
 0002:00007274       memcpy_xdata               000000018001b274     libvcruntime:memcpy.obj
 0002:00007278       memcpy_xdata_prolog        000000018001b278     libvcruntime:memcpy.obj
 0002:0000727c       __memcpy_forward_large_neon_xdata 000000018001b27c     libvcruntime:memcpy.obj
 0002:0000727c       memcpy_xdata_end           000000018001b27c     libvcruntime:memcpy.obj
 0002:00007280       __memcpy_forward_large_neon_xdata_prolog 000000018001b280     libvcruntime:memcpy.obj
 0002:00007284       __memcpy_forward_large_neon_xdata_end 000000018001b284     libvcruntime:memcpy.obj
 0002:00007284       __memcpy_reverse_xdata     000000018001b284     libvcruntime:memcpy.obj
 0002:00007288       __memcpy_reverse_xdata_prolog 000000018001b288     libvcruntime:memcpy.obj
 0002:0000728c       __memcpy_reverse_large_neon_xdata 000000018001b28c     libvcruntime:memcpy.obj
 0002:0000728c       __memcpy_reverse_xdata_end 000000018001b28c     libvcruntime:memcpy.obj
 0002:00007290       __memcpy_reverse_large_neon_xdata_prolog 000000018001b290     libvcruntime:memcpy.obj
 0002:00007294       __memcpy_reverse_large_neon_xdata_end 000000018001b294     libvcruntime:memcpy.obj
 0002:00007294       $unwind$free               000000018001b294     libucrt:free.obj
 0002:0000729c       $unwind$_query_new_handler 000000018001b29c     libucrt:new_handler.obj
 0002:000072c0       $unwind$?exit_or_terminate_process@@YAXI@Z 000000018001b2c0     libucrt:exit.obj
 0002:000072cc       $unwind$?common_exit@@YAXHW4_crt_exit_cleanup_mode@@W4_crt_exit_return_mode@@@Z 000000018001b2cc     libucrt:exit.obj
 0002:000072dc       $unwind$??R<lambda_6e4b09c48022b2350581041d5f6b0c4c>@@QEBA@XZ 000000018001b2dc     libucrt:exit.obj
 0002:00007304       $unwind$?fin$0@?0???$?RV<lambda_0ae27a3a962d80f24befdcbee591983d>@@AEAV<lambda_8d0ee55de4b1038c4002e0adecdf1839>@@V<lambda_dc504788e8f1664fe9b84e20bfb512f2>@@@?$__crt_seh_guarded_call@X@@QEAAX$$QEAV<lambda_0ae27a3a962d80f24befdcbee591983d>@@AEAV<lambda_8d0ee55de4b1038c4002e0adecdf1839>@@$$QEAV<lambda_dc504788e8f1664fe9b84e20bfb512f2>@@@Z@4HA 000000018001b304     libucrt:per_thread_data.obj
 0002:00007304       $unwind$?fin$0@?0???$?RV<lambda_2d41944a1d46af3157314b8a01080d33>@@AEAV<lambda_8f455de75cd7d7f24b4096f044d8b9e6>@@V<lambda_aa500f224e6afead328df44964fe2772>@@@?$__crt_seh_guarded_call@X@@QEAAX$$QEAV<lambda_2d41944a1d46af3157314b8a01080d33>@@AEAV<lambda_8f455de75cd7d7f24b4096f044d8b9e6>@@$$QEAV<lambda_aa500f224e6afead328df44964fe2772>@@@Z@4HA 000000018001b304     libucrt:per_thread_data.obj
 0002:00007304       $unwind$?fin$0@?0???$?RV<lambda_aa87e3671a710a21b5dc78c0bdf72e11>@@AEAV<lambda_92619d2358a28f41a33ba319515a20b9>@@V<lambda_6992ecaafeb10aed2b74cb1fae11a551>@@@?$__crt_seh_guarded_call@X@@QEAAX$$QEAV<lambda_aa87e3671a710a21b5dc78c0bdf72e11>@@AEAV<lambda_92619d2358a28f41a33ba319515a20b9>@@$$QEAV<lambda_6992ecaafeb10aed2b74cb1fae11a551>@@@Z@4HA 000000018001b304     libucrt:per_thread_data.obj
 0002:00007304       $unwind$?fin$0@?0???$?RV<lambda_f2e299630e499de9f9a165e60fcd3db5>@@AEAV<lambda_2ae9d31cdba2644fcbeaf08da7c24588>@@V<lambda_40d01ff24d0e7b3814fdbdcee8eab3c7>@@@?$__crt_seh_guarded_call@X@@QEAAX$$QEAV<lambda_f2e299630e499de9f9a165e60fcd3db5>@@AEAV<lambda_2ae9d31cdba2644fcbeaf08da7c24588>@@$$QEAV<lambda_40d01ff24d0e7b3814fdbdcee8eab3c7>@@@Z@4HA 000000018001b304     libucrt:per_thread_data.obj
 0002:00007304       $unwind$?fin$0@?0???$?RV<lambda_410d79af7f07d98d83a3f525b3859a53>@@AEAV<lambda_3e16ef9562a7dcce91392c22ab16ea36>@@V<lambda_38119f0e861e05405d8a144b9b982f0a>@@@?$__crt_seh_guarded_call@X@@QEAAX$$QEAV<lambda_410d79af7f07d98d83a3f525b3859a53>@@AEAV<lambda_3e16ef9562a7dcce91392c22ab16ea36>@@$$QEAV<lambda_38119f0e861e05405d8a144b9b982f0a>@@@Z@4HA 000000018001b304     libucrt:wsetlocale.obj
 0002:00007304       $unwind$?fin$0@?0???$?RV<lambda_751a882b2c74d4b022dec766aa51a29a>@@AEAV<lambda_628dfdc04ba53c8bfc02c9951375f3f5>@@V<lambda_f6c7be5f7998530c34de24c7437d6b54>@@@?$__crt_seh_guarded_call@H@@QEAAH$$QEAV<lambda_751a882b2c74d4b022dec766aa51a29a>@@AEAV<lambda_628dfdc04ba53c8bfc02c9951375f3f5>@@$$QEAV<lambda_f6c7be5f7998530c34de24c7437d6b54>@@@Z@4HA 000000018001b304     libucrt:close.obj
 0002:00007304       $unwind$?fin$0@?0???$?RV<lambda_a37b2b86f63e897a80ea819b0eb08c01>@@AEAV<lambda_38ce7e780aa69e748d6df282ebc68efe>@@V<lambda_99fb1378e971ab6e7edea83e3a7a83a2>@@@?$__crt_seh_guarded_call@H@@QEAAH$$QEAV<lambda_a37b2b86f63e897a80ea819b0eb08c01>@@AEAV<lambda_38ce7e780aa69e748d6df282ebc68efe>@@$$QEAV<lambda_99fb1378e971ab6e7edea83e3a7a83a2>@@@Z@4HA 000000018001b304     libucrt:commit.obj
 0002:00007304       $unwind$?fin$0@?0???$?RV<lambda_efdfa57d1f175319df784efa44bb7b81>@@AEAV<lambda_5f0a4c1567f8adc6734073e5d1e1b35c>@@V<lambda_2e8a7d3640ea6ccb4c2413664c2db6fd>@@@?$__crt_seh_guarded_call@X@@QEAAX$$QEAV<lambda_efdfa57d1f175319df784efa44bb7b81>@@AEAV<lambda_5f0a4c1567f8adc6734073e5d1e1b35c>@@$$QEAV<lambda_2e8a7d3640ea6ccb4c2413664c2db6fd>@@@Z@4HA 000000018001b304     libucrt:mbctype.obj
 0002:00007304       $unwind$?fin$0@?0???$?RV<lambda_450d765d439847d4c735a33c368b5fc0>@@AEAV<lambda_44731a7d0e6d81c3e6aa82d741081786>@@V<lambda_601a2a7da3b7a96e9554ac7215c4b07c>@@@?$__crt_seh_guarded_call@P6AXH@Z@@QEAAP6AXH@Z$$QEAV<lambda_450d765d439847d4c735a33c368b5fc0>@@AEAV<lambda_44731a7d0e6d81c3e6aa82d741081786>@@$$QEAV<lambda_601a2a7da3b7a96e9554ac7215c4b07c>@@@Z@4HA 000000018001b304     libucrt:signal.obj
 0002:00007304       $unwind$?filt$0@?0???R<lambda_6e4b09c48022b2350581041d5f6b0c4c>@@QEBA@XZ@4HA 000000018001b304     libucrt:exit.obj
 0002:00007304       $unwind$?fin$0@?0???$?RV<lambda_d80eeec6fff315bfe5c115232f3240e3>@@AEAV<lambda_6e4b09c48022b2350581041d5f6b0c4c>@@V<lambda_2358e3775559c9db80273638284d5e45>@@@?$__crt_seh_guarded_call@X@@QEAAX$$QEAV<lambda_d80eeec6fff315bfe5c115232f3240e3>@@AEAV<lambda_6e4b09c48022b2350581041d5f6b0c4c>@@$$QEAV<lambda_2358e3775559c9db80273638284d5e45>@@@Z@4HA 000000018001b304     libucrt:exit.obj
 0002:00007304       $unwind$?fin$0@?0???$?RV<lambda_7777bce6b2f8c936911f934f8298dc43>@@AEAV<lambda_f03950bc5685219e0bcd2087efbe011e>@@V<lambda_3883c3dff614d5e0c5f61bb1ac94921c>@@@?$__crt_seh_guarded_call@H@@QEAAH$$QEAV<lambda_7777bce6b2f8c936911f934f8298dc43>@@AEAV<lambda_f03950bc5685219e0bcd2087efbe011e>@@$$QEAV<lambda_3883c3dff614d5e0c5f61bb1ac94921c>@@@Z@4HA 000000018001b304     libucrt:onexit.obj
 0002:00007304       $unwind$?fin$0@?0???$?RV<lambda_842d9ff0dc9ef11c61343bbaebe7f885>@@AEAV<lambda_c5860995281e5c4ce005b3de8f5874ee>@@V<lambda_d90129c13df834fdcbf8d2b88dafcf2d>@@@?$__crt_seh_guarded_call@X@@QEAAX$$QEAV<lambda_842d9ff0dc9ef11c61343bbaebe7f885>@@AEAV<lambda_c5860995281e5c4ce005b3de8f5874ee>@@$$QEAV<lambda_d90129c13df834fdcbf8d2b88dafcf2d>@@@Z@4HA 000000018001b304     libucrt:fflush.obj
 0002:00007304       $unwind$?fin$0@?0???$?RV<lambda_886d6c58226a84441f68b9f2b8217b83>@@AEAV<lambda_ab61a845afdef5b7c387490eaf3616ee>@@V<lambda_f7f22ab5edc0698d5f6905b0d3f44752>@@@?$__crt_seh_guarded_call@X@@QEAAX$$QEAV<lambda_886d6c58226a84441f68b9f2b8217b83>@@AEAV<lambda_ab61a845afdef5b7c387490eaf3616ee>@@$$QEAV<lambda_f7f22ab5edc0698d5f6905b0d3f44752>@@@Z@4HA 000000018001b304     libucrt:fflush.obj
 0002:00007310       $unwind$??$?RV<lambda_d80eeec6fff315bfe5c115232f3240e3>@@AEAV<lambda_6e4b09c48022b2350581041d5f6b0c4c>@@V<lambda_2358e3775559c9db80273638284d5e45>@@@?$__crt_seh_guarded_call@X@@QEAAX$$QEAV<lambda_d80eeec6fff315bfe5c115232f3240e3>@@AEAV<lambda_6e4b09c48022b2350581041d5f6b0c4c>@@$$QEAV<lambda_2358e3775559c9db80273638284d5e45>@@@Z 000000018001b310     libucrt:exit.obj
 0002:00007330       $unwind$??$create_environment@D@@YAQEAPEADQEAD@Z 000000018001b330     libucrt:environment_initialization.obj
 0002:00007340       $unwind$??$?RV<lambda_7777bce6b2f8c936911f934f8298dc43>@@AEAV<lambda_f03950bc5685219e0bcd2087efbe011e>@@V<lambda_3883c3dff614d5e0c5f61bb1ac94921c>@@@?$__crt_seh_guarded_call@H@@QEAAH$$QEAV<lambda_7777bce6b2f8c936911f934f8298dc43>@@AEAV<lambda_f03950bc5685219e0bcd2087efbe011e>@@$$QEAV<lambda_3883c3dff614d5e0c5f61bb1ac94921c>@@@Z 000000018001b340     libucrt:onexit.obj
 0002:00007360       $unwind$terminate          000000018001b360     libucrt:terminate.obj
 0002:00007384       $unwind$abort              000000018001b384     libucrt:abort.obj
 0002:0000738c       $unwind$_invalid_parameter 000000018001b38c     libucrt:invalid_parameter.obj
 0002:0000739c       $unwind$__acrt_getptd      000000018001b39c     libucrt:per_thread_data.obj
 0002:000073ac       $unwind$__acrt_getptd_head 000000018001b3ac     libucrt:per_thread_data.obj
 0002:000073b8       $unwind$??$?RV<lambda_0ae27a3a962d80f24befdcbee591983d>@@AEAV<lambda_8d0ee55de4b1038c4002e0adecdf1839>@@V<lambda_dc504788e8f1664fe9b84e20bfb512f2>@@@?$__crt_seh_guarded_call@X@@QEAAX$$QEAV<lambda_0ae27a3a962d80f24befdcbee591983d>@@AEAV<lambda_8d0ee55de4b1038c4002e0adecdf1839>@@$$QEAV<lambda_dc504788e8f1664fe9b84e20bfb512f2>@@@Z 000000018001b3b8     libucrt:per_thread_data.obj
 0002:000073d8       $unwind$??$?RV<lambda_aa87e3671a710a21b5dc78c0bdf72e11>@@AEAV<lambda_92619d2358a28f41a33ba319515a20b9>@@V<lambda_6992ecaafeb10aed2b74cb1fae11a551>@@@?$__crt_seh_guarded_call@X@@QEAAX$$QEAV<lambda_aa87e3671a710a21b5dc78c0bdf72e11>@@AEAV<lambda_92619d2358a28f41a33ba319515a20b9>@@$$QEAV<lambda_6992ecaafeb10aed2b74cb1fae11a551>@@@Z 000000018001b3d8     libucrt:per_thread_data.obj
 0002:000073f8       $unwind$??$?RV<lambda_f2e299630e499de9f9a165e60fcd3db5>@@AEAV<lambda_2ae9d31cdba2644fcbeaf08da7c24588>@@V<lambda_40d01ff24d0e7b3814fdbdcee8eab3c7>@@@?$__crt_seh_guarded_call@X@@QEAAX$$QEAV<lambda_f2e299630e499de9f9a165e60fcd3db5>@@AEAV<lambda_2ae9d31cdba2644fcbeaf08da7c24588>@@$$QEAV<lambda_40d01ff24d0e7b3814fdbdcee8eab3c7>@@@Z 000000018001b3f8     libucrt:per_thread_data.obj
 0002:00007418       $unwind$??$?RV<lambda_2d41944a1d46af3157314b8a01080d33>@@AEAV<lambda_8f455de75cd7d7f24b4096f044d8b9e6>@@V<lambda_aa500f224e6afead328df44964fe2772>@@@?$__crt_seh_guarded_call@X@@QEAAX$$QEAV<lambda_2d41944a1d46af3157314b8a01080d33>@@AEAV<lambda_8f455de75cd7d7f24b4096f044d8b9e6>@@$$QEAV<lambda_aa500f224e6afead328df44964fe2772>@@@Z 000000018001b418     libucrt:per_thread_data.obj
 0002:00007438       $unwind$??$?RV<lambda_410d79af7f07d98d83a3f525b3859a53>@@AEAV<lambda_3e16ef9562a7dcce91392c22ab16ea36>@@V<lambda_38119f0e861e05405d8a144b9b982f0a>@@@?$__crt_seh_guarded_call@X@@QEAAX$$QEAV<lambda_410d79af7f07d98d83a3f525b3859a53>@@AEAV<lambda_3e16ef9562a7dcce91392c22ab16ea36>@@$$QEAV<lambda_38119f0e861e05405d8a144b9b982f0a>@@@Z 000000018001b438     libucrt:wsetlocale.obj
 0002:0000745c       $unwind$??$__acrt_wcs_to_mbs_cp@U__crt_win32_buffer_internal_dynamic_resizing@@@@YAHQEB_WAEAV?$__crt_win32_buffer@DU__crt_win32_buffer_internal_dynamic_resizing@@@@I@Z 000000018001b45c     libucrt:argv_wildcards.obj
 0002:00007468       $unwind$??$common_expand_argv_wildcards@D@@YAHQEAPEADQEAPEAPEAD@Z 000000018001b468     libucrt:argv_wildcards.obj
 0002:0000747c       $unwind$??$copy_and_add_argument_to_buffer@D@@YAHQEBD0_KAEAV?$argument_list@D@?A0x5f5c8891@@@Z 000000018001b47c     libucrt:argv_wildcards.obj
 0002:00007490       $unwind$??$expand_argument_wildcards@D@@YAHQEAD0AEAV?$argument_list@D@?A0x5f5c8891@@@Z 000000018001b490     libucrt:argv_wildcards.obj
 0002:000074ac       $unwind$__acrt_GetModuleFileNameA 000000018001b4ac     libucrt:getmodulefilenamea.obj
 0002:000074c0       $unwind$??$__acrt_wcs_to_mbs_cp@U__crt_win32_buffer_no_resizing@@@@YAHQEB_WAEAV?$__crt_win32_buffer@DU__crt_win32_buffer_no_resizing@@@@I@Z 000000018001b4c0     libucrt:getmodulefilenamea.obj
 0002:000074cc       $unwind$_setmbcp_nolock    000000018001b4cc     libucrt:mbctype.obj
 0002:000074e4       $unwind$?update_thread_multibyte_data_internal@@YAPEAU__crt_multibyte_data@@QEAU__acrt_ptd@@QEAPEAU1@@Z 000000018001b4e4     libucrt:mbctype.obj
 0002:0000750c       $unwind$?setmbcp_internal@@YAHH_NQEAU__acrt_ptd@@QEAPEAU__crt_multibyte_data@@@Z 000000018001b50c     libucrt:mbctype.obj
 0002:0000751c       $unwind$?setSBUpLow@@YAXPEAU__crt_multibyte_data@@@Z 000000018001b51c     libucrt:mbctype.obj
 0002:00007530       $unwind$??$?RV<lambda_efdfa57d1f175319df784efa44bb7b81>@@AEAV<lambda_5f0a4c1567f8adc6734073e5d1e1b35c>@@V<lambda_2e8a7d3640ea6ccb4c2413664c2db6fd>@@@?$__crt_seh_guarded_call@X@@QEAAX$$QEAV<lambda_efdfa57d1f175319df784efa44bb7b81>@@AEAV<lambda_5f0a4c1567f8adc6734073e5d1e1b35c>@@$$QEAV<lambda_2e8a7d3640ea6ccb4c2413664c2db6fd>@@@Z 000000018001b530     libucrt:mbctype.obj
 0002:00007554       $unwind$__acrt_initialize_lowio 000000018001b554     libucrt:ioinit.obj
 0002:00007578       $unwind$raise              000000018001b578     libucrt:signal.obj
 0002:000075b4       $unwind$??$?RV<lambda_450d765d439847d4c735a33c368b5fc0>@@AEAV<lambda_44731a7d0e6d81c3e6aa82d741081786>@@V<lambda_601a2a7da3b7a96e9554ac7215c4b07c>@@@?$__crt_seh_guarded_call@P6AXH@Z@@QEAAP6AXH@Z$$QEAV<lambda_450d765d439847d4c735a33c368b5fc0>@@AEAV<lambda_44731a7d0e6d81c3e6aa82d741081786>@@$$QEAV<lambda_601a2a7da3b7a96e9554ac7215c4b07c>@@@Z 000000018001b5b4     libucrt:signal.obj
 0002:000075d4       $unwind$??$?RV<lambda_842d9ff0dc9ef11c61343bbaebe7f885>@@AEAV<lambda_c5860995281e5c4ce005b3de8f5874ee>@@V<lambda_d90129c13df834fdcbf8d2b88dafcf2d>@@@?$__crt_seh_guarded_call@X@@QEAAX$$QEAV<lambda_842d9ff0dc9ef11c61343bbaebe7f885>@@AEAV<lambda_c5860995281e5c4ce005b3de8f5874ee>@@$$QEAV<lambda_d90129c13df834fdcbf8d2b88dafcf2d>@@@Z 000000018001b5d4     libucrt:fflush.obj
 0002:000075f4       $unwind$??$?RV<lambda_886d6c58226a84441f68b9f2b8217b83>@@AEAV<lambda_ab61a845afdef5b7c387490eaf3616ee>@@V<lambda_f7f22ab5edc0698d5f6905b0d3f44752>@@@?$__crt_seh_guarded_call@X@@QEAAX$$QEAV<lambda_886d6c58226a84441f68b9f2b8217b83>@@AEAV<lambda_ab61a845afdef5b7c387490eaf3616ee>@@$$QEAV<lambda_f7f22ab5edc0698d5f6905b0d3f44752>@@@Z 000000018001b5f4     libucrt:fflush.obj
 0002:00007618       $unwind$__acrt_update_thread_locale_data 000000018001b618     libucrt:locale_refcounting.obj
 0002:0000763c       $unwind$__acrt_GetStringTypeA 000000018001b63c     libucrt:getstringtypea.obj
 0002:00007658       $unwind$qsort              000000018001b658     libucrt:qsort.obj
 0002:00007678       $unwind$strncpy_s          000000018001b678     libucrt:strncpy_s.obj
 0002:00007684       $unwind$strpbrk            000000018001b684     libucrt:strpbrk.obj
 0002:00007698       $unwind$?__acrt_LCMapStringA_stat@@YAHPEAU__crt_locale_pointers@@PEB_WKPEBDHPEADHHH@Z 000000018001b698     libucrt:lcmapstringa.obj
 0002:000076b8       $unwind$__acrt_lowio_ensure_fh_exists 000000018001b6b8     libucrt:osfinfo.obj
 0002:000076f0       $unwind$??$?RV<lambda_a37b2b86f63e897a80ea819b0eb08c01>@@AEAV<lambda_38ce7e780aa69e748d6df282ebc68efe>@@V<lambda_99fb1378e971ab6e7edea83e3a7a83a2>@@@?$__crt_seh_guarded_call@H@@QEAAH$$QEAV<lambda_a37b2b86f63e897a80ea819b0eb08c01>@@AEAV<lambda_38ce7e780aa69e748d6df282ebc68efe>@@$$QEAV<lambda_99fb1378e971ab6e7edea83e3a7a83a2>@@@Z 000000018001b6f0     libucrt:commit.obj
 0002:00007710       $unwind$_write             000000018001b710     libucrt:write.obj
 0002:00007738       $unwind$_write_nolock      000000018001b738     libucrt:write.obj
 0002:00007754       $unwind$?write_double_translated_ansi_nolock@@YA?AUwrite_result@?A0x17268360@@HQEBDI@Z 000000018001b754     libucrt:write.obj
 0002:00007770       $unwind$?write_text_ansi_nolock@@YA?AUwrite_result@?A0x17268360@@HQEBDI@Z 000000018001b770     libucrt:write.obj
 0002:0000778c       $unwind$?write_text_utf16le_nolock@@YA?AUwrite_result@?A0x17268360@@HQEBDI@Z 000000018001b78c     libucrt:write.obj
 0002:000077a8       $unwind$?write_text_utf8_nolock@@YA?AUwrite_result@?A0x17268360@@HQEBDI@Z 000000018001b7a8     libucrt:write.obj
 0002:000077c4       $unwind$_fcloseall         000000018001b7c4     libucrt:closeall.obj
 0002:000077e8       $unwind$?__mbsrtowcs_utf8@__crt_mbstring@@YA_KPEA_WPEAPEBD_KPEAU_Mbstatet@@@Z 000000018001b7e8     libucrt:mbrtowc.obj
 0002:000077fc       $unwind$fclose             000000018001b7fc     libucrt:fclose.obj
 0002:00007820       $unwind$?__mbrtoc32_utf8@__crt_mbstring@@YA_KPEA_UPEBD_KPEAU_Mbstatet@@@Z 000000018001b820     libucrt:mbrtoc32.obj
 0002:00007830       $unwind$??$?RV<lambda_751a882b2c74d4b022dec766aa51a29a>@@AEAV<lambda_628dfdc04ba53c8bfc02c9951375f3f5>@@V<lambda_f6c7be5f7998530c34de24c7437d6b54>@@@?$__crt_seh_guarded_call@H@@QEAAH$$QEAV<lambda_751a882b2c74d4b022dec766aa51a29a>@@AEAV<lambda_628dfdc04ba53c8bfc02c9951375f3f5>@@$$QEAV<lambda_f6c7be5f7998530c34de24c7437d6b54>@@@Z 000000018001b830     libucrt:close.obj
 0002:00007850       __security_push_cookie_xdata 000000018001b850     LIBCMT:secpushpop.obj
 0002:00007858       __security_push_cookie_xdata_prolog 000000018001b858     LIBCMT:secpushpop.obj
 0002:0000785a       __security_push_cookie_xdata_epilog1 000000018001b85a     LIBCMT:secpushpop.obj
 0002:0000785c       __security_pop_cookie_xdata 000000018001b85c     LIBCMT:secpushpop.obj
 0002:0000785c       __security_push_cookie_xdata_end 000000018001b85c     LIBCMT:secpushpop.obj
 0002:00007864       __security_pop_cookie_xdata_prolog 000000018001b864     LIBCMT:secpushpop.obj
 0002:00007865       __security_pop_cookie_xdata_epilog1 000000018001b865     LIBCMT:secpushpop.obj
 0002:0000786c       __ppgsfailure_xdata        000000018001b86c     LIBCMT:secpushpop.obj
 0002:0000786c       __security_pop_cookie_xdata_end 000000018001b86c     LIBCMT:secpushpop.obj
 0002:00007874       __ppgsfailure_xdata_prolog 000000018001b874     LIBCMT:secpushpop.obj
 0002:00007878       __ppgsfailure_xdata_epilog1 000000018001b878     LIBCMT:secpushpop.obj
 0002:0000787c       $unwind$_IsNonwritableInCurrentImage 000000018001b87c     LIBCMT:pesect.obj
 0002:0000787c       __ppgsfailure_xdata_end    000000018001b87c     LIBCMT:secpushpop.obj
 0002:0000789c       $unwind$_IsNonwritableInCurrentImage$filt$0 000000018001b89c     LIBCMT:pesect.obj
 0002:000078a8       __chkstk_xdata             000000018001b8a8     LIBCMT:chkstk.obj
 0002:000078ac       __chkstk_xdata_prolog      000000018001b8ac     LIBCMT:chkstk.obj
 0002:000078b0       __chkstk_xdata_end         000000018001b8b0     LIBCMT:chkstk.obj
 0002:000078b0       memset_xdata               000000018001b8b0     libvcruntime:memset.obj
 0002:000078b4       memset_xdata_prolog        000000018001b8b4     libvcruntime:memset.obj
 0002:000078b8       memcmp_xdata               000000018001b8b8     libvcruntime:memcmp.obj
 0002:000078b8       memset_xdata_end           000000018001b8b8     libvcruntime:memset.obj
 0002:000078bc       memcmp_xdata_prolog        000000018001b8bc     libvcruntime:memcmp.obj
 0002:000078c0       memcmp_xdata_end           000000018001b8c0     libvcruntime:memcmp.obj
 0002:00007a10       .edata                     000000018001ba10     FarCmds.exp
 0002:00007a38       rgpv                       000000018001ba38     FarCmds.exp
 0002:00007a4c       rgszName                   000000018001ba4c     FarCmds.exp
 0002:00007a60       rgwOrd                     000000018001ba60     FarCmds.exp
 0002:00007a6a       szName                     000000018001ba6a     FarCmds.exp
 0002:00007a76       $N00001                    000000018001ba76     FarCmds.exp
 0002:00007a81       $N00002                    000000018001ba81     FarCmds.exp
 0002:00007a90       $N00003                    000000018001ba90     FarCmds.exp
 0002:00007a9f       $N00004                    000000018001ba9f     FarCmds.exp
 0002:00007aa5       $N00005                    000000018001baa5     FarCmds.exp
 0002:00008126       .idata$6                   000000018001c126     kernel32:KERNEL32.dll
 0002:00008176       .idata$6                   000000018001c176     advapi32:ADVAPI32.dll
 0002:000081ae       .idata$6                   000000018001c1ae     user32:USER32.dll
 0002:000081f0       .idata$6                   000000018001c1f0     ole32:ole32.dll
 0002:0000820c       .idata$6                   000000018001c20c     rpcrt4:RPCRT4.dll
 0003:00000014       ?__vcrt_flsindex@@3KA      000000018001d014     libvcruntime:per_thread_data.obj
 0003:0000001c       ?errno_no_memory@@3HA      000000018001d01c     libucrt:errno.obj
 0003:00000020       ?doserrno_no_memory@@3KA   000000018001d020     libucrt:errno.obj
 0003:00000024       ?__acrt_flsindex@@3KA      000000018001d024     libucrt:per_thread_data.obj
 0003:000003d0       _mbctypes                  000000018001d3d0     libucrt:mbctype.obj
 0003:000004e0       _mbcasemaps                000000018001d4e0     libucrt:mbctype.obj
 0003:000005e0       ?__rgctypeflag@@3PADA      000000018001d5e0     libucrt:mbctype.obj
 0003:000005f0       ?__rgcode_page_info@@3PAUcode_page_info@@A 000000018001d5f0     libucrt:mbctype.obj
 0003:00000990       ?__dcrt_lowio_console_output_handle@@3PEAXEA 000000018001d990     libucrt:initcon.obj
 0003:000009a0       ?OptName@@3UOptionsName@@A 000000018001d9a0     FARCmds.obj
 0003:000009d0       ?PRI@?7??OpenW@@9@4UPanelRedrawInfo@@A 000000018001d9d0     FARCmds.obj
 0003:000009f0       ?Pref@?7??OpenFromCommandLine@@YAPEA_WPEB_W@Z@4PAU<unnamed-type-Pref>@?7??1@YAPEA_W0@Z@A 000000018001d9f0     OpenCmd.obj
 0003:00000ad0       ?mode@?1??GetStreamAndMode@@YAXAEAPEA_WAEAH1@Z@4PAU<unnamed-type-mode>@?1??1@YAX011@Z@A 000000018001dad0     OpenCmd.obj
 0003:00000c70       ?__proc_attached@@3HA      000000018001dc70     LIBCMT:dll_dllmain.obj
 0003:00000c80       GS_ExceptionRecord         000000018001dc80     LIBCMT:gs_report.obj
 0003:00000d20       GS_ContextRecord           000000018001dd20     LIBCMT:gs_report.obj
 0003:000010d4       ?is_initialized_as_dll@@3_NA 000000018001e0d4     LIBCMT:utility.obj
 0003:000010e0       ?module_local_atexit_table@@3U_onexit_table_t@@A 000000018001e0e0     LIBCMT:utility.obj
 0003:000010f8       ?module_local_at_quick_exit_table@@3U_onexit_table_t@@A 000000018001e0f8     LIBCMT:utility.obj
 0003:00001110       ?module_local_atexit_table_initialized@@3_NA 000000018001e110     LIBCMT:utility.obj
 0003:00001130       ?__vcrt_startup_thread_ptd@@3U__vcrt_ptd@@A 000000018001e130     libvcruntime:per_thread_data.obj
 0003:000011b8       ?heap@@3V_HeapManager@@A   000000018001e1b8     libvcruntime:undname.obj
 0003:00001220       __vcrt_lock_table          000000018001e220     libvcruntime:locks.obj
 0003:00001248       __vcrt_locks_initialized   000000018001e248     libvcruntime:locks.obj
 0003:00001250       ?__acrt_new_handler@@3V?$dual_state_global@P6AH_K@Z@__crt_state_management@@A 000000018001e250     libucrt:new_handler.obj
 0003:00001258       ?c_termination_complete@@3JA 000000018001e258     libucrt:exit.obj
 0003:00001260       ?thread_local_exit_callback_func@@3P6AXPEAXK0@ZEA 000000018001e260     libucrt:exit.obj
 0003:00001270       ?program_name@?1???$common_configure_argv@D@@YAHW4_crt_argv_mode@@@Z@4PADA 000000018001e270     libucrt:argv_parsing.obj
 0003:000013c8       ?__acrt_invalid_parameter_handler@@3V?$dual_state_global@P6AXPEB_W00I_K@Z@__crt_state_management@@A 000000018001e3c8     libucrt:invalid_parameter.obj
 0003:000013e0       ?__acrt_lock_table@@3PAU_RTL_CRITICAL_SECTION@@A 000000018001e3e0     libucrt:locks.obj
 0003:00001610       ?__acrt_locks_initialized@@3IA 000000018001e610     libucrt:locks.obj
 0003:00001630       ?fSystemSet@@3HA           000000018001e630     libucrt:mbctype.obj
 0003:00001634       ?initialized@?1??__acrt_initialize_multibyte@@9@4_NA 000000018001e634     libucrt:mbctype.obj
 0003:00001670       ?module_handles@@3PAPEAUHINSTANCE__@@A 000000018001e670     libucrt:winapi_thunks.obj
 0003:00001710       ?encoded_function_pointers@@3PAPEAXA 000000018001e710     libucrt:winapi_thunks.obj
 0003:00001c38       ?ctrlc_action@@3V?$dual_state_global@P6AXH@Z@__crt_state_management@@A 000000018001ec38     libucrt:signal.obj
 0003:00001c40       ?ctrlbreak_action@@3V?$dual_state_global@P6AXH@Z@__crt_state_management@@A 000000018001ec40     libucrt:signal.obj
 0003:00001c48       ?abort_action@@3V?$dual_state_global@P6AXH@Z@__crt_state_management@@A 000000018001ec48     libucrt:signal.obj
 0003:00001c50       ?term_action@@3V?$dual_state_global@P6AXH@Z@__crt_state_management@@A 000000018001ec50     libucrt:signal.obj
 0003:00001c58       ?user_matherr@@3V?$dual_state_global@P6AHPEAU_exception@@@Z@__crt_state_management@@A 000000018001ec58     libucrt:matherr.obj
 0003:00001c80       ?internal_state@?1??_mbtowc_l@@9@4U_Mbstatet@@A 000000018001ec80     libucrt:mbtowc.obj
 0003:00001c88       ?__acrt_global_new_mode@@3V?$dual_state_global@J@__crt_state_management@@A 000000018001ec88     libucrt:new_mode.obj
 0003:00001c94       ?__acrt_app_type@@3W4_crt_app_type@@A 000000018001ec94     libucrt:report_runtime_error.obj
 0003:00001c98       ?internal_pst@?1??__mbrtoc32_utf8@__crt_mbstring@@YA_KPEA_UPEBD_KPEAU_Mbstatet@@@Z@4U3@A 000000018001ec98     libucrt:mbrtoc32.obj
 0003:00001f68       ?PluginConfigStrings@?1??GetPluginInfoW@@9@4PAPEB_WA 000000018001ef68     FARCmds.obj
 0003:00001f70       ?farcmdbuf@?1??OpenFromCommandLine@@YAPEA_WPEB_W@Z@4PA_WA 000000018001ef70     OpenCmd.obj
 0005:00000060       $R000000                   0000000180024060     FarCmds.res
